:100000005EC700008DC700008BC7000089C70000D5
:1000100087C7000085C7000083C7000081C70000B4
:100020007FC700007DC700007BC7000079C70000C4
:1000300077C700000C94084273C7000071C7000026
:100040006FC700006DC700006BC7000069C70000E4
:1000500067C7000065C7000063C700000C94644DCB
:100060005FC700000C94124C0C94E94B59C7000078
:1000700057C7000055C7000053C7000051C7000014
:100080004FC700004DC700004BC7000049C7000024
:1000900047C7000045C7000043C700000C941C433D
:1000A0003FC700003DC700003BC7000039C7000044
:1000B00037C7000035C7000033C7000031C7000054
:1000C0002FC700002DC700002BC700000C94C04BA9
:1000D0000C94974B25C700000C946E4B0C94454B29
:1000E0001FC70000DC30BE30E830E830E830E830D0
:1000F000E830E830E830E830E830E830CF1D202143
:1001000082238A23412454250F2713288B28A028D3
:10011000A428E830A928AD2A952BB22C292E2C2E04
:100120009C2EA32E1F2F7D2F8330C148C448B34877
:10013000B748BD48FB48C848CC48D248D648DA48FA
:10014000E048E448E848FB48EE48F248F648084AE8
:10015000D73B3BCE016E84BCBFFDC12F3D6C7431DB
:100160009ABD56833DDA3D00C77F11BED9E4BB4C32
:100170003E916BAAAABE000000803F07634236B7DB
:100180009BD8A71A39685618AEBAAB558C1D3CB728
:10019000CC5763BD6DEDFD753EF6177231BF0000A3
:1001A00000803F08000000BE922449123EABAAAA7C
:1001B0002ABECDCCCC4C3E00000080BEABAAAAAA81
:1001C0003E00000000BF000000803F000000000073
:1001D000084178D3BB4387D1133D190E3CC3BD42C0
:1001E00082AD2B3E68EC8276BED98FE1A93E4C8071
:1001F000EFFFBE01C4FF7F3F0000000000004E4142
:100200004E494E495459494E46CDCCCC3D0AD72390
:100210003C17B7D13877CC2B329595E6241FB14FD8
:100220000A000020410000C84200401C4620BCBE1D
:100230004CCA1B0E5AAEC59D7400407A10F35A008A
:10024000A0724E18090010A5D4E80000E8764817FF
:100250000000E40B54020000CA9A3B000000E1F5E4
:1002600005000080969800000040420F000000A0AA
:100270008601000000102700000000E803000000D5
:10028000006400000000000A0000000000010000FF
:100290000000002C76D888DC674F0823DFC1DFAE72
:1002A00059E1B1B796E5E3E453C63AE6519976963B
:1002B000E8E6C28426EB898C9B62ED407C6FFCEF04
:1002C000BC9C9F40F2BAA56FA5F490055A2AF75C32
:1002D000936B6CF9676DC11BFCE0E40D47FEF520E4
:1002E000E6B500D0ED902E030094357705008084AC
:1002F0001E080000204E0A000000C80C33333333C0
:100300000F986E12831141EF8D2114893BE655162B
:10031000CFFEE6DB18D1844B381BF77C1D901DA463
:10032000BBE424203284725E228100C9F124ECA156
:10033000E53D27616E6F7468657220495220696ED1
:100340007075743D00696E70757420445354636118
:100350006C6962726174653A0020766F6C746167D3
:10036000653D0054757262696469747920557070D6
:100370006572204C696D69743A200020766F6C7448
:100380006167653D00547572626964697479204CD7
:100390006F776572204C696D69743A2000547572EC
:1003A000626964697479204C6F776572204C696D5D
:1003B00069742056696E663A2000434F32204D41E1
:1003C0005820766F6C74202800434F32207A657273
:1003D0006F20766F6C742028004F322063616C6947
:1003E00062726174696F6E3A20005475726269645A
:1003F000697479204C6F776572204C696D6974203F
:1004000056313A200023506172616D6574657273D4
:10041000003E4D6F74696F6E20627920756C747246
:1004200061736F6E632073656E736F723A0A004E6C
:100430006F20445320546865726D6F6D65746572EA
:1004400021004F3220436F6E6300434F3220436FD1
:100450006E630053656E736F72206572726F7221E6
:1004600000234E6F2073656E736F722100434F320D
:1004700020436F6E63004D6561737572696E67002E
:10048000234E6F2073656E736F7220666F722050FB
:100490004D21004E6F2073656E736F722100504DB9
:1004A000313A322E353A3130004D656173757269DB
:1004B0006E672E2E00547572626964697479002328
:1004C0003A53686F772F48696465204C4344002A8B
:1004D0003A546869732048656C700044433A436C31
:1004E000656172204C43440044423A52657365741E
:1004F000204C6F676765720044373A4D6F74696FBF
:100500006E0044363A44532054656D700044353AC9
:10051000555620496E74656E736974790044343A97
:100520004F3220636F6E632E0044333A434F3220C4
:10053000636F6E632E0044323A504D28313A322EAA
:10054000353A3130290044323A504D28313A322E72
:10055000353A3130292A0044313A5475726269645F
:100560006974790044303A566F6C7461676500397C
:100570003A6F7220334420616363656C2E00393A10
:10058000496E636C2E20616E672E00383A704820E9
:1005900076616C756500373A49522054656D70007C
:1005A000373A49522054656D702A00363A4D6167DA
:1005B0006E65746963206669656C6400353A4761ED
:1005C00073204C6576656C00343A495220466C6164
:1005D0006D6500333A4C6967687420496E742E006B
:1005E000323A616E642048656967687400323A5433
:1005F000656D7020507265737375726500313A5481
:10060000656D702048756D696469747900303A537E
:100610006F756E64204C6576656C00303A536F756B
:100620006E64204C6576656C2A00234E6F207365DE
:100630006E736F7220666F722074656D7020262055
:1006400068756D696469747921004E6F2053656E19
:10065000736F72210054656D702048756D6964690F
:10066000747900466C616D65204952004E6F2073AD
:10067000656E736F72210049522054656D7065720A
:100680006174757265004D6561737572696E672E70
:100690002E0070482076616C756500496E76616C3D
:1006A0006964206B657921007265706C6965733DC2
:1006B0000067657453656C66546573744269742889
:1006C000293A20006973496E7465727275707445B9
:1006D0006E61626C65642831293A2000676574494F
:1006E0006E746572727570744D617070696E672892
:1006F00031293A2000676574496E746572727570AD
:1007000074536F757263652831293A2000676574E8
:10071000496E74657272757074536F757263652873
:10072000293A20006765745261746528293A20339C
:100730002E31343135393F00616363656C2E697346
:100740004C6F77506F77657228293A200061636398
:10075000656C2E697341736C65657028293A2000B9
:10076000616363656C2E6973546170536F75726356
:10077000654F6E5A28293A2000616363656C2E69C3
:1007800073546170536F757263654F6E5928293ABF
:100790002000616363656C2E6973546170536F75DB
:1007A0007263654F6E5828293A2000616363656C57
:1007B0002E69734163746976697479536F757263D6
:1007C000654F6E5A28293A2000616363656C2E6973
:1007D000734163746976697479536F757263654F99
:1007E0006E5928293A2000697341637469766974E7
:1007F00079536F757263654F6E5828293A200069E6
:1008000073546170446574656374696F6E4F6E5A9A
:1008100028293B2066616C73653F20006973546131
:1008200070446574656374696F6E4F6E5A28293B16
:1008300020747275653F200069735461704465745B
:10084000656374696F6E4F6E5928293B2066616C31
:1008500073653F2000697354617044657465637407
:10086000696F6E4F6E5928293B20747275653F2061
:10087000006973546170446574656374696F6E4F89
:100880006E5828293B2066616C73653F20006973B0
:10089000546170446574656374696F6E4F6E582857
:1008A000293B20747275653F20006765745375702D
:1008B000707265737342697428293B2066616C739A
:1008C000653F20006765745375707072657373427D
:1008D000697428293B20747275653F200069734153
:1008E00063746976697479416328293A20006973D1
:1008F000496E61637469766974795A456E61626C98
:10090000656428293A20006973496E6163746976C9
:1009100069747959456E61626C656428293A2000D2
:100920006973496E616374697669747958456E615B
:10093000626C656428293A200069734163746976A2
:100940006974795A456E61626C656428293A2000A1
:100950006973416374697669747959456E61626C33
:10096000656428293A200069734163746976697463
:100970007958456E61626C656428293A2000676584
:10098000744672656546616C6C4475726174696F1A
:100990006E28293A20006765744672656546616C69
:1009A0006C5468726573686F6C6428293A2000671C
:1009B000657454696D65496E6163746976697479AB
:1009C00028293A2000676574496E61637469766905
:1009D00074795468726573686F6C642829200067A5
:1009E0006574416374697669747954687265736873
:1009F0006F6C6428292000676574446F75626C65AC
:100A000054617057696E646F772829200067657498
:100A1000446F75626C655461704C6174656E637986
:100A200028293A20006765745461704475726174B6
:100A3000696F6E28293A2000676574417869734FA1
:100A400066667365742826782C2026792C20267AF1
:100A5000293A200067657454617054687265736840
:100A60006F6C6428293A200058595A2047733A205D
:100A70000058595A20434F554E54533A200073653D
:100A800074206761696E735B5D3A006761696E73BC
:100A90005F6F7269675B5D3A00005EBCE2613FDDDB
:100AA00083C29C7E20A3FD1F41009D23BE46DB65C3
:100AB000F88C11AF32CA57E9742343616C696272D2
:100AC0006174696F6E2050726573737572653D0055
:100AD00023536561206C6576656C20502863616CDA
:100AE00063293D00234572726F723A7072657373A9
:100AF00075726520424D503038352C20636865632F
:100B00006B20776972696E67210049522054656DC8
:100B1000702073656E736F7220666F756E6400501F
:100B20004D322E352073656E736F72206C696B6564
:100B30006C7920666F756E6400536F756E64204C1F
:100B40006576656C2073656E736F7220666F756E67
:100B5000640053656E736F7220736C6F7420616EE6
:100B60006420747970653A00000021002400270099
:100B70002A002D00300033000101000004010701AC
:100B80000A0100002200250028002B002E00310061
:100B9000340002010000050108010B0100002000E3
:100BA0002300260029002C002F0032000001000045
:100BB00003010601090105050505070508080808E0
:100BC000020202020A0A08080404040401010101E5
:100BD00001010101030303030303030304070707E0
:100BE0000C0C0C0C0C0C0C0C020202020606060685
:100BF000060606060B0B0B0B0B0B0B0B0102102052
:100C00002008081020401020408002010201080442
:100C100002010102040810204080804020100804D6
:100C2000020180040201804020100804020108042F
:100C30000201010204081020408001020408102073
:100C4000408000000A0B02090C0D0E080703040186
:100C50000000000000000000000000000000000094
:100C60000000000000000000000000000000121161
:100C70001000000000000000000000000000000064
:100C800000000000000000005072657373206120B6
:100C90006B6579004C4344206F6E006B6579323D83
:100CA000006B6579323D004F6666206169722D6385
:100CB0006F6E6421004974277320746F6F20636F17
:100CC0006F6C210054656D702069732066696E65D4
:100CD00021004973206169722D636F6E64206F6E0D
:100CE0003F004974277320717569746520686F74BB
:100CF000210049742773207665727920686F74210A
:100D000020004F6666206169722D636F6E6421005A
:100D10004974277320746F6F20636F6F6C210054C8
:100D2000656D702069732066696E652100497320C6
:100D30006169722D636F6E64206F6E3F0049742786
:100D40007320717569746520686F74210049742778
:100D500073207665727920686F74210054656D7018
:100D60002048756D696469747900416E676C6573BC
:100D70002F004C6967687420496E74656E736974DE
:100D800079004572726F72206E756D6265722066B1
:100D90006F722074686520617272617920746F20AF
:100DA0006176726167696E67212F6E002D2D2D2D82
:100DB0002D2D2D2D2D2D2D2D2D2D2D2D2D2D2D2D63
:100DC0002D2D2D2D2D2D2D2D2D2D2D2D2D2D2D2D53
:100DD000005265736F6C7574696F6E3A2020200045
:100DE0004D696E2056616C75653A20202020004DBB
:100DF00061782056616C75653A2020202000556E80
:100E0000697175652049443A2020202000447269A8
:100E1000766572205665723A2020200053656E7305
:100E20006F723A20202020202020002D2D2D2D20F3
:100E30004D61676E657469632053656E736F7220D0
:100E40002D2D2D2D2D2D2D2D2D2D2D2D2D2D2D2DD2
:100E50002D2D2D2D0020202020202020202020207E
:100E600020202020200020202020202020202020A2
:100E70002020202020200020202020202020202092
:100E80002020202020202000202020202020202082
:100E90002020202020202020002020202020202072
:100EA0002020202020202020002020202020202062
:100EB00020202020202020200000897D267D112454
:100EC0001FBECFEFD1E2DEBFCDBF00E00CBF1AE006
:100ED000A0E0B2E0ECE7F8E101E00BBF02C0079050
:100EE0000D92A03AB107D9F720E1A0EABAE001C01B
:100EF0001D92A13AB207E1F717E0CEE5D7E000E096
:100F000006C021970109802FFE010E949289CD35EC
:100F1000D10780E00807A9F70E9437770C942D8C41
:100F20006FC82F923F924F925F926F927F928F92F3
:100F30009F92AF92BF92CF92DF92EF92FF920F9368
:100F40001F93CF93DF93CDB7DEB7EA970FB6F89430
:100F5000DEBF0FBECDBF8AEB9AE00E94D332892B51
:100F600009F45AC20E9428560E9455746BE679E033
:100F7000CE0101960E943A4A4AE050E060E070E0FB
:100F8000CE0101960E94EC75CE0101960E94894621
:100F90004091BE0A5091BF0A6091C00A7091C10A87
:100FA00020E182E59DE00E949C4A82E59DE00E944E
:100FB000314B8091BE0A9091BF0AA091C00AB091B6
:100FC000C10A883025E09207A105B10509F401C2E4
:100FD00008F08DC0893461E09607A105B10509F4D8
:100FE000FBC1E0F58434E1E09E07A105B10509F4F9
:100FF000E4C1E8F4813421E09207A105B10509F4C8
:10100000CDC138F480349140A105B10509F4B7C1D0
:10101000E6C1823471E09707A105B10509F4C7C1A3
:1010200083349140A105B10509F4C4C1D8C1863407
:10103000F1E09F07A105B10509F4C5C108F4C0C1DD
:10104000873441E09407A105B10509F4BFC1883494
:101050009140A105B10509F4BCC1C1C1823075E060
:101060009707A105B10509F4A2C1E8F48437F1E0BE
:101070009F07A105B10509F44DC138F482379140AD
:10108000A105B10509F451C1AAC1811565E0960712
:10109000A105B10509F473C181309540A105B105E1
:1010A00009F47CC19CC18530E5E09E07A105B1052E
:1010B00009F486C170F4833025E09207A105B105DB
:1010C00009F478C184309540A105B10509F475C1D2
:1010D00086C1863065E09607A105B10509F473C1A4
:1010E00087309540A105B10509F470C178C18D3BE9
:1010F000E2E49E07EFEFAE07B10509F431C108F055
:101100004BC08F3E20E192072FEFA207B10509F4F3
:101110005DC118F5823365E09607A105B10509F4B4
:1011200004C138F489309540A105B10509F454C1D2
:1011300056C18433F5E09F07A105B10509F4EAC063
:101140008D3F9240AF4FB10509F049C164E775E0AA
:101150008BEE9EE00E945F46E5C08D3D42E2940723
:101160004FEFA407B10509F4D5C038F4873E984184
:10117000AF4FB10509F424C132C18F3CE0E39E07B3
:10118000EFEFAE07B10509F418C1873C9843AF4FA4
:10119000B10509F41EC123C1873928E692072FEF54
:1011A000A207B10509F4FAC048F58D3A62E5960741
:1011B0006FEFA607B10509F4C4C038F4853B9A4423
:1011C000AF4FB10509F4DBC00AC1853AFAE59F07C4
:1011D000FFEFAF07B10509F4FFC08D399246AF4F5D
:1011E000B10509F0FCC061E775E08BEE9EE00E945E
:1011F0005F461092770B8CEF9FEF89C0873548EAE6
:1012000094074FEFA407B105F9F078F485387AE731
:1012100097077FEFA707B10509F4D5C0873698492E
:10122000AF4FB10509F4C3C0DAC08F34F0EB9F07AC
:10123000FFEFAF07B10509F4BDC08D33924CAF4F3E
:10124000B10509F472C0CBC082E08093FB0D10920F
:10125000FE0D00E010E080EA9AE00E94D332892B74
:1012600069F40F5F1F4F093E43E0140739F06EE148
:1012700070E080E090E00E94204DEDCF63E373E0EA
:1012800082E59DE00E94634A4091A40A5091A50A1C
:101290006091A60A7091A70A2AE082E59DE00E946B
:1012A0009C4A82E59DE00E94314B8091A40A909176
:1012B000A50AA091A60AB091A70A853045E0940737
:1012C000A105B10509F497C108F09EC1873471E00A
:1012D0009707A105B10509F4B7C108F0B8C1833477
:1012E000F1E09F07A105B10509F4C1C108F07CC177
:1012F000813441E09407A105B10509F0C1C160E660
:1013000075E085EE9EE00E945F4689EF9FEF0E94A8
:10131000591D7CC064E775E08BEE9EE00E945F463D
:101320001092770B8BEF9FEFF2CF67E775E08BEEB4
:101330009EE00E945F4681E08093770B8DEF9FEFE8
:10134000E6CF6AE775E085EE9EE00E945F466AE7B9
:1013500075E08BEE9EE00E945F468EEF9FEFD7CF49
:101360006DE775E085EE9EE00E945F466DE775E0F3
:101370008BEE9EE00E945F468FEF9FEFC8CF6BE63B
:1013800075E085EE9EE00E945F466BE675E08BEEB1
:101390009EE00E945F4680E090E0B9CF6EE775E086
:1013A00085EE9EE00E945F4681E090E0B0CF82E053
:1013B00090E0ADCF83E090E0AACF84E090E0A7CFAB
:1013C00085E090E0A4CF86E090E0A1CF87E090E0B8
:1013D0009ECF88E090E09BCF89E090E098CF60E0DE
:1013E00070E0CE0101960E94875FBE016F5F7F4F64
:1013F00085EE9EE00E940746CE0101960E94894636
:1014000064E670E080E090E00E94204D82E08093EE
:10141000FB0D1092FE0DB3C069EC79E08BEE9EE0FF
:101420000E945F461092B10A69EC79E08BEE9EE073
:101430000E945F4601E082E59DE00E94C94720913D
:10144000B10A181619060CF096C1211194C10FC2E9
:1014500040910002509101026091020270910302DA
:1014600022E0CE0145960E94BD466FE676E0CE01B1
:1014700001960E943A4ABE016B5E7F4FCE010196F3
:101480000E94BC4562E278E00E94A545BC01CE0105
:1014900083960E944B47CE0183960E947367CE01CC
:1014A00083960E948946CE0101960E948946CE010C
:1014B00045960E94894640910C0250910D02609120
:1014C0000E0270910F0222E0CE0145960E94BD46A9
:1014D0006FE776E0CE0101960E943A4ABE016B5E4C
:1014E0007F4FCE0101960E94BC4562E278E00E94E7
:1014F000A545BC01CE0183960E944B47CE01839641
:101500000E947367CE0183960E948946CE010196A0
:101510000E948946CE0145960E948946B12C0E94C0
:1015200028560E9455746BE679E0CE0101960E9420
:101530003A4A4AE050E060E070E0CE0101960E9435
:101540003A75CE0101960E9489468091EF0E9091E6
:10155000F00E8330910508F0C7C58130910509F080
:1015600056C5E091EB0EF091EC0E309711F40C940F
:10157000331D1081812F0E947F680E94584D0E9468
:10158000584D6093B60A7093B70A8093B80A909347
:10159000B90A1CC08091770B81110C94DD1C0E944C
:1015A000584D0091B60A1091B70A2091B80A3091AF
:1015B000B90ADC01CB01801B910BA20BB30B883461
:1015C0009E4EA105B10510F00E941C568091770B2C
:1015D000882311F40C94401D64E670E080E090E0F4
:1015E0000E94204D0C94401D853471E09707A105A1
:1015F000B10509F054C06DE675E085EE9EE00E94ED
:101600005F4685EF9FEF83CE8F3CF0E39F07FFEFB0
:10161000AF07B10509F448C008F04FC0883045E075
:101620009407A105B10509F46FC008F080C08630A9
:1016300075E09707A105B10509F45DC087309540B5
:10164000A105B10509F0DCCE83EF9FEF60CE8130BC
:10165000F5E09F07A105B10509F451CE08F44EC08D
:10166000833075E09707A105B10509F059C066E61A
:1016700075E085EE9EE00E945F4687EF9FEF47CEC4
:1016800082349140A105B10509F0BACE63E675E058
:1016900085EE9EE00E945F4688EF9FEF38CE86344D
:1016A0009140A105B10538F569E675E085EE9EE04B
:1016B0000E945F4686EF9FEF2ACE873968E696073D
:1016C0006FEFA607B10509F41ACE08F447C08736B4
:1016D00028E992072FEFA207B105C1F28F3440EB42
:1016E00094074FEFA407B10511F285389A47AF4F21
:1016F000B10509F085CE84EF9FEF09CE883441E033
:101700009407A105B10519F482EF9FEF00CE89344B
:101710009140A105B10509F073CE81EF9FEFF7CDA0
:1017200084309540A105B10508F4B0CFBDCF8F3E00
:10173000F0E19F07FFEFAF07B10509F485CF873EC2
:1017400028E192072FEFA207B10509F454CF8930A1
:101750009540A105B10509F053CEDFCF873CE8E302
:101760009E07EFEFAE07B10579F2853A9A45AF4F84
:10177000B10599F245CE222361F02091B10A809102
:10178000EF0E9091F00E2111A6C0009709F0A3C0B2
:10179000E2C0E12CF12C01E088E19CE00E94C94705
:1017A00018161906DCF588E19CE00E94A747809393
:1017B000B00A8A30A9F08D3099F09091B10A911158
:1017C0000FC089831A8241E050E0BE016F5F7F4FF6
:1017D0008BEE9EE00E9478456FEFE61AF60A17C07E
:1017E0008091EF0E9091F00E892B89F00093B10A51
:1017F00088E19CE00E94C9471816190644F469EC78
:1018000079E08BEE9EE00E945F461092B10A6FE095
:1018100070E080E090E00E94204DBECF62E370E077
:1018200080E090E00E94204DEF2809F4A6CF69E8FF
:1018300075E0CE0101960E943A4A6BEE7EE0CE0141
:1018400001960E94BC45BC0182E59DE00E94344B9C
:10185000CE0101960E94894688E19CE00E9457488B
:1018600064E670E080E090E00E94204D86CF82E543
:101870009DE00E94A7478093B00A8A3071F08D30B6
:1018800061F089831A8241E050E0BE016F5F7F4FB3
:101890008BEE9EE00E94784517C00093B10A60E885
:1018A00075E0CE0101960E943A4A6BEE7EE0CE01D1
:1018B00001960E94BC45BC0182E59DE00E94344B2C
:1018C000CE0101960E9489466AE070E080E090E0D7
:1018D0000E94204DB0CD019709F058C062E278E037
:1018E000CE0101960E943A4ACE0101960E943B52D7
:1018F000811112C06EE875E0CE0145960E943A4A09
:10190000CE0145960E943B5201E0811100E0CE01DC
:1019100045960E94894601C000E0CE0101960E94D2
:101920008946002389F060E070E0CE0101960E94B4
:10193000875FBE016F5F7F4F85EE9EE00E94074686
:10194000CE0101960E94894664E170E080E090E05B
:101950000E94204D1BC064E670E080E090E00E9491
:10196000204D0E94584DCB0168EE73E00E947F89A4
:10197000CB0164E670E00E947F898236910534F0E5
:101980008091770B882311F40C94241D6AE070E099
:1019900080E090E00E94204D8091EF0E9091F00E3B
:1019A000009711F40C94BC1C0197E1F560E975E017
:1019B000CE0183960E943A4ACE0183960E943B5202
:1019C00081110C943A1D65EF78E0CE0145960E9496
:1019D0003A4ACE0145960E943B52811112C069E5F8
:1019E00079E0CE0101960E943A4ACE0101960E940A
:1019F0003B5201E0811100E0CE0101960E94894630
:101A000001C000E0CE0145960E948946CE01839632
:101A10000E948946002331F06BEE7EE085EE9EE069
:101A20000E9474468091EF0E9091F00E0497E8F5B5
:101A300062E975E0CE0101960E943A4ACE01019614
:101A40000E943B52082FCE0101960E948946002336
:101A500061F161E070E0CE0101960E94875FCE01E6
:101A600001960E940E452AEFC22EDD24DA94ED2C59
:101A7000FD2C46015701861A970AA80AB90AB50132
:101A8000A4012AE0CE0145960E94EC46BE016B5EA1
:101A90007F4F85EE9EE00E940746CE0145960E944C
:101AA0008946CE0101960E94894664E975E0CE011F
:101AB00045960E943A4ACE0145960E943B528111BA
:101AC00013C068E975E0CE0101960E943A4ACE0142
:101AD00001960E943B5201E0811101C000E0CE015D
:101AE00001960E94894601C001E0CE0145960E9400
:101AF0008946002309F488C265E074E0CE010196AE
:101B00000E944347CE0101960E947367CE01019661
:101B10000E9489466091430270914402809145027F
:101B2000909146020E94B48420E030E048EC52E4F8
:101B30000E940487AB01BC0122E0CE0145960E94C1
:101B4000BD466CE975E0CE0101960E943A4ABE019D
:101B50006B5E7F4FCE0101960E94BC4560EC76E043
:101B60000E94A545BC01CE0183960E944B47CE0141
:101B700083960E947367CE0183960E948946CE01A8
:101B800001960E948946CE0145960E948946409161
:101B90003F0250914002609141027091420224E064
:101BA000CE0145960E94BD4661EB75E0CE010196DF
:101BB0000E943A4ABE016B5E7F4FCE0101960E94A1
:101BC000BC45BC01CE0183960E944B47CE01839653
:101BD0000E947367CE0183960E948946CE010196CA
:101BE0000E948946CE0145960E9489464091330263
:101BF00050913402609135027091360222E0CE019C
:101C00008F960E94BD4640912B0250912C0260910C
:101C10002D0270912E0223E0CE0189960E94BD46CE
:101C200040913702509138026091390270913A0226
:101C300022E0CE0183960E94BD4640912F02509132
:101C40003002609131027091320223E0CE0145965C
:101C50000E94BD466EEC75E0CE0101960E943A4AA4
:101C6000BE016B5E7F4FCE0101960E94BC4563EEC4
:101C700075E00E94A545BE016D5D7F4F0E94BC4589
:101C800066EE75E00E94A545BE01675D7F4F0E942C
:101C9000BC4563EE75E00E94A545BE01615D7F4FC6
:101CA0000E94BC456CEE75E00E94A545BC01CE01CA
:101CB000C5960E944B47CE01C5960E947367CE0120
:101CC000C5960E948946CE0101960E948946CE01A2
:101CD00045960E948946CE0183960E948946CE0190
:101CE00089960E948946CE018F960E94894661EFAF
:101CF00075E0CE0101960E943A4A65EC7FE0CE0184
:101D000001960E94BC45BC01CE0145960E944B47FE
:101D1000CE0145960E947367CE0145960E94894682
:101D2000CE0101960E9489464091C0045091C104A1
:101D30006091C2047091C30423E0CE0183960E9497
:101D4000BD462091B8043091B9044091BA04509135
:101D5000BB0460E070E080E291E40E94B288AB01D5
:101D6000BC0121E0CE0145960E948E4662E076E0FD
:101D7000CE0101960E943A4ABE016B5E7F4FCE01B2
:101D800001960E94BC4565E176E00E94A545BE0132
:101D90006D5D7F4F0E94BC456BE176E00E94A545DA
:101DA000BC01CE0189960E944B47CE0189960E94C4
:101DB0007367CE0189960E948946CE0101960E94E2
:101DC0008946CE0145960E948946CE0183960E949F
:101DD00089464091BC045091BD046091BE0470914D
:101DE000BF0423E0CE0183960E94BD462091B40437
:101DF0003091B5044091B6045091B70460E070E0B2
:101E000080E291E40E94B288AB01BC0121E0CE01E6
:101E100045960E948E466EE176E0CE0101960E94C4
:101E20003A4ABE016B5E7F4FCE0101960E94BC45CF
:101E300065E176E00E94A545BE016D5D7F4F0E9481
:101E4000BC456BE176E00E94A545BC01CE018996B8
:101E50000E944B47CE0189960E947367CE018996F6
:101E60000E948946CE0101960E948946CE01459680
:101E70000E948946CE0183960E948946409127029E
:101E8000509128026091290270912A0222E0CE012D
:101E900045960E94BD4661E376E0CE0101960E9420
:101EA0003A4ABE016B5E7F4FCE0101960E94BC454F
:101EB00067E476E00E94A545BC01CE0183960E94AE
:101EC0004B47CE0183960E947367CE0183960E9492
:101ED0008946CE0101960E948946CE0145960E9410
:101EE000894640912302509124026091250270910D
:101EF000260222E0CE0145960E94BD466EE476E0C1
:101F0000CE0101960E943A4ABE016B5E7F4FCE0120
:101F100001960E94BC456BE176E00E94A545BC019C
:101F2000CE0183960E944B47CE0183960E94736731
:101F3000CE0183960E948946CE0101960E94894671
:101F4000CE0145960E94894603E1C02E02E0D02EC4
:101F5000EE24E394F12C07E180911102909112029A
:101F60008E159F050CF474CAF601A190B1906F0113
:101F70004AE0B501CE0183960E9418474AE0B701B6
:101F8000CE0145960E94184761E676E0CE010196A3
:101F90000E943A4ABE016B5E7F4FCE0101960E94BD
:101FA000BC4568E87AE00E94A545BE016D5D7F4FA3
:101FB0000E94BC4569E676E00E94A5450A9DB001F5
:101FC0000B9D700D1124675A7D4F0E94A545BC01E1
:101FD000CE0189960E944B47CE0189960E94736775
:101FE000CE0189960E948946CE0101960E948946BB
:101FF000CE0145960E948946CE0183960E9489466D
:10200000FFEFEF1AFF0AA8CFBB24B39488CA029748
:1020100009F0B0CA62E975E0CE0101960E943A4A21
:10202000CE0101960E943B52082FCE0101960E94DC
:102030008946002309F49ECA8091EF0E9091F00E1C
:10204000029740F0E091EB0EF091EC0E309711F01A
:10205000818101C080E01A8219821C821B821E824B
:102060001D828D8B1E8ABE016B5E7F4FCE01019655
:102070000E945F46BE016F5F7F4F85EE9EE00E942B
:102080000746CE0101960E9489468091EF0E9091FD
:10209000F00E892B41F0E091EB0EF091EC0E3097B1
:1020A00011F0108101C010E06AE776E0CE010196E0
:1020B0000E943A4A6BEE7EE0CE0101960E94BC453A
:1020C0006BE679E00E94A545BC0182E59DE00E9497
:1020D000554ACE0101960E94894665EE7EE082E572
:1020E0009DE00E94344B46CA41E050E060E070E061
:1020F000CE0101960E94455FBE016F5F7F4F83ED69
:102100009EE00E940746CE0101960E9489466CEB34
:1021100076E0CE0145960E943A4ACE0145960E944D
:102120003B52811113C065E579E0CE0101960E9412
:102130003A4ACE0101960E943B5211E0811101C042
:1021400010E0CE0101960E94894601C011E0CE0147
:1021500045960E948946112309F49DC062E070E013
:10216000CE0101960E94875FBE016F5F7F4F83EDB6
:102170009EE00E940746CE0101960E94894663EDCB
:102180007EE082E59DE00E94344B0E94B04420E056
:1021900030E048EC52E40E9413850E949D876093D2
:1021A00043027093440280934502909346020E943A
:1021B0000E5C6091430270914402809145029091BF
:1021C00046028B019C0100591F4521403109013411
:1021D0001C492105310588F06FE876E0CE010196B3
:1021E0000E943A4A63ED7EE0CE0101960E94BC4512
:1021F00062EA76E00E94A5455AC119821A821B82C2
:102200001C821D821E821F8218860E94B48420E0D8
:1022100030E048EC52E40E9404878E010F5F1F4FAC
:1022200022E047E00E94E07FBC0189ED9EE00E9431
:102230005F4662EB76E0CE0145960E943A4A69ED30
:102240007EE0CE0145960E94BC456FEB76E00E9491
:10225000A545BC0189ED9EE00E947446CE014596DD
:102260000E9489461092690B1092680B809143027C
:1022700090914402A0914502B091460280930910CA
:1022800090930A10A0930B10B0930C1080E090E094
:102290000E94F95F15C164EC76E0CE0145960E947C
:1022A0003A4ACE0145960E943B52811113C06AEC16
:1022B00076E0CE0101960E943A4ACE0101960E9434
:1022C0003B5211E0811101C010E0CE0101960E9445
:1022D000894601C011E0CE0145960E94894611232E
:1022E00009F467C046E050E065E070E0CE01019679
:1022F0000E94455FBE016F5F7F4F83ED9EE00E94AD
:102300000746CE0101960E94894683ED9EE00E9419
:102310000E456B017C0165E476E0CE0101960E94DA
:102320003A4ACE0101960E94BC44BC016F5F7F4FC8
:10233000CE0145960E94875FBE016B5E7F4F83EDA5
:102340009EE00E940746CE0145960E948946CE0136
:1023500001960E94894683ED9EE00E940E45DB01B6
:10236000E1E1F2E041E050E02091110230911202EF
:10237000241735075CF0228133812A173B0711F4BB
:10238000138212824F5F5F4F3296EECF9601220F7B
:10239000331FF901EF5EFD4F7183608382E090E0AF
:1023A0000E94A2576BEE7EE082E59DE00E94344BD6
:1023B00043C060ED76E0CE0145960E943A4ACE01D8
:1023C00045960E943B52811113C066ED76E0CE0126
:1023D00001960E943A4ACE0101960E943B5211E0BA
:1023E000811101C010E0CE0101960E94894601C012
:1023F00011E0CE0145960E948946112331F1E1E1B9
:10240000F2E081E090E02091110230911202281751
:10241000390774F0863091051CF49383828305C0DC
:102420009C012E5F3F4F3383228301963296EBCF80
:1024300082E090E00E94A2571092690B1092680B04
:1024400080E090E00E94F95F9AC86CED76E0CE01E2
:1024500045960E943A4ACE0145960E943B52811110
:1024600013C064EE76E0CE0101960E943A4ACE0196
:1024700001960E943B5211E0811101C010E0CE0193
:1024800001960E94894601C011E0CE0145960E9446
:102490008946112381F16CEE76E0CE0101960E940F
:1024A0003A4A6FEB7FE0CE0101960E94BC45BC0129
:1024B00089ED9EE00E947446CE0101960E948946F5
:1024C0006BE879E0CE0101960E943A4A69ED7EE020
:1024D000CE0101960E94BC45BC01CE0145960E94EA
:1024E0004B47CE0145960E947367CE0145960E94E8
:1024F00089460C94B61C66EF76E0CE0145960E94A4
:102500003A4ACE0145960E943B52811113C06BEFAF
:1025100076E0CE0101960E943A4ACE0101960E94D1
:102520003B5211E0811101C010E0CE0101960E94E2
:10253000894601C011E0CE0145960E9489461123CB
:1025400009F43FC065E476E0CE0101960E943A4A64
:10255000CE0101960E94BC44BC016F5F7F4FCE014B
:1025600045960E94875FBE016B5E7F4F83ED9EE0C4
:102570000E940746CE0145960E948946CE010196EB
:102580000E94894683ED9EE00E940E45611571050B
:1025900021F481E080937F0410C06130710519F44B
:1025A00010927F040AC06230710511F00C94BF0ACA
:1025B00081E080937F0410927E040E9435560C9433
:1025C000BF0A60E077E0CE0145960E943A4ACE010C
:1025D00045960E943B52811113C064E077E0CE0122
:1025E00001960E943A4ACE0101960E943B5211E0A8
:1025F000811101C010E0CE0101960E94894601C000
:1026000011E0CE0145960E948946112309F46FC05E
:1026100063E070E0CE0101960E94875FBE016F5FAC
:102620007F4F83ED9EE00E940746CE0101960E94F7
:10263000894663ED7EE082E59DE00E94344B109276
:10264000690B1092680B63ED7EE085EC9FE00E94C1
:10265000744685E290E1892BE1F00091C90F109159
:10266000CA0F0115110519F41092251012C0073078
:10267000110510F007E010E06091C50F7091C60FD2
:10268000A80185E290E10E94048CF801EB5DFF4E09
:1026900010828091680B9091690B0E94F95F68E04D
:1026A00077E0CE0145960E943A4A65EC7FE0CE0184
:1026B00045960E94BC45BC01CE0101960E944B4745
:1026C000CE0145960E948946BE016F5F7F4F88E12B
:1026D0009CE00E94554A68EB7BE080E090E00E941D
:1026E000204D85E290E10E94FD5B0C94B61C60E1F8
:1026F00077E0CE0145960E943A4ACE0145960E9467
:102700003B52811113C065E177E0CE0101960E9432
:102710003A4ACE0101960E943B5211E0811101C05C
:1027200010E0CE0101960E94894601C011E0CE0161
:1027300045960E9489461123C1F164E070E0CE0104
:1027400001960E94875FBE016F5F7F4F83ED9EE021
:102750000E940746CE0101960E9489466AE177E011
:10276000CE0145960E943A4A63ED7EE0CE01459641
:102770000E94BC45BC01CE0101960E944B47CE0190
:1027800045960E948946BE016F5F7F4F88E19CE0BD
:102790000E94554A68EB7BE080E090E00E94204D6B
:1027A000BE016F5F7F4F0C94B21C61E277E0CE01F7
:1027B00083960E943A4ACE0183960E943B52811131
:1027C000A2C764E277E0CE0145960E943A4ACE0164
:1027D00045960E943B52811113C067E277E0CE011B
:1027E00001960E943A4ACE0101960E943B5211E0A6
:1027F000811101C010E0CE0101960E94894601C0FE
:1028000011E0CE0145960E948946CE0183960E9432
:10281000894611117CC76BE577E0CE0101960E94D5
:102820003A4ACE0101960E943B52182FCE010196E2
:102830000E948946112309F46CC08091EF0E90919B
:10284000F00E079710F40C94A11C66E070E0CE0126
:1028500001960E94875FBE016F5F7F4F83ED9EE010
:102860000E940746CE0101960E9489460E94B0440C
:10287000AB01BC014093000250930102609302023D
:102880007093030221E0CE0145960E94BD466FE69B
:1028900076E0CE0101960E943A4ABE016B5E7F4F00
:1028A000CE0101960E94BC4562E278E00E94A545F7
:1028B000BC0189ED9EE00E947446CE0101960E9403
:1028C0008946CE0145960E94894669ED7EE0CE019B
:1028D00001960E944B47CE0101960E947367CE017C
:1028E00001960E9489460E94584D28EE33E040E050
:1028F00050E00E940C86CA01B9010E94B284609324
:10290000B20A7093B30A8093B40A9093B50A0C94F8
:10291000A11C62E677E0CE0101960E943A4ACE0100
:1029200001960E943B52182FCE0101960E948946C3
:102930001123E1F18091EF0E9091F00E079710F4C2
:102940000C94A11C66E070E0CE0101960E94875FA6
:10295000BE016F5F7F4F83ED9EE00E940746CE0170
:1029600001960E9489460E94B044AB01BC0140938D
:102970000C0250930D0260930E0270930F0221E03F
:10298000CE0145960E94BD466FE776E0CE010196E6
:102990000E943A4ABE016B5E7F4FCE0101960E94B3
:1029A000BC4562E278E00E94A54583C069E677E015
:1029B000CE0145960E943A4ACE0145960E943B526E
:1029C000811113C06DE677E0CE0101960E943A4A6C
:1029D000CE0101960E943B5211E0811101C010E02E
:1029E000CE0101960E94894601C011E0CE014596B4
:1029F0000E948946112309F468C080917204909165
:102A000073040E94C76960932F0270933002809311
:102A100031029093320260931D1070931E108093C8
:102A20001F109093201080E090E0A0E8BFE3809317
:102A3000370290933802A0933902B0933A02809300
:102A4000151090931610A0931710B09318106AEEFB
:102A500073E082E59DE00E94634A60912F027091CD
:102A6000300280913102909132020E948264109271
:102A7000690B1092680B80E090E00E94F95F409132
:102A80002F0250913002609131027091320222E0A7
:102A9000CE0145960E94BD4661E777E0CE010196E2
:102AA0000E943A4ABE016B5E7F4FCE0101960E94A2
:102AB000BC45BC0189ED9EE00E947446CE010196A2
:102AC0000E948946CE01459611C66AE777E0CE019D
:102AD00045960E943A4ACE0145960E943B5281118A
:102AE00014C060E877E0CE0101960E943A4ACE0118
:102AF00001960E943B52FF24F394811101C0F12CF6
:102B0000CE0101960E94894602C0FF24F394CE01B3
:102B100045960E9489468E010B5E1F4FFF2009F4E7
:102B2000B2C08091EF0E9091F00E0797D8F066E05A
:102B300070E0CE0101960E94875FBE016F5F7F4FFC
:102B400083ED9EE00E940746CE0101960E948946D1
:102B50000E94B04460932702709328028093290258
:102B600090932A02809170049091710499270E9499
:102B7000DD58BC01990F880B990B0E94B4842DE09D
:102B800038E643E55BE30E9413856B017C012091ED
:102B90009C0430919D0440919E0450919F040E949A
:102BA000AE8418164CF06091840470918504809175
:102BB0008604909187041BC02091B0043091B10429
:102BC0004091B2045091B304C701B6010E94F3874B
:102BD00087FF05C0C701B6010E94AE5E08C06091C4
:102BE00098047091990480919A0490919B0420E03C
:102BF00030E048EC52E40E9413856B017C0120E038
:102C000030E0A9010E94AE84181634F0C12CD12CFA
:102C1000A8EAEA2EA1E4FA2EC0922702D092280256
:102C2000E0922902F0922A02C0923D10D0923E100A
:102C3000E0923F10F092401069ED73E082E59DE074
:102C40000E94634A609127027091280280912902B4
:102C500090912A020E9482641092690B1092680B74
:102C600080E090E00E94F95F409127025091280295
:102C70006091290270912A0222E0C8010E94BD469B
:102C800066E877E020C560E977E0CE0145960E94CE
:102C90003A4ACE0145960E943B52811114C065E923
:102CA00077E0CE0101960E943A4ACE0101960E9439
:102CB0003B52FF24F394811101C0F12CCE01019607
:102CC0000E94894602C0FF24F394CE0145960E94DB
:102CD0008946FF2009F48EC08091EF0E9091F00E8E
:102CE0000697E8F065E070E0CE0101960E94875FEC
:102CF000BE016F5F7F4F83ED9EE00E940746CE01CD
:102D000001960E9489460E94B0440E9434886093D4
:102D1000B8047093B9048093BA049093BB04809173
:102D2000C4049091C5040E944A7D20E030E048E050
:102D300051E40E9404876093C0047093C10480939F
:102D4000C2049093C30460932D1070932E1080934F
:102D50002F10909330108091B8049091B904A091F5
:102D6000BA04B091BB048093351090933610A093B1
:102D70003710B093381069EC73E082E59DE00E9453
:102D8000634A2091B8043091B9044091BA0450913B
:102D9000BB0460E070E080E291E40E94B28841E010
:102DA00050E00E94005D6AE977E082E59DE00E94C4
:102DB000444B6091C0047091C1048091C204909111
:102DC000C3040E9482641092690B1092680B80E029
:102DD00090E00E94F95F4091C0045091C10460915D
:102DE000C2047091C30423E0C8010E94BD4661EA99
:102DF00077E0B5C06CEA77E0CE0145960E943A4A8A
:102E0000CE0145960E943B52811114C061EB77E0E0
:102E1000CE0101960E943A4ACE0101960E943B5291
:102E2000FF24F394811101C0F12CCE0101960E9480
:102E3000894602C0FF24F394C8010E948946FF20FE
:102E400009F499C08091EF0E9091F00E0697E8F08A
:102E500065E070E0CE0101960E94875FBE016F5F62
:102E60007F4F83ED9EE00E940746CE0101960E94AF
:102E700089460E94B0440E9434886093B4047093E1
:102E8000B5048093B6049093B7048091C4049091E4
:102E9000C5040E944A7D20E030E048E051E40E94F1
:102EA00004876093BC047093BD048093BE04909328
:102EB000BF0460933110709332108093331090935D
:102EC00034108091B4049091B504A091B604B091EF
:102ED000B7048093391090933A10A0933B10B093AD
:102EE0003C106AEB73E082E59DE00E94634A20910A
:102EF000B4043091B5044091B6045091B70460E039
:102F000070E080E291E40E94B28841E050E00E94CB
:102F1000005D6AE977E082E59DE00E94444B6091A4
:102F2000BC047091BD048091BE049091BF040E94C6
:102F300082641092690B1092680B80E090E00E940E
:102F4000F95F4091BC045091BD046091BE04709142
:102F5000BF0423E0C8010E94BD4666EB77E0CE01C6
:102F600001960E943A4AB801CE0101960E94BC45E2
:102F70006AEA77E092C06FEB77E0C8010E943A4AB4
:102F8000C8010E943B52811114C063EC77E0CE016E
:102F900001960E943A4ACE0101960E943B52FF24BC
:102FA000F394811101C0F12CCE0101960E94894653
:102FB00002C0FF24F394C8010E948946FF2009F44F
:102FC0006FC060E080916C040E94974CF9E1AF2ED5
:102FD000B12CC12CD12C760180916C040E94D64C6E
:102FE000BC01990F880B990B0E94B4849B01AC0122
:102FF000C701B6010E943E866B017C016AE070E069
:1030000080E090E00E94204D61E0A61AB10821F70F
:1030100020E030E040EA50E4C701B6010E94138589
:1030200020E030E040E85AE30E94138520E030E0E1
:1030300048EC51E40E9404876093230270932402B9
:10304000809325029093260260935310709354103E
:1030500080935510909356101092690B1092680B44
:1030600080E090E00E94F95F409123025091240299
:10307000609125027091260222E0C8010E94BD469F
:103080006EE476E0CE0101960E943A4AB801CE0184
:1030900001960E94BC456BE176E00E94A5451CC3E9
:1030A00067EC77E0C8010E943A4AC8010E943B528F
:1030B000811114C06BEC77E0CE0101960E943A4A70
:1030C000CE0101960E943B52FF24F394811101C06E
:1030D000F12CCE0101960E94894602C0FF24F39490
:1030E000C8010E948946FF2009F431C146E050E042
:1030F00064E070E0CE0101960E94455FBE016F5F03
:103100007F4F83ED9EE00E940746CE0101960E940C
:10311000894683ED9EE00E940E454B015C011B0138
:1031200065E476E0CE0101960E943A4ACE0101960E
:103130000E94BC44BC016F5F7F4FC8010E94875F43
:10314000B80183ED9EE00E940746C8010E948946AF
:10315000CE0101960E948946F0906A040E94B04414
:103160002B013C01640171E0C71AD10865E473E0EA
:1031700082E59DE00E94634A4AE050E0B40182E5A6
:103180009DE00E942B4B6BE679E082E59DE00E947A
:10319000444BC301B2010E9482646F2DC8010E949A
:1031A000224118870F831D821E82198289E08A833B
:1031B00081E08B838C831C8A1B8ACE0101960E943E
:1031C0007C40CE0101960E94AE4DCE0101960E9438
:1031D0004251EE80F12C8BE0E816F1041CF0EAE09D
:1031E000EE2EF12CEBE58E16910408F44CC070E441
:1031F000A72E7BE0B72E3501212C312C2101C12CCB
:10320000D12CCE14DF04B9F06C2DCE0101960E94B2
:10321000F44E9B01AC01F3016193719381939193FF
:103220003F01C201B1010E943E861B012C01FFEF4C
:10323000CF1ADF0AE6CFB7010F2C000C880B990BD1
:103240000E94B4849B01AC01C201B1010E940487B9
:103250002B013C01C12CD12CCE14DF0409F457C042
:10326000F5012081318142815381C301B2010E9465
:103270003D86F50161937193819391935F01FFEF17
:10328000CF1ADF0AE9CF121413040CF5E214F30489
:1032900024F4670121E0C21AD1086C2DCE010196F9
:1032A0000E94F44E9B01AC01C601880F991F880F44
:1032B000991FBC01605C744F6B01C301B2010E9495
:1032C0003D86F601608371838283938320C0232827
:1032D000F1F430E4A32E3BE0B32EC12CD12CCE145C
:1032E000DF04A9F06C2DCE0101960E94F44E9B01E3
:1032F000AC01C301B2010E943D86F5016193719357
:10330000819391935F01FFEFCF1ADF0AE8CFE0E4EA
:10331000FBE0A7E5B0E141915191619171914D932D
:103320005D936D937D932BE0E836F207A1F7109241
:10333000690B1092680B80E090E00E94F95F64E0F6
:1033400070E0C8010E94875F6FEC77E0BCC160EF5E
:1033500077E0C8010E943A4AC8010E943B5281119D
:1033600014C064EF77E0CE0101960E943A4ACE0184
:1033700001960E943B52FF24F394811101C0F12C6D
:10338000CE0101960E94894602C0FF24F394C80131
:103390000E948946FF2009F451C0809172049091E7
:1033A00073040E94C76960932B0270932C02809370
:1033B0002D0290932E02609321107093221080931F
:1033C00023109093241080E090E5A3ECB7E4809361
:1033D000330290933402A0933502B0933602809367
:1033E000191090931A10A0931B10B0931C106DE944
:1033F00073E082E59DE00E94634A60912B02709128
:103400002C0280912D0290912E020E9482641092D3
:10341000690B1092680B80E090E00E94F95F409188
:103420002B0250912C0260912D0270912E0222E00D
:10343000C8010E94BD4668EF77E045C163E078E0CF
:10344000C8010E943A4AC8010E943B52811114C02F
:1034500067E078E0CE0101960E943A4ACE010196DB
:103460000E943B52FF24F394811101C0F12CCE0144
:1034700001960E94894602C0FF24F394C8010E946D
:103480008946FF2009F47AC08091EF0E9091F00EEA
:103490000497D8F064E070E0CE0101960E94875F47
:1034A000BE016F5F7F4F83ED9EE00E940746CE0115
:1034B00001960E9489460E94B0446093370270933F
:1034C00038028093390290933A02809137029091AA
:1034D0003802A0913902B0913A028093151090936E
:1034E0001610A0931710B093181065E873E082E5EA
:1034F0009DE00E94634A609137027091380280918A
:10350000390290913A0242E050E00E94005D8091C1
:103510007204909173040E94C76960932F027093A4
:103520003002809331029093320260931D107093A9
:103530001E1080931F10909320106BE773E082E5BC
:103540009DE00E94634A60912F0270913002809149
:103550003102909132020E9482641092690B1092A3
:10356000680B80E090E00E94F95F40912F0250913B
:10357000300260913102709132029FC063E178E0C5
:10358000C8010E943A4AC8010E943B52811114C0EE
:1035900067E178E0CE0101960E943A4ACE01019699
:1035A0000E943B52FF24F394811101C0F12CCE0103
:1035B00001960E94894602C0FF24F394C8010E942C
:1035C0008946FF2009F4BDC18091EF0E9091F00E65
:1035D0000497D8F064E070E0CE0101960E94875F06
:1035E000BE016F5F7F4F83ED9EE00E940746CE01D4
:1035F00001960E9489460E94B04460933302709302
:103600003402809335029093360280913302909178
:103610003402A0913502B091360280931910909334
:103620001A10A0931B10B0931C1063E673E082E5A0
:103630009DE00E94634A6091330270913402809150
:1036400035029091360242E050E00E94005D809188
:103650007204909173040E94C76960932B02709367
:103660002C0280932D0290932E0260932110709370
:103670002210809323109093241069E573E082E573
:103680009DE00E94634A60912B0270912C02809110
:103690002D0290912E020E9482641092690B10926A
:1036A000680B80E090E00E94F95F40912B025091FE
:1036B0002C0260912D0270912E0222E0C8010E941E
:1036C000BD466BE078E0CE0101960E943A4AB8010F
:1036D000CE0101960E94BC45BC0189ED9EE00E948E
:1036E0007446CE0101960E948946C8010E9489460F
:1036F00069ED7EE0CE0101960E944B47CE01019616
:103700000E94736733C1CE0183960E9489460AE006
:1037100010E0C12CD12C760166246A9483E0782EC7
:103720006EE170E080E090E00E94204D8091740492
:103730000E94D64CB3010E947F89072E000C880B93
:10374000990B0E94B48420E030E040EA50E40E94EB
:1037500013859B01AC01C701B6010E943E866B0137
:103760007C0101501109E1F620E030E040E251E433
:103770000E9404876B017C016AE277E0CE014596E6
:103780000E943A4ACE0145960E943B5281116EC179
:103790006EE277E0CE0101960E943A4ACE01019690
:1037A0000E943B5211E0811101C010E0CE01019650
:1037B0000E948946CE0145960E948946112309F44C
:1037C0003FC020E030E040E650E4C701B6010E946F
:1037D00013859B01AC0160E070E080E890E40E94FA
:1037E0003D86AB01BC0140930402509305026093F7
:1037F00006027093070222E0CE0101960E94BD46A8
:10380000BE016F5F7F4F89ED9EE00E940746CE01AB
:1038100001960E94894662E377E0CE0101960E94FC
:103820003A4A69ED7EE0CE0101960E94BC45BC019A
:1038300089ED9EE00E947446CE0101960E94894661
:1038400061E477E0CE0145960E943A4ACE01459662
:103850000E943B5281110CC166E477E0CE010196D3
:103860000E943A4ACE0101960E943B5211E081111A
:1038700001C010E0CE0101960E948946CE01459616
:103880000E948946112309F43FC020E030E040E661
:1038900050E4C701B6010E9413859B01AC0160E0B2
:1038A00070E080E291E40E943D86AB01BC01409350
:1038B00008025093090260930A0270930B0222E0FF
:1038C000CE0101960E94BD46BE016F5F7F4F89ED1C
:1038D0009EE00E940746CE0101960E9489466BE455
:1038E00077E0CE0101960E943A4A69ED7EE0CE0172
:1038F00001960E94BC45BC0189ED9EE00E94744681
:10390000CE0101960E9489466BE879E0CE010196CE
:103910000E943A4A69ED7EE0CE0101960E94BC45C4
:10392000BC01CE0145960E944B47CE0145960E94B0
:103930007367CE0145960E948946CE0101960E948A
:103940008946BB2011F40C94BF0A6BE879E0CE01E4
:1039500001960E943A4A6BEE7EE0CE0101960E94EB
:10396000BC45BC0182E59DE00E94344BCE0101962E
:103970000E9489460C94BF0A0E941053182F882376
:1039800011F40C94CA0A69EC79E085EE9EE00E947D
:103990005F466BE178E082E59DE00E94444B612F39
:1039A00082E59DE00E944E4A82E59DE00E94314BF7
:1039B000812F0E947F680C94BF0A0E94584D28EE08
:1039C000C22E23E0D22EE12CF12CA70196010E94F9
:1039D0000C86CA01B9010E94B2842091B20A3091CA
:1039E000B30A4091B40A5091B50A0E943D862091D5
:1039F00000023091010240910202509103020E94A4
:103A0000F387181614F00C94CF0A0E94584DA701A2
:103A100096010E940C86CA01B9010E94B28460938B
:103A2000B20A7093B30A8093B40A9093B50A809156
:103A30003C0B90913D0B3DD064E170E080E090E064
:103A40000E94204D0C94E60A85EE9EE00E940E45F1
:103A5000613071058105910511F00C94C60C0E942E
:103A600008650C94C60C10E00C94BA0A11E0A2CEC2
:103A700011E004CFCE0183960E9489460C94120D6A
:103A8000EA960FB6F894DEBF0FBECDBFDF91CF919F
:103A90001F910F91FF90EF90DF90CF90BF90AF906C
:103AA0009F908F907F906F905F904F903F902F905E
:103AB00008952F923F924F925F926F927F928F92D2
:103AC0009F92AF92BF92CF92DF92EF92FF920F93AD
:103AD0001F93CF93DF93CDB7DEB7C955D1090FB68A
:103AE000F894DEBF0FBECDBF1C0100913C0B1091BE
:103AF0003D0B68EA76E082E59DE00E94634AC101E1
:103B00000E940F64C1010596059708F180913C0B56
:103B100090913D0B8215930519F10E9455743092D6
:103B20003D0B20923C0B0E9428564AE0B101CE0189
:103B300001960E941847BE016F5F7F4F85EE9EE0A1
:103B40000E940746CE0101960E94894609C02EEFC9
:103B500022162FEF3206B1F40E9435560C94B9327A
:103B60006BE679E0CE0101960E943A4A4AE050E0C5
:103B70006FEF7FEFCE0101960E943A75CE0101965C
:103B80000E948946F1017996E332F10510F00C9418
:103B9000E8308827EE58FF4F8F4F0C949289809120
:103BA000770B882309F458C161E0809182040E9458
:103BB000974C60E0809180040E94974C0E94AE6216
:103BC0006093CE0A7093CF0A8093D00A9093D10A63
:103BD00023E333E948E853E40E94048720E030E01F
:103BE00040E85FE30E943E860E94028926E636EAAC
:103BF00045EA53E40E9413856093780B7093790B28
:103C000080937A0B90937B0B0E94DA55AB01BC0139
:103C100023E0CE0180960E94BD46BE01605E7F4FCC
:103C2000CE0101960E944B476AED79E0CE010196E4
:103C30000E94A545BC0183ED9EE00E947446CE0122
:103C400001960E948946CE0180960E94894666E4CC
:103C500078E0CE0101960E943A4A63ED7EE0CE0103
:103C600001960E94BC45BC0189ED9EE00E9474460D
:103C7000CE0101960E9489460E94DA559B01AC0153
:103C800067966FAF679768963FAF689769964FAF33
:103C900069976A965FAF6A970E94FB4C2B013C01C3
:103CA0006EE170E080E090E00E94204D0E94DA55C5
:103CB0006B017C010E94FB4C4B015C018418950850
:103CC000A608B70867962FAD679768963FAD6897C7
:103CD00069964FAD69976A965FAD6A9781ED8816D0
:103CE00087E09806A104B1040CF43FC0C701B601F7
:103CF0000E943D866B017C0120E030E0A9010E941A
:103D0000F38718165CF426EA3BE944EC5BE3C70151
:103D1000B6010E94AE8487FF0BC027C026EA3BE9AC
:103D200044EC5BEBC701B6010E94F3871816ECF078
:103D3000C501B40128EE33E040E050E00E94E08588
:103D4000CA01B9010E94B4844B015C0120E030E05B
:103D50004AE754E4C701B6010E941385A501940106
:103D60000E940487AB01BC0103C040E050E0BA01EF
:103D700022E0CE0180960E94BD46BE01605E7F4F6C
:103D8000CE0101960E944B4760E278E0CE01019699
:103D90000E94A545BC018DEC9EE00E947446CE01B8
:103DA00001960E948946CE0180960E94894664E26F
:103DB00078E0CE0101960E943A4A6DEC7EE0CE0199
:103DC00001960E94BC45BC0189ED9EE00E94DB4546
:103DD000CE0101960E9489466BE679E0CE010196FC
:103DE0000E943A4A6DEC7EE0CE0101960E94BC45ED
:103DF000BC0183ED9EE00E94DB45CE0101960E944E
:103E0000894668E278E0CE0101960E943A4A4AE08B
:103E100050E060E070E0CE0101960E94EC75CE01AA
:103E200001960E94894663ED7EE0CE0101960E94D4
:103E30004B4745E050E06FEF7FEFCE0101960E94C7
:103E4000BB74CE0101960E9489466FE278E089ED4D
:103E50009EE00E94CD45EDC1C0900C02D0900D02B5
:103E6000E0900E02F0900F020E94584D2E966CAF1B
:103E70007DAF8EAF9FAF2E9761E0809182040E944C
:103E8000974C60E0809180040E94974C0E94AE6243
:103E90006093CE0A7093CF0A8093D00A9093D10A90
:103EA0000E94BD550E94DA5562966CAF7DAF8EAF11
:103EB0009FAF62970E94FB4C4B015C016AE070E08F
:103EC00080E090E00E94204D61E174E089ED9EE089
:103ED0000E94E14520E030E04AE754E4C701B60122
:103EE0000E94138566966CAF7DAF8EAF9FAF6697CD
:103EF000412C512C3201C12CD12C7601C701B601C5
:103F00000E94B48466962CAD3DAD4EAD5FAD669714
:103F10000E94AE8487FF8DC10E94584D2E962CAD15
:103F20003DAD4EAD5FAD2E97621B730B840B950BB1
:103F30000E94B28420E030E04AE754E40E94048703
:103F4000AB01BC0123E0CE0101960E94BD46BE013B
:103F50006F5F7F4F83ED9EE00E940746CE01019682
:103F60000E9489460E94DA556B017C010E94FB4C3D
:103F70009B01AC01281939094A095B0949015A0119
:103F800031ED831637E09306A104B1040CF443C06D
:103F900020E030E0A901C701B6010E94F38718169E
:103FA0005CF426EA3BE944EC5BE3C701B6010E94FE
:103FB000AE8487FF0BC02FC026EA3BE944EC5BEBE5
:103FC000C701B6010E94F38718162CF1C501B40190
:103FD00028EE33E040E050E00E94E085CA01B901DC
:103FE0000E94B4844B015C0162962CAD3DAD4EAD98
:103FF0005FAD6297C701B6010E943D8620E030E0C8
:104000004AE754E40E941385A50194010E940487A5
:104010004B015C0103C0812C912C540163ED7EE0C7
:10402000CE0101960E944B4762E278E0CE010196F4
:104030000E94A545BC0183ED9EE00E947446CE011E
:1040400001960E94894623E0B701A601CE01809621
:104050000E94BD46BE01605E7F4FCE0101960E9468
:104060004B4762E478E0CE0101960E94A545BC0171
:104070008DEC9EE00E947446CE0101960E94894616
:10408000CE0180960E94894622E0B501A401CE01AE
:1040900001960E94BD4660E37AE0CE0180960E94C0
:1040A0003A4A63ED7EE0CE0180960E94BC4565E40D
:1040B00078E00E94A5456DEC7EE00E94BC4565E27B
:1040C00078E00E94A545BE016F5F7F4F0E94BC450E
:1040D00060E278E00E94A545BC0189ED9EE00E9467
:1040E000DB45CE0180960E948946CE0101960E9452
:1040F000894620E030E0A901C501B4010E94F387A0
:1041000087FD06C06BE679E08DEC9EE00E94CD4510
:1041100022E0B501A401CE0180960E94BD46BE01F9
:10412000605E7F4FCE0101960E944B4760E278E0CF
:10413000CE0101960E94A545BC018DEC9EE00E9437
:10414000DB45CE0101960E948946CE0180960E94F1
:10415000894669ED7EE0CE0101960E944B47CE0173
:1041600001960E947367CE0101960E948946C301A1
:10417000B20125E030E040E050E00E94E085672B8E
:10418000682B692B21F568E278E0CE0101960E9448
:104190003A4A45E050E060E070E0CE0101960E94AE
:1041A000EC75CE0101960E9489466DEC7EE0CE0151
:1041B00001960E944B4745E050E06FEF7FEFCE0144
:1041C00001960E94BB74CE0101960E94894669EC5B
:1041D00079E089ED9EE00E945F4665E070E080E056
:1041E00090E00E94204D0E94584D6B017C012E965C
:1041F0002CAD3DAD4EAD5FAD2E97C21AD30AE40A89
:10420000F50A0E94DA5562966CAF7DAF8EAF9FAF14
:1042100062970E94FB4C4B015C016AE070E080E019
:1042200090E00E94204D3FEF431A530A630A730A3D
:1042300065CE60E0809182040E94974C0C94163108
:10424000F0906A0469EC79E0CE01805C9F4F0E9497
:104250003A4A8E01005E1F4F6F2DC8010E94224115
:1042600018870F831D821E82198289E08A8381E06C
:104270008B838C831C8A1B8ACE0101960E947C4012
:10428000CE0101960E94AE4DCE0101960E94425190
:104290000E8110E00330110509F46FC169E478E084
:1042A000CE01805C9F4F0E945F4669EC79E089ED0A
:1042B0009EE00E945F46BE01605C7F4FCE018E96FD
:1042C0000E944B474AE050E060E070E0CE018E96DD
:1042D0000E94EC75CE018E960E94894661E080E0D6
:1042E0000E94B25B6DE678E0CE01805C9F4F0E9439
:1042F0005F4660E4A62E6BE0B62ECC24C394D12C8E
:10430000E12CF12CE016F1060CF0EEC06E2DCE0182
:1043100001960E94F44ED5012D913D914D915D91F4
:104320005D010E943E862B013C0120E030E04CEF15
:1043300052EC0E94AE8487FF21C04AE0B601CE0154
:104340008E960E9418476AE975E0CE01C4960E94D5
:104350003A4ABE01625D7F4FCE01C4960E94BC45C1
:1043600063E578E00E94A545BC0189ED9EE00E94CE
:10437000DB45CE01C4960E94894645C022E0B301C8
:10438000A201CE018E960E94BD464AE0B601CE0142
:10439000C4960E9418476AE975E0CE01CA960E9449
:1043A0003A4ABE016C5C7F4FCE01CA960E94BC4562
:1043B00065E476E00E94A545BE01625D7F4F0E94E4
:1043C000BC45BC018DEC9EE00E947446CE01CA96AD
:1043D0000E948946CE01C4960E948946CE018E96DF
:1043E0000E9489466DEC7EE0CE018E960E944B477E
:1043F0006BE679E0CE018E960E94A545BC0189ED61
:104400009EE00E94DB45CE018E960E9489460130D7
:10441000110561F4E114F10409F05FC069ED7EE07B
:10442000CE01805C9F4F0E94744657C00230110538
:1044300019F522E0B301A201CE01C4960E94BD4647
:10444000BE016C5C7F4FCE018E960E944B476BE69F
:1044500079E0CE018E960E94A545BC01CE01805C1C
:104460009F4F0E94DB45CE018E960E948946CE0169
:10447000C4960E94894631C00330110571F16DEC7C
:104480007EE0CE018E960E944B4744E150E06FEFF4
:104490007FEFCE018E960E94BB74CE018E960E9455
:1044A000894669E579E0CE018E960E943A4ACE01AE
:1044B0008E960E947B74CE018E960E9489468091D2
:1044C0007F04882351F080917E04882331F060EDD1
:1044D00077E080E090E00E94204DBFEFEB1AFB0AEE
:1044E000EFEFCE1ADE0A0ECFCE01805C9F4F0E9406
:1044F000194589ED9EE00E94194501151105A9F4A1
:104500006FE274E089ED9EE00E94E1456FE578E09E
:10451000CE018E960E943A4A4AE050E06FEF7FEF5C
:10452000CE018E960E94BB74E4C00430110514F0D5
:104530000C943831BE01605C7F4FCE018E960E9494
:104540004B474AE050E06FEF7FEFCE018E960E941E
:10455000BB74CE018E960E94894669E579E0CE0152
:104560008E960E943A4ACE018E960E947B74CE01AE
:104570008E960E9489460C9438316AE678E0CE0126
:10458000805C9F4F0E945F46BE01605C7F4FCE0102
:104590008E960E944B474AE050E060E070E0CE010A
:1045A0008E960E94EC75CE018E960E94894669EC2B
:1045B00079E089ED9EE00E945F4669ED7EE0CE01E4
:1045C000805C9F4F0E94744600E010E0602FCE0197
:1045D00001960E94F44E6B017C0122E0AB01BC010C
:1045E000CE010115110569F48E960E94BD46BE01EB
:1045F000625D7F4F8BEC9FE00E94554ACE018E9604
:104600001CC0C4960E94BD46BE016C5C7F4FCE01AB
:104610008E960E944B476BE679E0CE018E960E9403
:10462000A545BC01CE01805C9F4F0E94DB45CE01B9
:104630008E960E948946CE01C4960E94894622E049
:10464000B701A601CE01C4960E94BD46BE016C5CB6
:104650007F4FCE018E960E944B476BE679E0CE01EC
:104660008E960E94A545BC0189ED9EE00E94DB4527
:10467000CE018E960E948946CE01C4960E9489463C
:104680000F5F1F4F0330110509F0A0CFCE01805CF2
:104690009F4F0E941945BE01605C7F4FCE018E96F0
:1046A0000E944B474AE050E06FEF7FEFCE018E96BD
:1046B0000E94BB74CE018E960E9489460E94997416
:1046C00089ED9EE00E94194560E778E0CE018E9664
:1046D0000E943A4A69ED7EE0CE018E960E94BC456A
:1046E0006AE778E00E94A545BC0189ED9EE00E9442
:1046F0007446CE018E960E948946CE01805C9F4F03
:104700000C94143180916C0490916D040E940159B5
:104710000C941631809170049091710499270E9435
:10472000DD58BC01990F880B990B0E94B4842DE0D1
:1047300038E643E55BE30E9413856B017C01209121
:104740009C0430919D0440919E0450919F040E94CE
:10475000AE8418164CF060918404709185048091A9
:104760008604909187041BC02091B0043091B1045D
:104770004091B2045091B304C701B6010E94F3877F
:1047800087FF05C0C701B6010E94AE5E08C06091F8
:1047900098047091990480919A0490919B0420E070
:1047A00030E048EC52E40E94138520E030E048EA13
:1047B00051E40E94138520912702309128024091F4
:1047C000290250912A020E9404876B017C0162E455
:1047D00074E083ED9EE00E94E14563ED7EE0CE0152
:1047E00001960E944B4742E350E060E070E0CE014A
:1047F00001960E94EC75CE0101960E94894622E046
:10480000B701A601CE0101960E94BD4663E978E09A
:10481000CE0180960E943A4ABE016F5F7F4FCE0163
:1048200080960E94BC456DE878E00E94A545BC01D9
:1048300089ED9EE00E947446CE0180960E948946D2
:10484000CE0101960E94894669ED7EE0CE01019677
:104850000E944B4742E350E06FEF7FEFCE0101969D
:104860000E94BB74CE0101960E9489468091770B0D
:10487000882311F40C94163160E273E080E090E03C
:10488000CAC20E94557466E774E089ED9EE00E94FA
:10489000E14569ED7EE0CE0101960E944B474AE07A
:1048A00050E060E070E0CE0101960E94EC75CE0110
:1048B00001960E9489466DE674E083ED9EE00E94B9
:1048C000E14563ED7EE0CE0101960E944B4744E155
:1048D00050E06FEF7FEFCE0101960E94BB74CE01D6
:1048E00001960E94894680913E0B90913F0B843047
:1048F000910549F40E94585281111AC010923F0B41
:1049000010923E0B15C0892B99F40E9458528823AF
:1049100039F084E090E090933F0B80933E0B08C009
:104920000E9458528111F5CF0E9458528111F1CF47
:1049300080913E0B90913F0B049741F161E674E04A
:1049400089ED9EE00E94E14569ED7EE0CE01019691
:104950000E944B474AE050E060E070E0CE010196D3
:104960000E94EC75CE0101960E94894669ED7EE0B9
:10497000CE0101960E944B476BE679E0CE0101968D
:104980000E94A54563ED7EE00C94932E8AE090E0B2
:104990000E948B566B017C0120E030E0A9010E944F
:1049A000AE84181634F08AE090E00E948B566B01BA
:1049B0007C0120E030E041EE53E4C701B6010E94E3
:1049C000AE8418164CF068EC70E080E090E00E9435
:1049D000204D83E090E0E9CF20E030E0A901C7015D
:1049E000B6010E94AE8418163CF063E574E089EDD0
:1049F0009EE00E94E14531C020E030E048EC52E406
:104A0000C701B6010E94AE8487FF02C021E001C049
:104A100020E0B701A601CE0101960E94BD4662E9E1
:104A200078E0CE0180960E943A4ABE016F5F7F4FC8
:104A3000CE0180960E94BC4567E978E00E94A545BA
:104A4000BC0189ED9EE00E947446CE0180960E94D2
:104A50008946CE0101960E94894669ED7EE0CE012D
:104A600001960E944B4742E350E06FEF7FEFCE018B
:104A700001960E94BB74CE0101960E9489466AE4A9
:104A800074E083ED9EE00E94E14563ED7EE0CE019F
:104A900001960E944B4742E350E060E070E0CE0197
:104AA00001960E94EC75DECE0E94584D2B013C0110
:104AB0000E94955064E670E080E090E00E94204DF6
:104AC00040E855E260E070E085EB9CE00E948B7668
:104AD00064E670E080E090E00E94204D69EA74E0B6
:104AE00083ED9EE00E94E14563ED7EE0CE010196FC
:104AF0000E944B4742E350E06FEF7FEFCE010196FB
:104B00000E94EC75CE0101960E9489466EE974E020
:104B100083ED9EE00E94E14563ED7EE0CE010196CB
:104B20000E944B4742E350E06FEF7FEFCE010196CA
:104B30000E94BB74CE0101960E94894680913E0B73
:104B400090913F0B8D7F2B961FAE2B97A12CB12CF4
:104B5000C12CD12CE12CF12C019709F477C09E01D6
:104B6000205E3F4F28963FAF2EAF2897AE01425EA2
:104B70005F4F2A965FAF4EAF2A970E94584DDC01D7
:104B8000CB0184199509A609B709883B9B40A1056B
:104B9000B10508F05BC085EB9CE00E94C947892BFA
:104BA00009F44DC02CED35E040E050E02093B90C05
:104BB0003093BA0C4093BB0C5093BC0C0E94935F93
:104BC00097FD06C082349105C9F780E090E002C0ED
:104BD0008FEF9FEF892B99F58E010F5F1F4F4801D3
:104BE0000E94935F97FF06C089818D3441F520E0D4
:104BF00030E00BC0D4018D934D0128962EAD3FAD12
:104C00002897A217B30761F7EFCFD8018D918D01D7
:104C1000280F311D2A964EAD5FAD2A97A417B50710
:104C2000A1F72E5B3F4F8E8D90E0982F88274F8DF8
:104C3000840F911D2817390711F40C94403162E359
:104C400070E080E090E00E94204D97CF0E94584D88
:104C5000DC01CB0184199509A609B709883B9B4063
:104C6000A105B10528F42B962FAD2B972111C7C0B4
:104C70000E94557463ED7EE0CE0180960E944B4702
:104C800042E350E066E070E0CE0180960E94EC7551
:104C9000CE0180960E9489462B963FAD2B973323F9
:104CA00011F40C945B3182E090E090933F0B809381
:104CB0003E0B4AE0B501CE0180960E9418474AE0BB
:104CC000B601CE018E960E9418474AE0B701CE0188
:104CD000CA960E941847BE01665C7F4FCE01C496FB
:104CE0000E944B4769E577E0CE01C4960E94A54536
:104CF000BE01625D7F4F0E94BC4569E577E00E947E
:104D0000A545BE01605E7F4F0E94BC45BC0189ED98
:104D10009EE00E947446CE01C4960E948946CE0150
:104D2000CA960E948946CE018E960E948946CE017F
:104D300080960E94894669ED7EE0CE0180960E94B1
:104D40004B474AE050E06FEF7FEFCE0180960E9424
:104D5000BB74CE0180960E9489466BE978E08BECAB
:104D60009FE00E94444B61EA78E089ED9EE00E945A
:104D70005F464AE0B501CE0180960E9418474AE09E
:104D8000B601CE018E960E9418474AE0B701CE01C7
:104D9000CA960E941847BE01665C7F4FCE01C4963A
:104DA0000E944B476BE679E0CE01C4960E94A54570
:104DB000BE01625D7F4F0E94BC456BE679E00E94B8
:104DC000A545BE01605E7F4F0E94BC456BE978E05F
:104DD0000E94A545BC0189ED9EE00E94DB45CE0105
:104DE000C4960E948946CE01CA960E948946CE0189
:104DF0008E960E948946CE0180960E94894662E383
:104E000070E080E090E00E94204D0E94955062E3A7
:104E100070E080E090E00E94204D0C9416310091EB
:104E200072041091730465EB74E083ED9EE00E94C0
:104E3000E1450E94557463ED7EE0CE0101960E942B
:104E40004B474AE050E06FEF7FEFCE0101960E94A2
:104E5000EC75CE0101960E948946C8010E94C7697F
:104E600062966CAF7DAF8EAF9FAF629780902F023E
:104E700090903002A0903102B0903202A5019401CE
:104E800060912B0270912C0280912D0290912E0244
:104E90000E943D862B013C0120E030E0A9010E94E8
:104EA000AE84882309F45BC0C0903702D0903802EA
:104EB000E0903902F0903A0220E030E0A901C70109
:104EC000B6010E94AE8418160CF049C080913302DE
:104ED00090913402A0913502B09136022E968CAF9B
:104EE0009DAFAEAFBFAF2E979C01AD01C701B6011C
:104EF0000E94AE84882399F1A70196012E966CAD8D
:104F00007DAD8EAD9FAD2E970E9404870E943F8895
:104F10002E966CAF7DAF8EAF9FAF2E97A5019401FB
:104F200062966CAD7DAD8EAD9FAD62970E943D8661
:104F3000A30192010E9404872E962CAD3DAD4EAD8B
:104F40005FAD2E970E9413850E9471879B01AC0173
:104F5000C701B6010E9413856B017C0103C0C12CFF
:104F6000D12C760163ED7EE0CE0101960E944B4785
:104F70004AE050E060E070E0CE0101960E94EC75DE
:104F8000CE0101960E94894620E030E64AEE56E4C2
:104F9000C701B6010E94F38718163CF461EB78E074
:104FA00089ED9EE00E945F4625C021E0B701A60181
:104FB000CE0180960E94BD4660EC78E0CE0101965D
:104FC0000E943A4ABE01605E7F4FCE0101960E9468
:104FD000BC4564EC78E00E94A545BC0189ED9EE0EB
:104FE0000E947446CE0101960E948946CE018096A9
:104FF0000E94894669ED7EE0CE0101960E944B47F2
:105000004AE050E06FEF7FEFCE0101960E94BB7443
:10501000CE0101960E94894664E670E080E090E04F
:105020000E94204D23CC00917C0410917D040E94AD
:105030005574C8010E94DD588C0162E370E080E085
:1050400090E00E94204DB801110F880B990B0E942F
:10505000B48420E030E040EA50E40E94138520E070
:1050600030EC4FE754E40E940487AB01BC0123E01D
:10507000CE0101960E94BD4665EE79E0CE01809694
:105080000E943A4ABE016F5F7F4FCE0180960E9418
:10509000BC456BE176E00E94A545BC0189ED9EE030
:1050A0000E947446CE0180960E948946CE010196E8
:1050B0000E94894668EC78E083ED9EE00E945F469E
:1050C00063ED7EE0CE0101960E944B474AE050E03E
:1050D00068E070E0CE0101960E94EC75CE01019669
:1050E0000E94894669ED7EE0CE0101960E944B4701
:1050F0004AE050E06FEF7FEFCE0101960E94BB7453
:10510000CE0101960E94894663ED7EE089ED9EE026
:105110000E94DB45ABCB9091F40A81E08927809314
:10512000F40A8091770B882331F069ED7EE088E105
:105130009CE00E94344B68EC70E080E090E06BCE25
:105140001092770B0C94163181E08093770B0C94BE
:10515000163160ED78E0CE0180960E943A4A65EC07
:105160007FE0CE0180960E94BC45BC01CE01019635
:105170000E944B4748EC50E06FEF7FEFCE01019665
:105180000E94EC75CE0101960E948946CE01809660
:105190000E94894664ED78E0CE0180960E943A4AEA
:1051A0006FEB7FE0CE0180960E94BC45BC01CE0132
:1051B00001960E944B4740ED57E06FEF7FEFCE0125
:1051C00001960E94BB74CE0101960E948946CE01D1
:1051D00080960E94894680913E0B90913F0B0197EB
:1051E00019F46BE176E002C06DE076E0CE01019645
:1051F0000E94434748EC50E06FEF7FEFCE010196ED
:105200000E943A75CE0101960E9489466DEF75E0C5
:10521000CE0101960E94434740ED57E06FEF7FEFCC
:10522000CE0101960E94BB74CE0101960E94894670
:105230006DEE75E0CE0101960E94434748EC50E0C8
:105240006FEF7FEFCE0101960E943A75CE01019675
:105250000E94894660EE75E0CE0101960E944347A8
:1052600040ED57E06FEF7FEFCE0101960E94BB74D7
:10527000CE0101960E94894663ED75E0CE0101964C
:105280000E94434748EC50E06FEF7FEFCE0101965C
:105290000E943A75CE0101960E94894668EC75E03D
:1052A000CE0101960E94434740ED57E06FEF7FEF3C
:1052B000CE0101960E94BB74CE0101960E948946E0
:1052C0006CEB75E0CE0101960E94434748EC50E03C
:1052D0006FEF7FEFCE0101960E943A75CE010196E5
:1052E0000E9489466BEA75E0CE0101960E94434711
:1052F00040ED57E06FEF7FEFCE0101960E94BB7447
:10530000CE0101960E94894680913E0B90913F0B01
:10531000039719F460EA75E002C066E975E0CE0112
:1053200001960E94434748EC50E06FEF7FEFCE01BB
:1053300001960E943A75CE0101960E9489466BE85B
:1053400075E0CE0101960E94434740ED57E06FEFB4
:105350007FEFCE0101960E94BB74CE0101960E94A0
:1053600089466EE775E0CE0101960E94434748ECFE
:1053700050E06FEF7FEFCE0101960E943A75CE01AB
:1053800001960E9489466FE675E0CE0101960E9463
:10539000434740ED57E06FEF7FEFCE0101960E944B
:1053A000BB74CE0101960E94894664E675E0CE0189
:1053B00001960E94434748EC50E06FEF7FEFCE012B
:1053C00001960E943A75CE0101960E94894667E5D2
:1053D00075E0CE0101960E94434740ED57E06FEF24
:1053E0007FEFCE0101960E94BB74CE0101960E9410
:1053F000894680913E0B90913F0B029719F466E429
:1054000075E002C066E375E0CE0101960E94434755
:1054100048EC50E06FEF7FEFCE0101960E943A75A5
:10542000CE0101960E94894669E275E0CE0101969F
:105430000E94434740ED57E06FEF7FEFCE010196AA
:105440000E94BB74CE0101960E9489466DE175E011
:10545000CE0101960E94434748EC50E06FEF7FEF8A
:10546000CE0101960E943A75CE0101960E948946AE
:105470006DE075E0CE0101960E94434740ED57E094
:105480006FEF7FEFCE0101960E94BB74CE010196B3
:105490000E94894662E075E0CE0101960E94434772
:1054A00048EC50E06FEF7FEFCE0101960E943A7515
:1054B000CE0101960E94894668EF74E0CE01019604
:1054C0000E94434740ED57E06FEF7FEFCE0101961A
:1054D0000E94BB74CE0101960E94894668EE74E07A
:1054E000CE0101960E94434748EC50E06FEF7FEFFA
:1054F000CE0101960E943A75CE0101960E9489461E
:105500006BED74E0CE0101960E94434740ED57E0F9
:105510006FEF7FEFCE0101960E94BB74CE01019622
:105520000E9489466FEC74E0CE0101960E944347C9
:1055300048EC50E06FEF7FEFCE0101960E943A7584
:10554000CE0101960E9489466FEB74E0CE01019670
:105550000E94434740ED57E05FC60E94955040E0EF
:1055600052EC61E070E085EB9CE00E948B768CED64
:1055700095E0A0E0B0E08093B90C9093BA0CA093B2
:10558000BB0CB093BC0C64E670E080E090E00E943D
:10559000204D69ED78E089ED9EE00E945F4669ED5F
:1055A0007EE082E59DE00E94344B62E370E080E0A3
:1055B00090E00E94204D69ED7EE0CE0101960E94B0
:1055C0004B4742E350E06FEF7FEFCE0101960E9420
:1055D000EC75CE0101960E94894665EE78E083ED78
:1055E0009EE00E945F4663ED7EE0CE0101960E9440
:1055F0004B4744E150E06FEF7FEFCE0101960E94F0
:10560000BB74CE0101960E94894680913E0B909119
:105610003F0B019739F484E090E00E94D85A6B0167
:105620007C0103C0C12CD12C760180913E0B90915E
:105630003F0B892B31F481E090E00E94D85A6B0136
:105640007C0120E030E040EA51E4C701B6010E944D
:10565000F387181664F521E0B701A601CE01019683
:105660000E94BD4661EF78E0CE0180960E943A4AE2
:10567000BE016F5F7F4FCE0180960E94BC4564EFF4
:1056800078E00E94A545BC0189ED9EE00E94744629
:10569000CE0180960E948946CE0101960E948946DD
:1056A00081E090E090933F0B80933E0B10C067EF3A
:1056B00078E089ED9EE00E945F4680913E0B9091DC
:1056C0003F0B019721F410923F0B10923E0B69EDB6
:1056D0007EE0CE0101960E944B474AE050E060E038
:1056E00070E0CE0101960E94EC75CE0101960E94F9
:1056F000894669ED7EE0CE0101960E944B476BE63C
:1057000079E0CE0101960E94A54563ED7EE00E94FE
:10571000BC45BC0189ED9EE00E947446CE01019615
:105720000E9489460E949550A1C865E576E0CE01A9
:1057300001960E9443474AE050E06FEF7FEFCE01B1
:1057400001960E94BB74CE0101960E948946809109
:105750007A0490917B040E940D6300E010E064E6FF
:1057600070E080E090E00E94204D80917A0490915A
:105770007B040E940D630F5F1F4F033011057CF304
:105780000A3011051CF4892B51F703C0892B09F04D
:10579000D0C06091E70F7091E80F072E000C880BC6
:1057A000990B0E94B4846B017C0160938510709307
:1057B000861080938710909388108091E50F9091C8
:1057C000E60FBC01990F880B990B0E94B48460937B
:1057D000811070938210809383109093841021E045
:1057E000B701A601CE0101960E94BD466DE678E0A4
:1057F000CE0180960E943A4ABE016F5F7F4FCE0174
:1058000080960E94BC45BC0189ED9EE00E947446D2
:10581000CE0180960E948946CE0101960E9489465B
:10582000409181105091821060918310709184108A
:1058300021E0CE0101960E94BD4663E079E0CE01F1
:1058400080960E943A4ABE016F5F7F4FCE018096DC
:105850000E94BC45BC0189ED9EE00E94DB45CE0163
:1058600080960E948946CE0101960E94894660E991
:1058700078E089ED9EE00E94CD4569EC79E0CE01AB
:1058800001960E943A4A44E150E060E070E0CE01A7
:1058900001960E94EC75CE0101960E9489466091A6
:1058A00085107091861080918710909188100E94C9
:1058B0009D874AE0CE0101960E941847BE016F5FA6
:1058C0007F4F83ED9EE00E940746CE0101960E9425
:1058D000894660E086E00E94B25B63ED7EE08BEC7F
:1058E0009FE00E94554A6FED8BEC9FE00E944E4A6C
:1058F00069E079E08BEC9FE00E94444B609181105D
:105900007091821080918310909184100E949D87E5
:105910004AE050E08BEC9FE00E942B4B60E978E07E
:105920008BEC9FE00E94444B64E670E080E090E0E6
:1059300072CA6AE476E0CE0101960E9443474AE0CB
:1059400050E060E070E0CE0101960E94EC75CE015F
:1059500001960E9489466AE276E089ED9EE00E9407
:10596000E14564C480911002882309F45FC469ECA6
:1059700079E0CE0101960E943A4A4AE050E061E0A7
:1059800070E0CE0101960E94EC75CE0101960E9456
:1059900089460E9455740E94D6602B013C010E94EA
:1059A000AE624B015C0160914302709144028091B0
:1059B0004502909146020E94B4849B01AC01679617
:1059C0006FAF679768963FAF689769964FAF6997D3
:1059D0006A965FAF6A970E94D6600E94B484679609
:1059E0002FAD679768963FAD689769964FAD6997F9
:1059F0006A965FAD6A970E94048721E03EED42E41B
:105A00005EE30E94B2889B01AC0160E070E080E838
:105A10009FE30E943D8620E03AE24DE257E40E9477
:105A200013856B017C01C301B2010E94B48420E0A4
:105A300030E048EC52E40E940487AB01BC0122E054
:105A4000CE0101960E94BD46BE016F5F7F4F8DEC77
:105A50009EE00E940746CE0101960E94894660ECB6
:105A600076E08DEC9EE00E94CD456DEC7EE083ED0E
:105A70009EE00E9474466CEB76E0CE0101960E9497
:105A80003A4A6DEC7EE0CE0101960E94BC45BC0115
:105A90008DEC9EE00E947446CE0101960E948946DC
:105AA0006DE678E089ED9EE00E945F4621E0B50159
:105AB000A401CE0101960E94BD46BE016F5F7F4FDB
:105AC00089ED9EE00E94DB45CE0101960E94894649
:105AD0006CE079E089ED9EE00E94CD4521E0B701C0
:105AE000A601CE0180960E94BD46BE01605E7F4F3A
:105AF000CE0101960E944B476AED79E0CE010196F6
:105B00000E94A545BC0189ED9EE00E94DB45CE01C7
:105B100001960E948946CE0180960E9489466DECCE
:105B20007EE0CE0101960E944B476BE679E0CE0104
:105B300001960E94A54569ED7EE00E94BC45BC012E
:105B400089ED9EE00E947446CE0101960E9489462E
:105B500063ED7EE0CE0101960E944B474AE050E0A3
:105B600060E070E0CE0101960E94EC75CE010196D6
:105B70000E94894621E0B501A401CE0101960E9450
:105B8000BD46BE016F5F7F4F8FED9EE00E940746CE
:105B9000CE0101960E9489466FED7EE0CE0101960E
:105BA0000E944B474AE050E06FEF7FEFCE01019635
:105BB0000E94BB74CE0101960E94894669E079E09B
:105BC000CE0101960E943A4ACE0101960E947B7452
:105BD000CE0101960E94894621E0B701A601CE01BF
:105BE00080960E94BD46BE01605E7F4FCE01019649
:105BF0000E944B476AED79E0CE0101960E94A545CF
:105C0000BC018FED9EE00E947446CE0101960E9479
:105C10008946CE0180960E9489466FED7EE0CE01D6
:105C200001960E944B474AE050E068EF7FEFCE01BB
:105C300001960E94BB74CE0101960E948946809114
:105C4000770B882309F4F2C268E572E080E090E007
:105C5000E2C80E94EE69EAC20091780410917904CA
:105C600081E08093500264E670E080E090E00E9462
:105C7000204D0E945574C8010E94DD5860E074E018
:105C8000681B790B4AE0CE0101960E94184762E139
:105C900079E0CE0180960E943A4ABE016F5F7F4F45
:105CA000CE0180960E94BC45BC0189ED9EE00E9419
:105CB0007446CE0180960E948946CE0101960E94CC
:105CC000894660E086E00E94B25B63E676E0CE0142
:105CD00001960E94434742E350E068E070E0CE0145
:105CE00001960E94EC75CE0101960E94894669EDED
:105CF0007EE0CE0101960E944B4742E350E06FEFF9
:105D00007FEFCE0101960E94BB74CE0101960E94E6
:105D1000894669E179E0CE0101960E943A4A69ED2F
:105D20007EE0CE0101960E94BC45BC0189ED9EE05B
:105D30000E9474460C9432248091760490917704EA
:105D40000E948A6773C280911002882309F46EC290
:105D50008091770B882329F082E090E00E94736F96
:105D600065C2C0900C02D0900D02E0900E02F0903F
:105D70000F0220E030E040E450E4C701B6010E9489
:105D8000F38718166CF420E030E04AE754E4C701CA
:105D9000B6010E9413850E949D876B017C0106C09D
:105DA00040E3C42E45E7D42EE12CF12C0E9455741B
:105DB00060E080E00E94B25B63E279E08BEC9FE000
:105DC0000E94444B61E080E00E94B25B64E379E0B2
:105DD0008BEC9FE00E94444B64E670E080E090E032
:105DE0000E94204D0E94584D6093CA0A7093CB0ABE
:105DF0008093CC0A9093CD0A0E94584D0091CA0A14
:105E00001091CB0A2091CC0A3091CD0ADC01CB0154
:105E1000801B910BA20BB30B8C159D05AE05BF0526
:105E20000CF004C283E090E00E94736F0E94584D12
:105E300064E170E080E090E00E94204DDDCF809131
:105E4000770B811102C00E9455740E94955064E640
:105E500070E080E090E00E94204D66E876E083EDFF
:105E60009EE00E94E14563ED7EE0CE0101960E9436
:105E70004B4744E150E060E070E0CE0101960E94A3
:105E8000EC75CE0101960E94894667E776E083EDC6
:105E90009EE00E94E14563ED7EE0CE0101960E9406
:105EA0004B4744E150E06FEF7FEFCE0101960E9437
:105EB000BB74CE0101960E9489468CE40E94DF4F9C
:105EC0006B017C0104E010E0A7019601C701B60157
:105ED0000E944389882309F42DC20150110909F455
:105EE00084C264E670E080E090E00E94204D8CE483
:105EF0000E94DF4F6B017C01E7CF62E976E083ED22
:105F00009EE00E94E14563ED7EE0CE0101960E9495
:105F10004B474AE050E060E070E0CE0101960E94FD
:105F2000EC75CE0101960E948946909174042B96DF
:105F30009FAF2B978091EC0A81110DC00E94584DA4
:105F40006093E80A7093E90A8093EA0A9093EB0A57
:105F500081E08093EC0A8091E00A81110DC00E94DB
:105F6000584D6093DC0A7093DD0A8093DE0A9093AB
:105F7000DF0A81E08093E00A1092DB0A1092DA0ACD
:105F80000091DA0A1091DB0A083211050CF085C085
:105F90002B968FAD2B970E94D64CF801EE0FFF1F6A
:105FA000E458F44F918380830E948E5D20E030E0BE
:105FB00040EA50E40E94138520E030E040E85AE3D4
:105FC0000E9413856B017C016093D60A7093D70AF7
:105FD0008093D80A9093D90A409004025090050209
:105FE0006090060270900702A3019201609108027E
:105FF0007091090280910A0290910B020E943D86E5
:106000009B01AC0160E070E080EC90E40E943D8672
:106010004B015C0120E030E0A9010E94AE8420E049
:1060200030E040E650E4811105C0C701B6010E948E
:1060300013851EC0C701B6010E941385A3019201FA
:106040000E943E8620E030E040E850E40E943D8619
:10605000A50194010E94048720E030E040EC50E468
:106060000E94138520E030E040E850E40E943E8624
:106070006093D20A7093D30A8093D40A9093D50A7E
:1060800064E170E080E090E00E94204D0F5F1F4FC0
:106090001093DB0A0093DA0A73CFC090D20AD09033
:1060A000D30AE090D40AF090D50A20E030E0A901AC
:1060B000C701B6010E94F38787FD1EC022E0B70129
:1060C000A601CE0101960E94BD466CE379E0CE01A7
:1060D00080960E943A4ABE016F5F7F4FCE01809644
:1060E0000E94BC45BC0189ED9EE00E947446CE0131
:1060F00080960E94894684C060E479E089ED9EE044
:106100000E945F4681C080911002882309F48EC0EE
:106110008091770B811127C0C0900C02D0900D02A6
:10612000E0900E02F0900F0220E030E04AE754E4E5
:10613000C701B6010E9413850E949D874B015C0137
:1061400020E030E040EA50E4C701B6010E94138528
:1061500020E030E040EA50E40E943E860E949D87A5
:10616000A501940108C021E030E040E050E06AE081
:1061700070E080E090E00E943D6B58C080917F10FD
:1061800090918010892BA1F481E090E09093801091
:1061900080937F108EED93E09093690B8093680B52
:1061A0000E94D25F68EC70E080E090E00E94204D99
:1061B000E0E0F0E019953AC020E042E060E18BECCD
:1061C0009FE00E94DA410E9428560E9455742EC01A
:1061D00010933D0B00933C0B6BE976E089ED9EE05C
:1061E0000E94E14569EC79E0CE0101960E943A4AAD
:1061F0004AE050E060E070E0CE0101960E94EC754C
:10620000CE0101960E94894669ED7EE0CE0101969D
:106210000E944B474AE050E06FEF7FEFCE010196BE
:106220000E94BB74CE0101960E9489468091DD0ECA
:106230009091DE0E0097A9F0419728F4F2E02F1616
:1062400031040CF064C069ED7EE0CE0101960E943D
:106250004B47CE0101960E947367CE0101960E94C2
:10626000894664E670E080E090E00E94204D81C1A4
:106270006AE778E089ED9EE00E94CD450C947D238D
:10628000EC80F12CFE2CEE248D81E80EF11CCE80EA
:10629000D12CDC2CCC248F81C80ED11CA884B12C2D
:1062A000BA2CAA248985A80EB11C21E02B962FAF09
:1062B0002B970C941F2663E974E089ED9EE00E9401
:1062C000E14569ED7EE0CE0180960E944B474AE0B1
:1062D00050E060E070E0CE0180960E94BB74CE0179
:1062E00080960E94894660E874E089ED9EE00E94F5
:1062F000E14580913E0B90913F0B029711F00C9479
:10630000FF2610923F0B10923E0B0C94FF2669ED76
:106310007EE0CE0101960E944B474AE050E06FEFCD
:106320007FEFCE0101960E94BB74CE0101960E94C0
:10633000894689CF21E0B701A601CE0101960E94CE
:10634000BD466FE479E0CE0180960E943A4ABE01D4
:106350006F5F7F4FCE0180960E94BC45BC0189EDE6
:106360009EE00E947446CE0180960E948946CE012E
:1063700001960E94894669ED7EE0CE0101960E9459
:106380004B4742E350E06FEF7FEFCE0101960E9452
:10639000BB74CE0101960E9489460E94997468E5FB
:1063A00079E089ED9EE00E94CD4586E60E94DF4FB0
:1063B0006B017C0104E010E0A7019601C701B60162
:1063C0000E944389882309F449C00150110909F446
:1063D000C9C068EC70E080E090E00E94204D86E645
:1063E0000E94DF4F6B017C01E7CF6CE676E083ED26
:1063F0009EE00E94E14563ED7EE0CE0101960E94A1
:106400004B474AE050E060E070E0CE0101960E9408
:10641000EC75CE0101960E9489466BE579E0CE01CC
:1064200001960E943A4A63ED7EE0CE0101960E94F9
:10643000BC45BC0189ED9EE00E947446CE010196E8
:106440000E94894680913E0B90913F0B039709F083
:1064500074C010923F0B10923E0B6FC021E0B70149
:10646000A601CE0101960E94BD466DE678E0CE0100
:1064700080960E943A4ABE016F5F7F4FCE018096A0
:106480000E94BC45BC018FED9EE00E947446CE0187
:1064900080960E948946CE0101960E9489466BE64D
:1064A00079E0CE0101960E943A4A6FED7EE0CE017E
:1064B00001960E94BC45BC0183ED9EE00E9474469B
:1064C000CE0101960E94894663ED7EE0CE010196E1
:1064D0000E944B474AE050E060E070E0CE01019638
:1064E0000E943A75CE0101960E9489460E949974D5
:1064F00068E579E08FED9EE00E94CD456FED7EE08E
:10650000CE0101960E944B476BE679E0CE010196E1
:106510000E94A54569ED7EE00E94BC45BC0189ED65
:106520009EE00E947446CE0101960E94894683E057
:1065300090E090933F0B80933E0B64E670E080E028
:1065400090E00E94204D8091770B882331F060E22B
:1065500073E080E090E00E94204D88E19CE00E9482
:10656000574864CE69EC79E08FED9EE00E945F466B
:10657000C5CFC75ADF4F0FB6F894DEBF0FBECDBFF1
:10658000DF91CF911F910F91FF90EF90DF90CF900F
:10659000BF90AF909F908F907F906F905F904F9043
:1065A0003F902F9008952F923F924F925F926F925B
:1065B0007F928F929F92AF92BF92CF92DF92EF9293
:1065C000FF920F931F93CF93DF93CDB7DEB728973A
:1065D0000FB6F894DEBF0FBECDBFFC0181E09EE098
:1065E000938782878091FE0D90E0958784878091C4
:1065F000CB0E90E0978786878091FB0D853009F060
:10660000B7C38091030E9091040E885891098D357F
:10661000910588F48091FE0D843041F48091050E3F
:106620009091060E8097479708F407C28091FE0D5F
:10663000843408F0E8C18091FE0D8A3108F448C026
:106640008091010E9091020E843F914050F411868A
:1066500010868FEF9FEFDC0184839583A683B78339
:1066600051C08091030E9091040E85974B9780F551
:1066700017E0E12E1EE0F12E82E090E040E050E0D5
:10668000BA018C010F5F1F4F2091FE0D30E0021701
:1066900013076CF4970122503109D9012D913C91D7
:1066A000275031092730310508F40AC2C801019783
:1066B00095958795918780870C971CF41186108695
:1066C00007C0448355836683778384E090E01CC1D0
:1066D0008091FE0D8A3108F448C08091010E90919E
:1066E000020E8032934008F4B2CF8091030E909155
:1066F000040EC697869708F403C237C044835583B7
:10670000668377838BE090E0FFC0D7012D913C91A9
:10671000255231092B31310508F004C2440F551FB1
:10672000661F771F41600296B4E0EB0EF11C8C01EE
:106730000F5F1F4F2091FE0D30E00217130764F426
:10674000970122503109D9012D913C912C503109EA
:106750002B303105D0F2C801019795958795918727
:1067600080870C975CF6118610868091FE0D823230
:1067700008F44CC08091030E9091040E0697079781
:1067800008F044C047E0C42E4EE0D42E82E090E0F2
:1067900040E050E0BA018C010F5F1F4F2091FE0DC9
:1067A00030E0021713070CF5D6011297ED90FC901C
:1067B00011979D01BEE1EB1AF108A7E1EA16F10479
:1067C00008F0BEC1440F551F661F771F4160D601F8
:1067D0002D913C91B4E0CB0ED11C235031092530D2
:1067E000310510F40296D7CFC8010197959587958A
:1067F0009187808740971CF41186108607C04483D8
:106800005583668377838CE090E07EC07F011C8295
:106810001B8281E090E09A8389838091FE0D8D3008
:1068200008F475C029E733E0AE014D5F5F4FBE014C
:106830006F5F7F4FCF010E945154892B09F067C0D1
:1068400029E733E0AE014D5F5F4FBE016F5F7F4FC1
:10685000C7010E945154019709F059C029E733E05C
:10686000AE014D5F5F4FBE016F5F7F4FC7010E945A
:106870005154892B09F04BC0812C912C540100E01C
:1068800010E08091FE0D90E029813A8128173907A8
:106890007CF529E733E0AE014D5F5F4FBE016F5FCE
:1068A0007F4FC7010E9451546C0129E733E0AE01CC
:1068B0004D5F5F4FBE016F5F7F4FC7010E94515414
:1068C000E1E0CE16D10449F4892B09F5880C991C16
:1068D000AA1CBB1C689480F808C0CD28C1F401979D
:1068E000B1F4880C991CAA1CBB1C0F5F1F4FC9CFA9
:1068F000D70119961C930E931897F70184829582FD
:10690000A682B78281E090E09183808329C21C82B5
:106910001B8281E090E09A838983D7011C968D9138
:106920009C911D97181619060CF061C01A96ED91EE
:10693000FC911B9782E090E09A8389838281938106
:1069400089974E9708F053C083E090E09A8389833B
:10695000848195810B970A9708F049C02CEB31E0B0
:10696000AE014D5F5F4FBE016F5F7F4FC7010E9459
:106970005154892BE1F52CEB31E0AE014D5F5F4FB7
:10698000BE016F5F7F4FC7010E945154019779F597
:10699000412C512C320100E010E029813A81D701CD
:1069A0001C968D919C911D97281739070CF010C1EA
:1069B0002CEB31E0AE014D5F5F4FBE016F5F7F4F4B
:1069C000C7010E9451545C010330110509F0C6C093
:1069D0002CEB31E0AE014D5F5F4FBE016F5F7F4F2B
:1069E000C7010E945154A816B90609F4B7C0D701CF
:1069F0001A96ED91FC911B9782819381C697869799
:106A000008F4F2C03EC18091050E9091060E8254AA
:106A100091098E9708F00FCE20E030E0C12CD12CE8
:106A20007601A901495F514FDA014D915C914950BE
:106A300051094930510598F0FECD8091070E909193
:106A4000080E0997099708F0F1CD118610868FEF8F
:106A50009FEFDC0184839583A683B7838CC1B90142
:106A6000675F714FDB014D915C9147515109423194
:106A70005105C0F4D701C601880F991FAA1FBB1F7B
:106A80006C017D016894C0F82C5F3F4F20383105C0
:106A900041F620E230E031872087C482D582E68249
:106AA000F78269C1DB014D915C9146505109473035
:106AB000510508F0C0CDCC0CDD1CEE1CFF1CE4CF52
:106AC000D7012D913C91235131092F30310550F4DC
:106AD000440F551F661F771F41600296B4E0EB0E0E
:106AE000F11CCFCDD7012D913C912A50310929308D
:106AF000310508F0EDCD440F551F661F771FEDCF10
:106B00008091050E9091060EC697869708F02DCEBF
:106B100089E0E82E8EE0F82E83E090E040E050E03F
:106B2000BA0105CED7012D913C912C5031092A3064
:106B3000310508F01ACE440F551F661F771FF3CD9D
:106B4000D9012D913C912C5031092B30310508F0A1
:106B50005DCE440F551F661F771F39CE2CEB31E0F9
:106B6000AE014D5F5F4FBE016F5F7F4FC7010E9457
:106B700051546C010330110579F42CEB31E0AE0176
:106B80004D5F5F4FBE016F5F7F4FC7010E94515441
:106B9000C816D90609F02BCFA114B10459F4CA9430
:106BA000CD2809F024CF440C551C661C771C689432
:106BB00040F80BC0AA94AB2809F019CFCD2809F0F2
:106BC00016CF440C551C661C771C0F5F1F4FE5CE7B
:106BD00019961C930E931897F7014482558266828A
:106BE000778282E090E090CE848195814B974597A3
:106BF00008F047C0DF0116966F0126ECC20ED11CCB
:106C000020E030E040E050E060E070E080E090E0C4
:106C10000D911C911197095011090830110588F543
:106C200012960D911C911397015111090D30110508
:106C3000D8F401E00E949A8921601496AC15BD0534
:106C400039F7F701248335834683578300E20E9496
:106C5000B5892283338385E090E09183808380E34C
:106C600090E0918780877CC012960D911C911397BC
:106C7000045011090530110520F401E00E949A89A1
:106C8000DCCF8091FE0D893340F08281938189575A
:106C900091098335910508F47CC18091FE0D823203
:106CA00009F46CC0828193818957910983359105DC
:106CB00008F4E6C1828193818C549109C59708F04C
:106CC00064C08091FE0D843031F484819581809779
:106CD000479708F434C28091FE0D843408F455C0FF
:106CE0008481958189549109C39708F04EC09F0112
:106CF0002A5F3F4FAF014A575F4F812C912C5401BF
:106D0000D9016D917C916950710969307105E8F57F
:106D1000D90112966D917C91139766517109613179
:106D2000710508F022C2D501C401880F991FAA1F5E
:106D3000BB1F4C015D01689480F82C5F3F4F241706
:106D40003507F1F620E230E0F70131872087D701DF
:106D500084829582A682B78287E090E08D939C938F
:106D600081E090E0BFC282E08093FB0D1092FE0DA7
:106D700080E090E0B7C283E090E0C6CD828193814D
:106D80000A97099708F460C18DCF8091FE0D863473
:106D900060F1828193810C970B9708F4F6C125C0AE
:106DA000D90112966D917C9113976E5171096731DB
:106DB000710508F01EC2D501C401880F991FAA1FD2
:106DC000BB1F4C015D01689480F84E5F5F4F2C5FE4
:106DD0003F4F4534510509F4F3C1D9016D917C91C0
:106DE0006C5071096B307105D8F28091FE0D8835B9
:106DF00078F182819381855891098B35910508F44A
:106E000008C226C0BC016F5F7F4FD8012D913C9115
:106E1000275031092730310508F00AC2440F551FA9
:106E2000416002960C5F1F4F2091FE0D30E0245010
:106E30003109821793070CF004C2980122503109DE
:106E4000D9012D913C912950310928303105D0F2DA
:106E50008091FE0D8032E1F482819381069706973E
:106E6000B8F4848195810997099790F49F012A5F6E
:106E70003F4FAF01425C5F4F812C912C5401D901EF
:106E80006D917C91665071096630710508F4F3C10B
:106E9000D7011C962D903C901D97B6E02B1631041F
:106EA0000CF461CF8F010A5F1F4F73E0C72ED12C06
:106EB000E5EC8E2EEDE99E2EECE1AE2EE1E8BE2E45
:106EC000F8016081718134976080718080E090E08A
:106ED0000E94B2846D837E838F839887B30180E0A4
:106EE00090E00E94B2842B013C012DEC3CEC4CE480
:106EF0005FE30E9413859B01AC016D817E818F81D0
:106F000098850E94AE8487FD19C02DEC3CEC4CE4C2
:106F10005FE36D817E818F8198850E9413859B013F
:106F2000AC01C301B2010E94AE84E82F880FFF0BB1
:106F3000EE27FF0FEE1FFF27319602C0E0E0F0E0E2
:106F4000A501940163E971E080E091E00E945C8911
:106F50004F01FF0FAA08BB0886269726A826B92648
:106F6000FFEFCF1ADF0A0E5F1F4FC214D30409F0E0
:106F7000A7CFD70114968D929D92AD92BC92179790
:106F800080E290E019969C938E9318978FEF9FEF75
:106F9000E5CE84819581CA97899708F07ECE9F01BE
:106FA0002A5F3F4F812C912C540143E050E0D901DE
:106FB0006D917C916A5071096930710508F06DCE50
:106FC000D90112966D917C911397665171096131C7
:106FD000710550F5D501C401880F991FAA1FBB1F69
:106FE0004C015D01689480F84E5F5F4F2C5F3F4F0E
:106FF0004B335105E1F69F012A583F4FD9012D919E
:107000003C912A5031092930310508F046CE2CE157
:1070100030E0F70131872087D70184829582A682EC
:10702000B7828AE090E09ACED90112966D917C9158
:107030001397665071096730710508F02ECE880CE1
:10704000991CAA1CBB1CD0CF2091FE0DCF01820F32
:10705000911D820F911DDC0112978D919C910A97D1
:10706000099708F01FCEF701118610868FEF9FEF6A
:10707000DC0184839583A683B78386E090E044CCCB
:107080008091FE0D813208F415CE84819581CA97D6
:10709000899708F00FCE9F012A5F3F4F812C912CDA
:1070A000540143E050E0D9016D917C916A5071091F
:1070B0006930710508F0FECDD90112966D917C9171
:1070C0001397665171096131710570F112966D91D6
:1070D0007C911397665071096730710508F0EACD0D
:1070E000880C991CAA1CBB1C4E5F5F4F2C5F3F4F46
:1070F00043325105C1F69F012A5B3F4FD9012D91C3
:107100003C912A5031092930310508F0D3CD20E1D6
:1071100030E0F70131872087D70184829582A682EB
:10712000B78286E090E01ACED501C401880F991F7E
:10713000AA1FBB1F4C015D01689480F8D5CF8681E2
:1071400097810997099708F0C6CDD70119961C9227
:107150001E9218978FEF9FEFDC01F70184839583D0
:10716000A683B78387E090E0CFCBD90112966D91CB
:107170007C911397665071096730710508F005CE50
:10718000880C991CAA1CBB1CD8CD848195810997B9
:10719000099708F02ACE868197818C974F9708F03F
:1071A00024CE8085918589974D9708F01ECE9F014A
:1071B000265F3F4F812C912C540145E050E00DCECD
:1071C0009F0126573F4FD9012D913C912C503109F9
:1071D0002B30310508F009CE20E230E0F70131878D
:1071E0002087D70184829582A682B78288E090E0CA
:1071F000B5CDD90112966D917C91139769507109A3
:107200006930710508F0F1CD880C991CAA1CBB1CD3
:10721000DCCD84819581825491098E9708F018CE37
:107220008F01045C1F4F8DE190E040E050E0FCCD09
:10723000D8012D913C912851310922313105C0F0FE
:10724000CB01019795958795D70119969C938E93BD
:1072500018978A970CF4FCCD052E000C660B770B63
:10726000F701448355836683778389E090E04CCBB4
:10727000440F551FD6CDD90112966D917C9113976D
:107280006951710963317105E8F4D501C401880FB2
:10729000991FAA1FBB1F4C015D01689480F82C5FE9
:1072A0003F4F2417350709F0EACD2EE030E0F70113
:1072B00031872087D70184829582A682B7828FE0AA
:1072C00090E04CCDD90112966D917C911397695045
:1072D00071096930710508F0DBCD880C991CAA1C76
:1072E000BB1CDDCF28960FB6F894DEBF0FBECDBF16
:1072F000DF91CF911F910F91FF90EF90DF90CF9092
:10730000BF90AF909F908F907F906F905F904F90C5
:107310003F902F9008954F925F926F927F929F922D
:10732000AF92BF92CF92DF92EF92FF920F931F9393
:10733000CF93DF93CDB7DEB7A9970FB6F894DEBF32
:107340000FBECDBF982E882321F089EC99E00E94D2
:10735000FD5B0E94685D60E08DE20E943F6460E139
:107360008DE20E943F6468E08DE20E943F6440909D
:107370003B0F50903C0F60903D0F70903E0F498244
:107380005A826B827C82C0903F0FD090400FE09079
:10739000410FF090420FCD82DE82EF82F88680911D
:1073A000430F9091440FA091450FB091460F8EA3CB
:1073B0009FA3A8A7B9A789879A87AB87BC8799207D
:1073C00011F18BE89AE00E94EC5B8E010F5F1F4F7A
:1073D0005E019DE0A90EB11CD8016D917D918D914A
:1073E0009D918D0146E050E00E94005D6BE679E0E2
:1073F00082E59DE00E94444B0A151B0569F789EC64
:1074000099E00E94FD5B23E938E144E85FE3C301B2
:10741000B2010E9413852B013C016D877E878F8707
:10742000988B22E430E645E85FE3C701B6010E948D
:1074300013856B017C01698B7A8B8B8B9C8B25E888
:107440003BEE41E95FE36EA17FA188A599A50E946B
:1074500013856D8B7E8B8F8B988F40923B0F509254
:107460003C0F60923D0F70923E0FC0923F0FD09242
:10747000400FE092410FF092420F6093430F7093E0
:10748000440F8093450F9093460F992009F490C0C4
:107490008EE79AE00E94EC5B8E01035F1F4F7E0136
:1074A000B9E1EB0EF11CF80161917191819191911B
:1074B0008F0142E050E00E94005D6BE679E082E5DA
:1074C0009DE00E94444B0E151F0569F789EC99E079
:1074D0000E94FD5B47E45FE066E070E082E30E94AB
:1074E000DA63A090480FB12CBA2CAA248091470FE0
:1074F000A82AC0904A0FD12CDC2CCC248091490FB3
:10750000C82AE0904C0FF12CFE2CEE2480914B0FFA
:10751000E82A61E77AE082E59DE00E94634A4AE05A
:1075200050E0B50182E59DE00E942B4B6BE679E0CF
:1075300082E59DE00E94444B4AE050E0B60182E5BE
:107540009DE00E942B4B6BE679E082E59DE00E9476
:10755000444B4AE050E0B70182E59DE00E942B4B8E
:1075600089EC99E00E94FD5BC8010E94916468E685
:107570007AE082E59DE00E94634A7E01F5E2EF0E2B
:10758000F11CD8016D917D918D919D918D014AE005
:1075900050E00E94005D6BE679E082E59DE00E948C
:1075A000444B0E151F0569F789EC99E00E94FD5BBD
:1075B00061E08DE10E943F64992091F064E57AE0FA
:1075C00082E59DE00E94634AAE014B5D5F4F61E042
:1075D00070E08DE10E94DA638DA190E00E940F645B
:1075E00062E08EE10E943F6463E08FE10E943F64AD
:1075F00064E080E20E943F64992009F449C068E396
:107600007AE082E59DE00E94634AAE014B5D5F4FE8
:1076100061E070E08EE10E94DA63CDA0D12CAE0172
:107620004B5D5F4F61E070E08FE10E94DA63EDA097
:10763000F12CAE014B5D5F4F61E070E080E20E9493
:10764000DA630DA110E04AE050E0B60182E59DE06A
:107650000E942B4B6BE679E082E59DE00E94444B53
:107660004AE050E0B70182E59DE00E942B4B6BE6BB
:1076700079E082E59DE00E94444B4AE050E0B80189
:1076800082E59DE00E942B4B89EC99E00E94FD5B16
:1076900065E081E20E943F64992091F065E27AE022
:1076A00082E59DE00E94634AAE014B5D5F4F61E061
:1076B00070E081E20E94DA638DA190E00E940F6485
:1076C00066E082E20E943F64992091F06DE07AE0EA
:1076D00082E59DE00E94634AAE014B5D5F4F61E031
:1076E00070E082E20E94DA638DA190E00E940F6454
:1076F00067E083E20E943F64992091F067EF79E0B0
:1077000082E59DE00E94634AAE014B5D5F4F61E000
:1077100070E083E20E94DA638DA190E00E940F6422
:1077200068E084E20E943F64992091F06FED79E077
:1077300082E59DE00E94634AAE014B5D5F4F61E0D0
:1077400070E084E20E94DA638DA190E00E940F64F1
:1077500069E085E20E943F64992091F065EC79E050
:1077600082E59DE00E94634AAE014B5D5F4F61E0A0
:1077700070E085E20E94DA638DA190E00E940F64C0
:107780006AE086E20E943F64992091F06FEA79E016
:1077900082E59DE00E94634AAE014B5D5F4F61E070
:1077A00070E086E20E94DA638DA190E00E940F648F
:1077B0006BE088E20E943F64992091F066E979E0ED
:1077C00082E59DE00E94634AAE014B5D5F4F61E040
:1077D00070E088E20E94DA638DA190E00E940F645D
:1077E0006CE089E20E943F64992009F474C06EE75E
:1077F00079E082E59DE00E94634AAE014B5D5F4FF8
:1078000061E070E089E20E94DA638DA190E00E945D
:107810000F6467E679E082E59DE00E94634A66E0D6
:1078200070E087E20E94256490E00E940F6460E5AA
:1078300079E082E59DE00E94634A65E070E087E2BE
:107840000E94256490E00E940F6469E379E082E57C
:107850009DE00E94634A64E070E087E20E94256434
:1078600090E00E940F6460E279E082E59DE00E9472
:10787000634A62E070E087E20E94256490E00E9423
:107880000F6467E079E082E59DE00E94634A61E071
:1078900070E087E20E94256490E00E940F646EEE23
:1078A00078E082E59DE00E94634A60E070E087E254
:1078B0000E94256490E00E940F646DED78E082E5FF
:1078C0009DE00E94634A63E070E087E20E942564C5
:1078D00090E00E940F6441E067E070E087E20E9460
:1078E000526441E063E070E087E20E94526441E04C
:1078F00063E070E08AE20E945264992071F064ECC7
:1079000078E082E59DE00E94634A63E070E08AE2ED
:107910000E94256490E00E940F6440E063E070E004
:107920008AE20E945264992071F06AEA78E082E566
:107930009DE00E94634A63E070E08AE20E94256451
:1079400090E00E940F6441E062E070E08AE20E94F1
:107950005264992071F06EE878E082E59DE00E9423
:10796000634A62E070E08AE20E94256490E00E942F
:107970000F6440E062E070E08AE20E945264992065
:1079800071F061E778E082E59DE00E94634A62E081
:1079900070E08AE20E94256490E00E940F6441E05A
:1079A00061E070E08AE20E945264992071F065E51E
:1079B00078E082E59DE00E94634A61E070E08AE23F
:1079C0000E94256490E00E940F6440E061E070E056
:1079D0008AE20E945264992071F068E378E082E5BF
:1079E0009DE00E94634A61E070E08AE20E942564A3
:1079F00090E00E940F6441E060E070E08AE20E9443
:107A00005264992071F06CE178E082E59DE00E947B
:107A1000634A60E070E08AE20E94256490E00E9480
:107A20000F6440E060E070E08AE20E9452649920B6
:107A300071F06FEF77E082E59DE00E94634A60E0BD
:107A400070E08AE20E94256490E00E940F6441E0A9
:107A500066E070E087E20E94526441E065E070E019
:107A600087E20E94526441E064E070E087E20E9495
:107A7000526440E062E070E087E20E94526440E0BD
:107A800061E070E087E20E94526440E060E070E0F4
:107A900087E20E945264992009F470C067EE77E093
:107AA00082E59DE00E94634A66E070E08BE20E94FE
:107AB000256490E00E940F6469EC77E082E59DE028
:107AC0000E94634A65E070E08BE20E94256490E0CA
:107AD0000E940F646BEA77E082E59DE00E94634AB2
:107AE00064E070E08BE20E94256490E00E940F64E5
:107AF00062E977E082E59DE00E94634A62E070E01F
:107B00008BE20E94256490E00E940F6469E777E0B1
:107B100082E59DE00E94634A61E070E08BE20E9492
:107B2000256490E00E940F6460E677E082E59DE0C6
:107B30000E94634A60E070E08BE20E94256490E05E
:107B40000E940F646DE477E082E59DE00E94634A45
:107B500063E070E08BE20E94256490E00E940F6475
:107B600068E377E082E59DE00E94634A64E070E0AC
:107B70008CE20E94256490E00E940F6440E064E083
:107B800070E08CE20E945264AE014B5D5F4F61E099
:107B900070E08CE20E94DA636DA1607F66608CE227
:107BA0000E943F64992009F460C064E277E082E5B6
:107BB0009DE00E94634AAE014B5D5F4F61E070E063
:107BC0008CE20E94DA636DA16F7070E066507109FB
:107BD000072E000C880B990B0E94B4849B01AC010A
:107BE00060E070E080E090E40E94B28820E030E045
:107BF00048EC50E40E9413850E9482646DE077E0B7
:107C000082E59DE00E94634AAE014B5D5F4F61E0FB
:107C100070E080E30E94DA634DA150E060E070E024
:107C20002AE082E59DE00E949C4A82E59DE00E9458
:107C3000314B65EF76E082E59DE00E94634A61E0AA
:107C400070E080E30E94256490E00E940F646CED78
:107C500076E082E59DE00E94634A61E070E08FE299
:107C60000E94256490E00E940F6441E061E070E0B2
:107C70008FE20E945264992071F064EC76E082E514
:107C80009DE00E94634A61E070E08EE20E942564FC
:107C900090E00E940F6441E061E070E08EE20E949B
:107CA000526440E067E070E081E30E9452649920F2
:107CB00009F44AC061EB76E082E59DE00E94634AE8
:107CC00067E070E081E30E94256490E00E940F6409
:107CD0006DE679E082E59DE00E94444BAE014B5D8C
:107CE0005F4F61E070E080E00E94DA638DA180D494
:107CF00089EC99E00E94FD5B0DE110E064E779E01A
:107D000082E59DE00E94444B40E150E0B80182E5ED
:107D10009DE00E942B4B6EE977E082E59DE00E949A
:107D2000444BAE014B5D5F4F61E070E0802F0E94DD
:107D3000DA638DA15DD489EC99E00E94FD5B0F5F51
:107D40001F4F0A331105D1F6A9960FB6F894DEBF7E
:107D50000FBECDBFDF91CF911F910F91FF90EF909C
:107D6000DF90CF90BF90AF909F907F906F905F908B
:107D70004F90089521E001C0220F6A95EAF7DC01D7
:107D80001C962C931C971A965C934E931997ED9121
:107D9000FC910484F585E02D60E01994DC01ED91FF
:107DA000FC910684F785E02D41E0199581E090E093
:107DB00008950895089585ED8093BC008091BC00DE
:107DC00084FDFCCF1092F40B08950895CF93DF93B8
:107DD000FC012381222391F0EC01818180956823AD
:107DE000608382810E945E5D68818FEE9DE00E94CB
:107DF00024550E94015D282F30E002C020E030E0D1
:107E000081E090E0232B11F080E090E0DF91CF91B2
:107E10000895EF92FF920F931F93CF938C01FC0173
:107E2000759684E0C0E060FF02C09081C92B669522
:107E3000815031968111F7CF413011F4F801448916
:107E4000F8018585C82BC42B7801FEE0EF0EF11CEC
:107E5000F80162896C2BC701B9DFF801628960956E
:107E60006C23C701CF911F910F91FF90EF90AECF80
:107E70000F931F93CF93DF93062F0F70423019F4A7
:107E800040E0602F0FC0142F262FEC0130E0B90125
:107E900084E0759567958A95E1F7CE01BADF412FA9
:107EA000602FCE01DF91CF911F910F91B2CFFC01D6
:107EB00084858823A1F0218532852115310519F4A7
:107EC000611106C007C02130310521F4611102C0E3
:107ED000858701C015866585CF010E9677CF0895F9
:107EE000DC0180E0615090F09D919827E92FEF70C0
:107EF000F0E0E756F54F249192959F70E92FF0E05E
:107F0000E755F54FE4918E2F8227ECCF0895FC01C1
:107F100090810180F281E02DF8948181892B818309
:107F20002281892F809528232283A7E0B0E0119732
:107F3000F1F7218182238183A3E2B0E01197F1F769
:107F400080817894EFECF0E03197F1F7982381E0AD
:107F500009F480E00895FC0190810180F281E02D18
:107F6000892F809560FF12C0F8942281822382833A
:107F70008181892B8183A3E2B0E01197F1F782819F
:107F8000982B9283789487ED90E011C0F894228129
:107F9000822382838181892B8183AFEFB0E01197A7
:107FA000F1F78281982B928378948FE090E001978B
:107FB000F1F70895CF92DF92EF92FF920F931F9304
:107FC000CF93DF931F92CDB7DEB76C01E62E08E0AA
:107FD00010E0FF24F39461E08F2D8E2109F460E01E
:107FE000C6014983B8DFFF0C015011094981011511
:107FF000110589F7411115C0F894D6011196ED913C
:10800000FC91129791818C9180958923818311969F
:10801000ED91FC91129792818C91809589238283B6
:1080200078940F90DF91CF911F910F91FF90EF9077
:10803000DF90CF900895CF92DF92EF92FF920F934F
:108040001F93CF93DF931F92CDB7DEB78C01F62E2F
:1080500040E065E57983AEDFCF2C7981D72E7601BC
:1080600088E0E80EF11CF60161916F0140E0C80163
:10807000A1DFCE14DF04B9F70F90DF91CF911F91EC
:108080000F91FF90EF90DF90CF900895FC019081C9
:108090000180F281E02DF8948181292F209582239F
:1080A000818378948DE743E050E0815021F1DA013B
:1080B0001197F1F730813923C1F3F894828182233B
:1080C00082838181892B81837894ABE7B7E0119714
:1080D000F1F7F894818128232183A3E1B1E011977E
:1080E000F1F78081982381E009F080E07894E3E65D
:1080F000F6E03197F1F70895EF92FF920F931F93F7
:10810000CF93DF93CDB7DEB728970FB6F894DEBFD5
:108110000FBECDBF8C01DC011696ED91FC91179737
:10812000138615861486DF011B9633961E92AE17B2
:10813000BF07E1F7F80114821582EE24E394BE0133
:108140006F5F7F4FF801868197810E94B25088232C
:1081500009F46BC067E0CE010196C2DE98858913F1
:10816000EECFD8018C91811121C016968D919C91F2
:1081700017978CDFBE016F5F7F4FF8018681978173
:108180005ADF40E064EBD80116968D919C911797C9
:1081900011DFF80186819781BADEF82ED801169694
:1081A0008D919C91179772DFFF20C1F1F801F1804A
:1081B00089818031B1F1BE016F5F7F4FC8010E949C
:1081C0008A4E8F1520F4D80111968C910BC08981AD
:1081D000803111F48CE006C0BE016F5F7F4FC80193
:1081E0000E948A4EF801818384818F5F8483898114
:1081F000883261F030F4803149F0823209F09FCF4B
:1082000005C08B3319F0823409F099CFD801159647
:108210008C9115978F5F15968C9391CFD801EC9226
:10822000C5CFBCE0BF1578F2D5CF28960FB6F8942D
:10823000DEBF0FBECDBFDF91CF911F910F91FF9099
:10824000EF9008950F931F93CF93DF93EC01162FB8
:1082500060E0812F0E94974C612F70E0FB01E45099
:10826000F44FE491E883FB01EA54F44FE491F0E029
:10827000EE0FFF1FE456F44F859194919A83898302
:108280001B861D861C86FE013B968E010D5F1F4FCF
:108290001292E017F107E1F7DF91CF911F910F9153
:1082A0000895DC01ED91FC910684F785E02D40E016
:1082B00019940F931F93CF93DF93EC01423018F082
:1082C0008C8188608C834F836887222329F041301A
:1082D00019F48C8184608C8364E670E080E090E027
:1082E0000E94204D6C8164FD31C0E881F9810684D3
:1082F000F785E02D42E063E0CE0119950BE416E42A
:10830000C8010197F1F7E881F9810684F785E02D2E
:1083100042E063E0CE011995C8010197F1F7E881C9
:10832000F9810684F785E02D42E063E0CE011995DE
:1083300083E592E00197F1F7E881F9810684F785FA
:10834000E02D42E062E0CE01199513C06062CE01DB
:10835000A8DF8BE496E40197F1F76C816062CE01AF
:10836000A0DF83E592E00197F1F76C816062CE01B6
:1083700098DF6C816062CE0194DF84E08D836CE0D5
:10838000CE018FDF61E0CE018CDF8BE39FE10197AF
:10839000F1F782E08E8366E0CE0183DFE881F98128
:1083A0000484F585E02D6FEFCE01DF91CF911F9111
:1083B0000F911994FF920F931F93CF93DF93EC01CA
:1083C000162F042FF22E8B85888B0E94685D61E04A
:1083D00088890E942A6091E0811101C090E0998B08
:1083E0008FEE9DE00E94D4548E878989882331F0D6
:1083F0001F861C8260E0CE010E96E8DC2F2D402FF8
:10840000612FCE01DF91CF911F910F91FF9051CF3E
:108410001F920F920FB60F9211240BB60F922F934B
:108420003F934F935F936F937F938F939F93AF93FC
:10843000BF93EF93FF938091FC0D0E943B4C2091E2
:10844000FF0D3091000E2F5F3F4F3093000E2093B1
:10845000FF0D9091FE0D953618F096E09093FB0D70
:108460009091FB0D9430C9F128F4923069F093306B
:10847000D1F05EC0953009F451C0963009F058C073
:1084800091E09093CB0E51C0811152C02091FF0D0D
:108490003091000E2436310508F442C01092CB0E04
:1084A0001092FE0D1CC0813009F042C0E091FE0D1B
:1084B00091E09E0F9093FE0DF0E02091FF0D309122
:1084C000000EEE0FFF1FEF5FF14F318320831092FC
:1084D000000E1092FF0D94E029C0811117C0E091A9
:1084E000FE0D91E09E0F9093FE0DF0E02091FF0DA8
:1084F0003091000EEE0FFF1FEF5FF14F31832083AD
:108500001092000E1092FF0D93E010C02091FF0D0D
:108510003091000E2536310558F007C0811108C092
:108520001092000E1092FF0D03C095E09093FB0D8A
:108530009091FD0D992329F0811102C02F9A01C05D
:108540002F98FF91EF91BF91AF919F918F917F9164
:108550006F915F914F913F912F910F900BBE0F90B4
:108560000FBE0F901F901895CF92DF92EF92FF925F
:10857000CF93DF93EC01072E000C880B990B0E9420
:10858000B4846B017C0120E030E040E45FE30E94B2
:10859000138520E030E048E452E40E9404870E9402
:1085A0009D87C617D707D4F020E030E040EA5FE3AC
:1085B000C701B6010E94138520E030E048E452E490
:1085C0000E94048720E030E040E85FE30E943E869E
:1085D0000E949D8721E06C177D070CF420E0822F1C
:1085E00090E0DF91CF91FF90EF90DF90CF900895D2
:1085F0000F931F93CF93DF93082F65EF78E082E509
:108600009DE00E94444BC7E0D0E010E0B8010C2E82
:1086100002C0759567950A94E2F76170772742E08A
:1086200050E082E59DE00E942B4B219778F7DF9187
:10863000CF911F910F9108951F920F920FB60F9235
:1086400011240BB60F922F933F934F935F936F9329
:108650007F938F939F93AF93BF93EF93FF938091FB
:10866000B900887F803609F49CC068F5883209F427
:108670005BC090F4803109F454C038F4882309F4C5
:10868000F6C0883009F44DC0F5C0883109F44CC0FB
:10869000803209F45DC0EEC0803409F468C048F44B
:1086A000803309F455C0883309F0E4C08093F20B9D
:1086B000D8C0803509F44FC0883509F45DC08834CE
:1086C00009F0D8C0D6C0883909F4C7C0A8F48837E3
:1086D00009F467C038F4883609F463C0803709F4B8
:1086E00060C0C8C0883809F4B8C0803909F45FC0D8
:1086F000803809F0BFC05BC0803B09F486C038F405
:10870000803A09F466C0883A09F47FC0B3C0803C5F
:1087100009F4A7C0883C09F4A4C0883B09F48AC0C6
:10872000A9C08091CF0B10C09091F10B8091F00BFC
:10873000981770F5E091F10B81E08E0F8093F10BAB
:10874000F0E0E053F44F80818093BB0085EC86C05D
:108750008093F20B8EC0E091F10B81E08E0F80933D
:10876000F10B8091BB00F0E0E053F44F80839091D7
:10877000F10B8091F00B6EC0E091F10B81E08E0F58
:108780008093F10B8091BB00F0E0E053F44F8083C5
:108790008091F30B81116DC081E08093CE0B84EA50
:1087A00061C083E08093F40B10923B0BCFCF80919C
:1087B0003B0B803208F051C0E0913B0B81E08E0F03
:1087C00080933B0B8091BB00F0E0E55EF44F80832B
:1087D000BDCF85EC8093BC001092F40B80913B0BD5
:1087E000803230F4E0913B0BF0E0E55EF44F108214
:1087F00060913B0B70E0E091190BF0911A0B8BE14B
:108800009BE0199510923B0B35C084E08093F40BEC
:108810001092180B1092170BE091150BF091160B9C
:1088200019958091170B811105C081E08093170B7A
:108830001092F50AE091180B81E08E0F8093180BCF
:10884000F0E0EB50F54F80818093BB009091180BC6
:108850008091170B981708F479CF85E88093BC00B6
:1088600009C085EC8093BC001092F40B03C01092F9
:10887000F20BA1DAFF91EF91BF91AF919F918F9190
:108880007F916F915F914F913F912F910F900BBE10
:108890000F900FBE0F901F9018954091170B262F29
:1088A00030E0240F311D21323105DCF42091F40B2E
:1088B0002430C9F4FC0180E090E0861758F4309130
:1088C000170B2191DC01AB50B54FA30FB11D2C93B9
:1088D0000196F3CF8091170B680F6093170B80E020
:1088E000089581E0089582E008950E94E28BCF937D
:1088F000DF93EC0188819981009711F00E94668ACC
:10890000198218821D821C821B821A82DF91CF91EC
:1089100008950F931F93CF93DF93EC018881998182
:10892000009729F02A813B812617370788F48B01AD
:108930006F5F7F4F0E94FE8A009761F09983888362
:108940001B830A832C813D81232B11F4FC011082AF
:1089500081E001C080E0DF91CF911F910F910895D8
:108960008091D30E9091D40E009711F00C94FF7F5C
:1089700060E070E0CB010895AF92BF92CF92DF929A
:10898000EF92FF920F931F93CF93DF932091EF0EFF
:108990003091F00EFC01448155818901041B150BB7
:1089A0004115510559F12115310541F124173507BC
:1089B00028F10217130718F08901015011097C01F1
:1089C000A090EB0EB090EC0EC501DFEFCFEF65018C
:1089D000C00ED11EC816D906A0F0F70160817181C2
:1089E0000E94138C009769F09C012A193B09021719
:1089F000130710F0D22FC32F0196ECCF8FEF9FEF0C
:108A000002C08D2F9C2FDF91CF911F910F91FF906E
:108A1000EF90DF90CF90BF90AF900895FC018081E0
:108A20009181009711F00C94028060E070E0CB011E
:108A30000895AF92BF92CF92DF92EF92FF920F9381
:108A40001F93CF93DF93DC01CD90DC901197C1147D
:108A5000D10409F442C01496CD91DC91159720976A
:108A6000E1F18C0156017501BFEFAB1ABB0AF701AA
:108A70008081082E000C990B0E947E84892B99F727
:108A80002197CC0DDD1D8881082E000C990B0E94CA
:108A90007E84892B91F4AE014F5F5F4F4E195F09C1
:108AA000D80115965C934E931497CE14DF0450F4BE
:108AB000B701C6010E94E68B05C0CE15DF0558F34D
:108AC0002197E1CFD801ED91FC91119714968D91EA
:108AD0009C911597E80FF91F1082DF91CF911F919C
:108AE0000F91FF90EF90DF90CF90BF90AF900895DF
:108AF000EF92FF920F931F93CF93DF93FC0124819A
:108B000035816115710511F480E018C041155105DA
:108B1000A1F07B01EC018A01020F131FB801F9DEFD
:108B2000882391F3288139818C819D81B701820F3F
:108B3000931F0E94EF8B1D830C8381E0DF91CF9107
:108B40001F910F91FF90EF900895CF93DF93EC0169
:108B50006115710559F0FB0101900020E9F731978B
:108B6000AF01461B570BC4DF811102C0CE01BFDE2F
:108B7000CE01DF91CF910895CF93DF93EC01FB01FC
:108B80004481558160817181B3DF811102C0CE01C2
:108B9000AEDECE01DF91CF9108956115710549F0E8
:108BA000FB0101900020E9F73197AF01461B570BFD
:108BB0009FCF80E00895FB014481558160817181E0
:108BC00097CFEF92FF920F931F93CF93DF93EC0118
:108BD0008B016115710549F0CB010E942F807C014A
:108BE000BC01CE0196DE811103C0CE0180DE07C03C
:108BF000FD82EC82B801888199810E942880CE0193
:108C0000DF91CF911F910F91FF90EF9008950F93F7
:108C10001F93CF93DF938C01EB01FC018081918145
:108C20000097B1F0688179816115710579F0428111
:108C300053812C813D814217530740F00E94EF8BF6
:108C40008C819D81F8019583848313C00E94668A7C
:108C500088819981F801918380838A819B819383A4
:108C600082838C819D8195838483198218821B82E3
:108C70001A821D821C82DF91CF911F910F9108955E
:108C8000EF92FF920F931F93CF93DF93EC017B0141
:108C90008A01BA013EDE811103C0CE0128DE07C081
:108CA0001D830C83B701888199810E94EF8BCE01CF
:108CB000DF91CF911F910F91FF90EF900895CF9387
:108CC000DF93EC016115710551F0FB01019000206B
:108CD000E9F73197AF01461B570BD2DF01C007DE22
:108CE000CE01DF91CF910895CF93DF93EC01FB018B
:108CF0008617970751F0608171816115710521F028
:108D000044815581BDDF01C0F2DDCE01DF91CF91FD
:108D10000895FC01808191810C94668AEF92FF9204
:108D20000F931F93CF93DF93CDB7DEB7A1970FB605
:108D3000F894DEBF0FBECDBF7C01CB01BA01F701B5
:108D400011821082138212821582148242E0420F35
:108D50008E010F5F1F4F0E94E07FBC01C701AFDF94
:108D6000A1960FB6F894DEBF0FBECDBFDF91CF91B5
:108D70001F910F91FF90EF900895EF92FF920F9344
:108D80001F93CF93DF93CDB7DEB7A1970FB6F894BB
:108D9000DEBF0FBECDBF7C01CB01BA01F70111824E
:108DA0001082138212821582148242E0420F8E01D9
:108DB0000F5F1F4F0E94E07FBC01C70180DFA196BB
:108DC0000FB6F894DEBF0FBECDBFDF91CF911F91DC
:108DD0000F91FF90EF9008950F931F93CF93DF9320
:108DE000CDB7DEB7A2970FB6F894DEBF0FBECDBFEA
:108DF0008C01CB01BA01F801118210821382128218
:108E00001582148230E0AE014F5F5F4F0E944C80AC
:108E1000BE016F5F7F4FC80152DFA2960FB6F89474
:108E2000DEBF0FBECDBFDF91CF911F910F9108958F
:108E30000F931F93CF93DF93CDB7DEB762970FB633
:108E4000F894DEBF0FBECDBF8C01CB01F8011182BB
:108E50001082138212821582148250E0BE016F5F6D
:108E60007F4F0E943880BE016F5F7F4FC80127DFB0
:108E700062960FB6F894DEBF0FBECDBFDF91CF91E3
:108E80001F910F910895FC011182108213821282AA
:108E90001582148296CEFC011182108213821282F6
:108EA0001582148221CF0895CF92DF92EF92FF9224
:108EB0000F931F93CF93DF936C017A018B01C0E076
:108EC000D0E0CE15DF0589F0D8016D918D01D60176
:108ED000ED91FC910190F081E02DC6011995892B4F
:108EE00011F47E0102C02196ECCFC701DF91CF9132
:108EF0001F910F91FF90EF90DF90CF900895FC01AC
:108F0000A089B1898C91A689B78982FD0FC09C91F7
:108F1000818D8F5F8F73228D821749F0218DDF0144
:108F2000A20FB11D5D969C93818F08958C91089539
:108F3000FC01538D448D252F30E0842F90E0821B5F
:108F4000930B541710F0CF96089501970895FC01E4
:108F5000918D828D981761F0828DDF01A80FB11D70
:108F60005D968C91928D9F5F9F73928F90E0089594
:108F70008FEF9FEF0895FC01918D828D981731F04E
:108F8000828DE80FF11D858D90E008958FEF9FEFA2
:108F90000895FC01918D228D892F90E0805C9F4F78
:108FA000821B91098F739927089588E19CE0F1DF76
:108FB00021E0892B09F420E0822F089585EB9CE0C5
:108FC000E8DF21E0892B09F420E0822F089582E573
:108FD0009DE0DFDF21E0892B09F420E0822F089556
:108FE000FC01848DDF01A80FB11DA35ABF4F2C9146
:108FF000848D90E001968F739927848FA689B78915
:109000002C93A089B1898C9180648C93938D848DED
:10901000981306C00288F389E02D80818F7D8083BC
:109020000895EF92FF920F931F93CF93DF93EC017C
:1090300081E0888F9B8D8C8D981305C0E889F98914
:10904000808185FD23C0F62E0B8D10E00F5F1F4F32
:109050000F731127E02E8C8DE8120BC00FB607FCA2
:10906000FACFE889F989808185FFF5CFCE01B8DF95
:10907000F2CF8B8DFE01E80FF11DE35AFF4FF08216
:109080000B8FEA89FB898081806207C0EE89FF89A6
:109090006083E889F98980818064808381E090E041
:1090A000DF91CF911F910F91FF90EF900895CF9393
:1090B000DF93EC01888D8823C1F0EA89FB898081E8
:1090C00085FD05C0A889B9898C9186FD0EC00FB6B3
:1090D00007FCF5CF808185FFF2CFA889B9898C91F3
:1090E00085FFEDCFCE017CDFE8CFDF91CF910895F2
:1090F00080E090E0892B19F06ADF81111BC080E0CD
:1091000090E0892B41F080E090E0892B21F00E94D3
:109110000000811112C080E090E0892B19F04EDF31
:1091200081110EC080E090E0892B79F03EDF811143
:109130000AC008950E940000E2CF0E940000EBCF19
:109140000E940000EFCF0C940000089590E0FC0115
:109150003197E231F10508F04EC08827EB56FF4FFA
:109160008F4F0C949289809180008F7703C08091FB
:1091700080008F7D80938000089580918000877F9C
:10918000F9CF84B58F7702C084B58F7D84BD0895F3
:109190008091B0008F7703C08091B0008F7D809365
:1091A000B0000895809190008F7707C08091900063
:1091B0008F7D03C080919000877F809390000895F9
:1091C0008091A0008F7707C08091A0008F7D03C0A1
:1091D0008091A000877F8093A00008958091200156
:1091E0008F7707C0809120018F7D03C0809120017F
:1091F000877F8093200108950F931F93CF93DF9370
:109200008C01EB0188E2FB0111928A95E9F74BE0B2
:1092100050E06FEB79E0CE010E94048C1B8681E068
:1092200090E0A0E0B0E08C879D87AE87BF87F80113
:1092300085899689A789B08D888B998BAA8BBB8BE2
:1092400082E090E0A0E0B0E08C8B9D8BAE8BBF8B7A
:109250001CA21DA21EA21FA280E090E0A8E4B4E41C
:10926000888F998FAA8FBB8F80E090E0A8E4B4EC40
:109270008C8F9D8FAE8FBF8F8DEC9CECACE4BEE3EA
:1092800088A399A3AAA3BBA3DF91CF911F910F91AC
:1092900008954F925F926F927F928F929F92AF92BA
:1092A000BF92CF92DF92EF92FF920F931F93CF93D3
:1092B000DF938C01EB0184E2FB0111928A95E9F7BF
:1092C0008EE10E945E5D83E090E00E94CD5F0E948F
:1092D000015D66E08EE10E942A608091CC0B90E0F7
:1092E0002091CD0B821B910986309105ECF38FEE16
:1092F0009DE00E94D454882E8FEE9DE00E94D454AD
:10930000982E8FEE9DE00E94D454682E8FEE9DE043
:109310000E94D454782E8FEE9DE00E94D454482EA3
:109320008FEE9DE00E94D454582EB82CA12CB5018C
:109330006929072E000C880B990B0E94B4844B01FD
:109340005C01F8016583768387839087D42CC12CD8
:10935000B6016529072E000C880B990B0E94B48476
:10936000F8016187728783879487F62CE12CB70117
:109370006729072E000C880B990B0E94B484F80112
:10938000658776878787908B118A128A138A148A59
:1093900084E290E0A0E0B0E088839983AA83BB8355
:1093A00085899689A789B08D8C839D83AE83BF8381
:1093B00082E090E0A0E0B0E088879987AA87BB8729
:1093C000188A198A1A8A1B8AC0904C02D0904D02C2
:1093D000E0904E02F0904F02A7019601C501B40142
:1093E0000E94048720E030E048EC52E40E9413859C
:1093F0006C8B7D8B8E8B9F8BA7019601F80161850D
:109400007285838594850E94048720E030E048ECD3
:1094100052E40E941385688F798F8A8F9B8F2091E9
:1094200048023091490240914A0250914B02F801A2
:1094300065857685878590890E94048720E030E0E5
:1094400048EC52E40E9413856C8F7D8F8E8F9F8F26
:1094500081E0DF91CF911F910F91FF90EF90DF900E
:10946000CF90BF90AF909F908F907F906F905F90C4
:109470004F900895FC01118210821382128215828E
:1094800014826115710549F0FB0101900020E9F794
:109490003197AF01461B570BF3CB0895DC01ED91DB
:1094A000FC910190F081E02D1994DC01ED91FC918B
:1094B000DB0114964D915C9115976D917C91028022
:1094C000F381E02D1994EF92FF920F931F93CF93A6
:1094D000DF938C017B01C0E0D0E0F701EC0FFD1FB2
:1094E0006491662361F0D801ED91FC910190F081C7
:1094F000E02DC8011995892B11F02196EECFCE01F0
:10950000DF91CF911F910F91FF90EF90089561151A
:10951000710579F0FB0101900020E9F73197AF0167
:10952000461B570BDC01ED91FC910280F381E02D8D
:10953000199480E090E008954F925F926F927F922D
:10954000EF92FF920F931F93CF93DF93CDB7DEB7C8
:10955000A1970FB6F894DEBF0FBECDBF7C01FA0114
:10956000CB0119A2223008F42AE08E010F5D1F4FB3
:10957000422E512C612C712CBF01A30192010E943B
:109580000C86F901CA01015011096A3014F4605DBA
:1095900001C0695CD8016C93232B242B252B61F728
:1095A000B801C701B4DFA1960FB6F894DEBF0FBEB5
:1095B000CDBFDF91CF911F910F91FF90EF907F90E2
:1095C0006F905F904F900895CF92DF92EF92FF924D
:1095D0000F931F93CF93DF93EC016A017B01211559
:1095E000310579F4E881F9810190F081E02D642F53
:1095F000DF91CF911F910F91FF90EF90DF90CF906F
:1096000019942A303105D9F477FF18C06DE246DF8E
:109610008C0144275527BA014C195D096E097F0951
:109620002AE0CE0189DF800F911FDF91CF911F913A
:109630000F91FF90EF90DF90CF9008952AE0B7014F
:10964000A601CE01DF91CF911F910F91FF90EF9076
:10965000DF90CF9071CF9A01AB01770F660B770B3C
:10966000B3CF67EC79E053CF0F931F93CF93DF9382
:10967000EC011BDF8C01CE01F4DF800F911FDF9125
:10968000CF911F910F91089542CF1F920F920FB665
:109690000F9211240BB60F922F933F934F935F932A
:1096A0006F937F938F939F93AF93BF93EF93FF93AA
:1096B00088E19CE095DCFF91EF91BF91AF919F9184
:1096C0008F917F916F915F914F913F912F910F906B
:1096D0000BBE0F900FBE0F901F9018951F920F9208
:1096E0000FB60F9211240BB60F922F933F934F9307
:1096F0005F936F937F938F939F93AF93BF93EF93FA
:10970000FF9388E19CE0FBDBFF91EF91BF91AF916C
:109710009F918F917F916F915F914F913F912F9189
:109720000F900BBE0F900FBE0F901F9018951F92B9
:109730000F920FB60F9211240BB60F922F933F93F7
:109740004F935F936F937F938F939F93AF93BF9349
:10975000EF93FF9385EB9CE043DCFF91EF91BF918A
:10976000AF919F918F917F916F915F914F913F91B9
:109770002F910F900BBE0F900FBE0F901F9018955A
:109780001F920F920FB60F9211240BB60F922F93C8
:109790003F934F935F936F937F938F939F93AF9379
:1097A000BF93EF93FF9385EB9CE0A9DBFF91EF91D3
:1097B000BF91AF919F918F917F916F915F914F91E9
:1097C0003F912F910F900BBE0F900FBE0F901F90E7
:1097D00018951F920F920FB60F9211240BB60F928D
:1097E0002F933F934F935F936F937F938F939F93A9
:1097F000AF93BF93EF93FF9382E59DE0F1DBFF9181
:10980000EF91BF91AF919F918F917F916F915F91F8
:109810004F913F912F910F900BBE0F900FBE0F9065
:109820001F9018951F920F920FB60F9211240BB62E
:109830000F922F933F934F935F936F937F938F93E9
:109840009F93AF93BF93EF93FF9382E59DE057DB28
:10985000FF91EF91BF91AF919F918F917F916F9108
:109860005F914F913F912F910F900BBE0F900FBEC4
:109870000F901F901895CF93DF93282F30E0F901B8
:10988000EE5BF34F8491F901E450F44FD491F90168
:10989000EA54F44FC491CC2389F0811157DCEC2FAA
:1098A000F0E0EE0FFF1FE456F44FA591B491EC9158
:1098B000ED2381E090E021F480E002C080E090E0C0
:1098C000DF91CF910895862FD6CF1F93CF93DF934B
:1098D000282F30E0F901EE5BF34F8491F901E45059
:1098E000F44FD491F901EA54F44FC491CC23C1F060
:1098F000162F81112BDCEC2FF0E0EE0FFF1FEE573F
:10990000F44FA591B4918FB7F894111105C09C91B3
:10991000ED2FE095E92302C0EC91ED2BEC938FBF86
:10992000DF91CF911F910895862F642FCECFCF93D3
:10993000DF9390E0FC01E450F44F2491FC01EA54E1
:10994000F44F8491882361F190E0880F991FFC0106
:10995000E859F44FC591D491FC01EE57F44FA5910D
:10996000B491611109C09FB7F89488812095822332
:109970008883EC912E230BC0623061F49FB7F8947A
:109980003881822F809583238883EC912E2B2C9312
:109990009FBF06C08FB7F894E8812E2B28838FBF16
:1099A000DF91CF910895862F642FC1CF863308F0C1
:1099B000865390917B00282F2870977F922B90934D
:1099C0007B0087702091500290E4299F9001112420
:1099D000822B80937C0080917A00806480937A004F
:1099E00080917A0086FDFCCF8091780020917900EB
:1099F00090E0922B08953FB7F89480916F0B90916F
:109A0000700BA091710BB091720B26B5A89B05C08D
:109A10002F3F19F00196A11DB11D3FBFBA2FA92FED
:109A2000982F8827820F911DA11DB11DBC01CD016A
:109A300042E0660F771F881F991F4A95D1F7089556
:109A40008F929F92AF92BF92CF92DF92EF92FF924E
:109A50006B017C01D0DF4B015C01C114D104E10436
:109A6000F104E9F0C8DFDC01CB0188199909AA09E2
:109A7000BB09883E9340A105B10578F321E0C21AE5
:109A8000D108E108F10888EE880E83E0981EA11C39
:109A9000B11CC114D104E104F10421F7DECFFF9021
:109AA000EF90DF90CF90BF90AF909F908F900895F0
:109AB0002FB7F89460916B0B70916C0B80916D0BCC
:109AC00090916E0B2FBF08951F920F920FB60F92B9
:109AD00011242F933F938F939F93AF93BF938091C4
:109AE0006B0B90916C0BA0916D0BB0916E0B309144
:109AF0006A0B23E0230F2D3720F40196A11DB11D21
:109B000005C026E8230F0296A11DB11D20936A0B04
:109B100080936B0B90936C0BA0936D0BB0936E0BBB
:109B200080916F0B9091700BA091710BB091720BA3
:109B30000196A11DB11D80936F0B9093700BA093A4
:109B4000710BB093720BBF91AF919F918F913F9129
:109B50002F910F900FBE0F901F9018958F929F928C
:109B6000AF92BF92CF92DF92EF92FF920F931F932B
:109B7000CF93DF93EC018E819F810E94464040E0AD
:109B80006CEC8E819F810E94DA3F488164E48E8173
:109B90009F810E94DA3F8A81882309F43FC0E981CE
:109BA000E950E33040F4F0E0EE0FFF1FEC51FB4FC3
:109BB0000081118102C00EEE12E08B818823E9F052
:109BC000888181111AC074DF4B015C016801110F9B
:109BD000EE08FF088E819F810E94873F8130F1F05F
:109BE00067DFDC01CB018C199D09AE09BF0988151F
:109BF0009905AA05BB0570F311C0B801110F880BB8
:109C0000990BDF91CF911F910F91FF90EF90DF9013
:109C1000CF90BF90AF909F908F9012CFDF91CF9158
:109C20001F910F91FF90EF90DF90CF90BF90AF907A
:109C30009F908F9008954F925F926F927F928F9234
:109C40009F92AF92BF92CF92DF92EF92FF920F93CB
:109C50001F93CF93DF931F921F92CDB7DEB72C01D6
:109C60008A01FC018681978169837A830E9446403C
:109C700069817A818823C9F1F201868197810E94E6
:109C80001B4040E06EEBF201868197810E94DA3F33
:109C900078014801F9E08F0E911CF201668077800F
:109CA00088E0A82EB12CCC24C394D12CC3010E94EF
:109CB000873F8111DC28CC0CF1E0AF1AB108B1F775
:109CC000F701D1927F01E815F90539F7F201868194
:109CD00097810E944640813041F468E0C8010E94AB
:109CE000703F91E0F8012085821390E0892F0F905A
:109CF0000F90DF91CF911F910F91FF90EF90DF9028
:109D0000CF90BF90AF909F908F907F906F905F901B
:109D10004F900895CF93DF93CDB7DEB729970FB655
:109D2000F894DEBF0FBECDBFAE014F5F5F4F83DF44
:109D3000882389F08D818F3361F020F48F3159F4BD
:109D400089E00CC08F3519F08F3739F004C08BE0F3
:109D500005C08AE003C080E001C08CE029960FB600
:109D6000F894DEBF0FBECDBFDF91CF910895DF9293
:109D7000EF92FF920F931F93CF93DF937C018B01A0
:109D8000D42EDC011696ED91FC911797138615865B
:109D90001486DF011B9633961E92AE17BF07E1F7BC
:109DA000C0E0B801D70116968D919C911797DAD132
:109DB000D82F811102C0D0E00EC0CD1108C067E0DD
:109DC000C8010E94703FF8019781891721F0CF5F89
:109DD000DC1688F3E6CF8D2FDF91CF911F910F9185
:109DE000FF90EF90DF9008950F931F93CF93DF9331
:109DF000CDB7DEB761970FB6F894DEBF0FBECDBF0B
:109E00008C01462FBE01665F7F4FB1DF811105C017
:109E100060E070E08EEF92EC4AC0AE014F5F5F4FA2
:109E2000BE01665F7F4FC80106DF882359F1698153
:109E300048E0649FB00111248A81282F30E0322F3E
:109E40002227330F330F330F262B372B8A85803190
:109E5000E1F4688570E08F81AB01481B5109CA01AC
:109E60009695982F8827979587950E947F896051AE
:109E70007109207F53E0220F331F5A95E1F7620FDB
:109E8000731F04C060E874EE01C0B901613854EE7C
:109E900075070CF4BDCF072E000C880B990B0E94A0
:109EA000B48420E030E040E05CE30E9413856196DA
:109EB0000FB6F894DEBF0FBECDBFDF91CF911F91DB
:109EC0000F91089596E0899FD0011124A35BB04FB4
:109ED00090967C936E935F9791E091969C93919767
:109EE0009091B90FE091BA0FF091BB0F992339F01F
:109EF000309751F0811108C08091690F04C03097EC
:109F000019F05C968C91199408950F931F93CF9339
:109F1000DF93C82FD62F86E0C89FF0011124E35BA2
:109F2000F04F11A2878D90A181309105E1F01CF4D2
:109F3000892B49F03FC08230910591F10397D1F50B
:109F400060E070E031C06623A9F161E070E08C2F21
:109F5000B9DFAEDD6093A50F7093A60F8093A70FB6
:109F60009093A80F27C0A4DD0091A50F1091A60F14
:109F70002091A70F3091A80FAB01BC01401B510BE2
:109F8000620B730B8091B70F9091B80FA0E0B0E017
:109F900084179507A607B70718F462E070E004C0BD
:109FA000D11108C063E070E08C2FDF91CF911F9139
:109FB0000F9188CFDF91CF911F910F9108953F921C
:109FC0004F925F926F927F928F929F92AF92BF92C9
:109FD000CF92DF92EF92FF920F931F93CF93DF9375
:109FE00000D01F921F92CDB7DEB7982E61DD2B01F6
:109FF0003C0120ED420E27E0521E611C711C60E006
:10A000008091BC0F62DC35E0832ECE0101966C019D
:10A01000AA24A394B12C55E0352E380EF601282D34
:10A0200011922A95E9F7860127E0E22EF12C809122
:10A03000BD0F21DC019731F43BDD64157505860504
:10A040009705A8F38091BD0F16DC892B31F430DD24
:10A050006415750586059705A8F38091BE0F0BDC86
:10A06000892B51F0F8012081C5010E2C01C0880F09
:10A070000A94EAF7822B8083F1E0EF1AF108B8F630
:10A080000F5F1F4F3012D0CF13DD641575058605A5
:10A09000970548F061E08091BC0F17DC60E070E04C
:10A0A00080EC9FE72BC089818911B8CF9B818A8181
:10A0B000980F990D8C818913B1CF8D818D3009F066
:10A0C000ADCF61E08091BC0F00DC6A818B8170E0D4
:10A0D000762F6627680F711D072E000C880B990BD1
:10A0E0000E94B48420E030E040E85DE30E941385E4
:10A0F00023E333E948E853E40E943D860F900F9034
:10A100000F900F900F90DF91CF911F910F91FF90C3
:10A11000EF90DF90CF90BF90AF909F908F907F9007
:10A120006F905F904F903F90089585EB9CE00E9468
:10A130005748E5EBFCE0A289B3898C918F7E8C9324
:10A14000A289B3898C91877F8C93A289B3898C91E2
:10A150008F778C93A289B3898C918F7D8C93828D1C
:10A16000818F0895AF92BF92CF92DF92EF92FF92CC
:10A170000F931F93CF93DF931F92CDB7DEB75C0190
:10A18000D62EE72EFC018585811105C0C5010E94F0
:10A190004640811106C0F50113861586148680E0BD
:10A1A00065C040E060EFC5010E94DA3F01E0F12C9C
:10A1B000C12C11E0C5010E94873F682FC50169834A
:10A1C0000E94873F6981613019F48130B9F433C04E
:10A1D0004F2D50E068131BC0F5018385181730F42C
:10A1E000E40FF51F8381802349F402C0181731F072
:10A1F00060E0193058F4F501148708C0F501EF0D3F
:10A20000F11D8381802B838361E009C0C12EF5019C
:10A21000E40FF51F9381802F809589238383C501E7
:10A220000E94AB3F1F5F000F11F4F39401E0F7E0D1
:10A23000FF1508F0BFCF113408F4ADCFF501C38688
:10A24000C11002C081E08587F5018381882309F46C
:10A25000A2CFD5011396ED2DFE2D9501255F3F4F21
:10A260008D918193A217B307D9F781E00F90DF9109
:10A27000CF911F910F91FF90EF90DF90CF90BF9003
:10A28000AF9008959F92AF92BF92CF92DF92EF92DC
:10A29000FF920F931F93CF93DF93CDB7DEB76197F4
:10A2A0000FB6F894DEBF0FBECDBF8C018CE0F80175
:10A2B0008183C12CD12C2FE5E22E3FE7B32E4FE155
:10A2C000A42E5FE3952EF801848190E0C816D9068C
:10A2D0000CF09DC04C2DBE01665F7F4FC80147DD6D
:10A2E000F8018181893038F0F82EFCE0F81728F465
:10A2F0009CE0F92E02C089E0F82E8A85803131F089
:10A30000BE01665F7F4FC80105DD01C08CE08F157F
:10A3100009F479C0AE014F5F5F4FBE01665F7F4FAA
:10A32000C80189DC882309F46EC08A85803109F46C
:10A330006AC08BE0F81651F0ECE0FE1629F0FAE066
:10A34000FF1206C09D8205C0BD8203C0ED8201C020
:10A35000AD82F801868197810E944640BE01665F0A
:10A360007F4FF801868197810E941B4040E06EE498
:10A37000F801868197810E94DA3F40E06B81F80105
:10A38000868197810E94DA3F40E06C81F8018681E6
:10A3900097810E94DA3F8A85803139F040E06D81F3
:10A3A000F801868197810E94DA3FF80186819781C2
:10A3B0000E944640BE01665F7F4FF801868197810B
:10A3C0000E941B40F801408168E4868197810E94C9
:10A3D000DA3F64E170E080E090E032DBF8018081F8
:10A3E000882329F06AE070E080E090E029DBF80142
:10A3F000868197810E944640F8018181F81608F411
:10A40000F82EF801F182FFEFCF1ADF0A5CCF6196D8
:10A410000FB6F894DEBF0FBECDBFDF91CF911F9175
:10A420000F91FF90EF90DF90CF90BF90AF909F90F3
:10A4300008950F931F93CF93DF9360E48BEC9FE01D
:10A440000E94514183E790E00197F1F7C1E5D2E026
:10A450000BE910E069918BEC9FE00E94CE3EC801B1
:10A460000197F1F782E0C935D807A1F7DF91CF91C5
:10A470001F910F910895FC01448155818091EF0E49
:10A480009091F00E8417950780F08091EB0E9091DB
:10A49000EC0E009751F0608171816115710529F012
:10A4A0000E94F68B21E0892B09F020E0822F08958D
:10A4B000FF920F931F93CF93DF93CDB7DEB72B9708
:10A4C0000FB6F894DEBF0FBECDBF2FDE40E855E2D9
:10A4D00060E070E085EB9CE00E948B7664E670E0C3
:10A4E00080E090E0ADDA8CED95E0A0E0B0E0809304
:10A4F000B90C9093BA0CA093BB0CB093BC0C64E65F
:10A5000070E080E090E09CDA8FEF898381E08A83BD
:10A5100086E88B831C821D821E821F82188689E733
:10A52000898785EB9CE00E94574862E370E080E0F9
:10A5300090E086DA85EB9CE00E94984708974CF003
:10A5400049E050E0BE016F5F7F4F85EB9CE00E94C9
:10A55000544762E370E080E090E072DA85EB9CE0C3
:10A560000E94C947892B01F185EB9CE00E94984726
:10A57000089784F465E070E080E090E061DA00E044
:10A5800010E0F12C85EB9CE00E94C94702301105D8
:10A59000A4F50CC049E050E0BE016F5F7F4F85EB32
:10A5A0009CE00E945447E6CFF12C27C085EB9CE04D
:10A5B0000E94C947892B99F465E070E080E090E043
:10A5C0003FDA02301105F1F69A8589819813DACFC6
:10A5D0009B858B819813D6CFFF24F394D3CF85EB43
:10A5E0009CE00E94A747EAE0F0E0EC0FFD1FE00FBF
:10A5F000F11F80830F5F1F4FDFCF62E370E080E0C9
:10A6000090E01EDA92DD8F2D2B960FB6F894DEBF08
:10A610000FBECDBFDF91CF911F910F91FF90089595
:10A620006F927F928F929F92AF92BF92CF92DF9262
:10A63000EF92FF920F931F93CF93DF9381E080936C
:10A64000B90F36DA0091A90F1091AA0F2091AB0F24
:10A650003091AC0FAB01BC01401B510B620B730B73
:10A660008091B50F9091B60FA0E0B0E084179507E8
:10A67000A607B70708F003C1C0E08091B30FC81761
:10A6800058F4E091AF0FF091B00FEC0FF11D62E0C4
:10A6900080814DD9CF5FF1CF712C812C912C540149
:10A6A00083948091B40F781608F05AC0072D10E0FB
:10A6B000E091B10FF091B20FE00FF11F61E08081E6
:10A6C00036D9E091B10FF091B20FE00FF11F60E0C9
:10A6D0008081FBD8D501C401072C04C0880F991FC5
:10A6E000AA1FBB1F0A94D2F76C017C01E094F0947E
:10A6F000612C8091B30F6816F0F4C62DD0E0E09184
:10A70000AF0FF091B00FEC0FFD1F8081B4D82496ED
:10A71000CC0FDD1FC35BD04F892B29F48881998131
:10A720008C299D2904C0888199818E219F2199833C
:10A7300088836394DECFE091B10FF091B20FE00F08
:10A74000F11F61E08081C1D88091B10F9091B20F6B
:10A75000FC01E00FF11F60E08081E9D87394A1CF84
:10A76000E9E6FFE08FEF9FEF23813481232B21F473
:10A77000108292838183158236962FE0E53AF207A4
:10A7800099F710E096E0F92E8091B30F181708F0B2
:10A7900051C000E0C12FD0E0CC0FDD1FCB5AD04F0D
:10A7A0002091B40F021708F043C068817981002E10
:10A7B00002C0769567950A94E2F761707727129F39
:10A7C00090011124200F311DE091AD0FF091AE0FDB
:10A7D000E20FF31F4081EDE4FFE080E0A58DB68D30
:10A7E000A217B30711F461701AC08F5F36968A30D2
:10A7F000A9F7672BD9F0E9E6FFE080E090E050810F
:10A8000051110FC0F89EF001F99EF00D1124E35B89
:10A81000F04F448F368F258F10A2178E61E075DBC5
:10A8200005C0019636968A30910549F70F5FB8CF7B
:10A830001F5FAACF80E090E0C0E0FC01E35BF04F37
:10A8400021A12111C1E006968C339105B1F730D9D1
:10A850006093A90F7093AA0F8093AB0F9093AC0FE6
:10A86000CC2369F080916E0F882349F080916C0FA2
:10A8700090916D0F019719F48091690F03C01092A8
:10A88000B90F80E0DF91CF911F910F91FF90EF9072
:10A89000DF90CF90BF90AF909F908F907F906F9000
:10A8A00008958F929F92AF92BF92CF92DF92EF92D4
:10A8B000FF920F931F93CF93DF93DB01CD91DC9138
:10A8C000DC011C96ED91FC911D97CE17DF070CF073
:10A8D0004AC0FE01EE0FFF1F1A968D919C911B97A7
:10A8E000E80FF91F80809180C170DD27B1E0CB2790
:10A8F000209719F404E610E002C00CE91FEF79017B
:10A900005A016B01020F131FB801C4010E94B44227
:10A91000892B99F40E0D1F1DB801C4010E94B44289
:10A92000892B71F4B8016E0D7F1DC4010E94B442E1
:10A93000892BE1F023E030E005C021E030E002C0E7
:10A9400022E030E0F5018081918101968217930722
:10A9500034F011821082F6018081918101969183F9
:10A960008083CE0105C081E090E002C08FEF9FEFB1
:10A97000DF91CF911F910F91FF90EF90DF90CF90DB
:10A98000BF90AF909F908F900895E091CD0B8091F4
:10A99000CC0BE81730F4F0E0E751F04F808190E005
:10A9A00008958FEF9FEF08959091CD0B8091CC0B80
:10A9B000981750F4E92FF0E0E751F04F208130E094
:10A9C0009F5F9093CD0B02C02FEF3FEFC901089519
:10A9D0008091CC0B90E02091CD0B821B91090895C2
:10A9E000089580E090E00895CF92DF92EF92FF9279
:10A9F0000F931F93CF93DF937C01262F972F8A010C
:10AA00008091F50B882391F0C62FD72F6E01C40ECD
:10AA1000D51ECC15DD0571F06991D701ED91FC9142
:10AA20000190F081E02DC7011995F3CF642F822F9B
:10AA30000E944D44C801DF91CF911F910F91FF906B
:10AA4000EF90DF90CF900895CF93DF931F92CDB713
:10AA5000DEB769832091F50B2223D1F02091170CEA
:10AA6000203240F021E030E0FC013383228380E09B
:10AA700090E015C08091F60BE82FF0E0E950F44F1C
:10AA8000998190838F5F8093F60B8093170C05C09C
:10AA900061E0CE0101960E944D4481E090E00F906C
:10AAA000DF91CF9108950C94668A0F931F93CF93F3
:10AAB000C091820460E08C2F0E94654C83E090E09E
:10AAC0000197F1F761E08C2F0E94654C83E290E0E2
:10AAD0000197F1F760E08C2F0E94654C8091800413
:10AAE000909181049927FC01E450F44F6491FC019A
:10AAF000EA54F44FE491F0E0EE0FFF1FE456F44FF8
:10AB00008591949100E412E42FE030E0462F0E94FA
:10AB1000F276611571058105910549F0DC01CB01E3
:10AB20000196A11DB11DBC01CD019F7003C060E065
:10AB300070E0CB010E94B28420E030E048EC52E4A7
:10AB40000E9404872091780B3091790B40917A0B09
:10AB500050917B0B0E94138520E030E44CE156E4D9
:10AB60000E94048720E030E040E05FE30E9413850C
:10AB7000CF911F910F910895089523E333E948E899
:10AB800053E40E94048720E030E040E85FE30E9445
:10AB90003E860E94028926E636EA45EA53E40E9490
:10ABA00013856093780B7093790B80937A0B909355
:10ABB0007B0B0895CF92DF92EF92FF9276DF6B01CD
:10ABC0007C0120E030E040E050E40E94F38718165A
:10ABD0001CF46BDF6B017C0120E030E040E050E4CE
:10ABE000C701B6010E94F38718161CF45EDF6B01E3
:10ABF0007C0120E030E040E050E4C701B6010E9453
:10AC0000F38718161CF451DF6B017C0120E030E063
:10AC100040E050E4C701B6010E94F38718162CF4F7
:10AC2000FF90EF90DF90CF9040CFC701B601FF902B
:10AC3000EF90DF90CF900895EBECFFE065816B7FA4
:10AC400065836860CF010E94514110927E0408958F
:10AC500081E080937E04EBECFFE06581862F8460C9
:10AC600085836C60CF010C945141CF93DF9300D06A
:10AC700000D0CDB7DEB780917F04811136C061E08E
:10AC800089E10E94654C20E042E060E18BEC9FE0AE
:10AC90000E94DA41CEDB81E080937F0480937E04C2
:10ACA00064E97CE0CE0101960E9443474AE050E00F
:10ACB00060E070E0CE0101960E94EC75CE01019635
:10ACC0000E94894668E87CE0CE0101960E944347D5
:10ACD0004AE050E060E070E0CE0101960E94BB7453
:10ACE000CE0101960E9489460CC080917E04882383
:10ACF00041F0A2DF60E089E10E94654C10927F0480
:10AD000001C0A6DF26960FB6F894DEBF0FBECDBFFA
:10AD1000DF91CF9108952F923F924F925F926F9261
:10AD20007F928F929F92AF92BF92CF92DF92EF92DB
:10AD3000FF920F931F93CF93DF93CDB7DEB7649746
:10AD40000FB6F894DEBF0FBECDBF7C01EED940E850
:10AD500055E260E070E085EB9CE00E948B7664E653
:10AD600070E080E090E00E94204D8CED95E0A0E046
:10AD7000B0E08093B90C9093BA0CA093BB0CB09345
:10AD8000BC0C64E670E080E090E00E94204D8FEF04
:10AD9000898381E08A8386E88B831C821D821E82E0
:10ADA0001F82188689E78987C701880F991F9C8BA6
:10ADB0008B8B212C312CC12CD12C812C912C54012A
:10ADC000CE14DF0434F0B1D9C114D104A1F176015D
:10ADD00032C08B899C8928163906ACF785EB9CE03C
:10ADE0000E94984708974CF049E050E0BE016F5F21
:10ADF0007F4F85EB9CE00E94544765E070E080E067
:10AE000090E00E94204D00E010E0412C512C3201D6
:10AE100085EB9CE00E94C947892B31F484E04816F9
:10AE20005104610471041CF4023011057CF19FEFA0
:10AE3000291A390AC5CFC501B4010E94B4844B0157
:10AE40005C01B701FF0C880B990B0E94B4849B0135
:10AE5000AC01C501B4010E94048764960FB6F89452
:10AE6000DEBF0FBECDBFDF91CF911F910F91FF903D
:10AE7000EF90DF90CF90BF90AF909F908F907F909A
:10AE80006F905F904F903F902F90089585EB9CE0DE
:10AE90000E94C947892B69F085EB9CE00E94A74777
:10AEA000EAE0F0E0EC0FFD1FE00FF11F80830F5F81
:10AEB0001F4F65E070E080E090E00E94204D02307E
:10AEC0001105D1F59A858981981336C09B858B81B0
:10AED000981332C085EB9CE00E94C947892B31F45E
:10AEE00094E049165104610471048CF40930110591
:10AEF00089F085EB9CE00E94A747EAE0F0E0EC0FC8
:10AF0000FD1FE00FF11F80830F5F1F4FE3CF043061
:10AF100011057CF02D858C8590E0982F8827820F75
:10AF2000911D092E000CAA0BBB0B880E991EAA1EA0
:10AF3000BB1E8FEFC81AD80A9FEF491A590A690A2F
:10AF4000790A66CF2F923F924F925F927F928F92B3
:10AF50009F92AF92BF92CF92DF92EF92FF920F93A8
:10AF60001F93CF93DF9300D01F92CDB7DEB76C0154
:10AF70008EEE94E09C838B83E3E1F2E0FA83E98335
:10AF800003E410E1EE24E394F12C9DE3292E312C0F
:10AF90002EE3422E512C30E1A32EB12C41E1842E20
:10AFA000912C57E1752E80911102909112028E150D
:10AFB0009F050CF4ECC0F1E0CF16D10431F4F80198
:10AFC00080819181E981FA8109C0F2E0CF16D10434
:10AFD00039F4E981FA8180819181F801918380833C
:10AFE000E981FA8180819181009749F4EB81FC81AC
:10AFF0008281938190937D0480937C0428C081306A
:10B00000910549F4EB81FC818281938190937B04CB
:10B0100080937A041CC08230910549F4EB81FC8155
:10B0200082819381909379048093780410C0039770
:10B0300071F4EB81FC8182819381909377048093FA
:10B04000760469EC79E083E39FE00E945F46E98142
:10B05000FA8181919191FA83E9838430910549F4D1
:10B06000EB81FC8122813381309375042093740439
:10B0700030C08530910549F4EB81FC812281338118
:10B08000309373042093720424C08630910549F4F0
:10B09000EB81FC81228133813093C5042093C40469
:10B0A00024C08730910549F4EB81FC8122813381F2
:10B0B000309371042093700424C08A30910549F4C0
:10B0C000EB81FC812281338130936F0420936E04E5
:10B0D0003AC08531910549F4EB81FC8122813381AD
:10B0E00030936D0420936C042EC08631910549F491
:10B0F000EB81FC812281338130936B0420936A04BD
:10B1000022C087319105F9F4EB81FC8122813381E2
:10B11000A901475051094230510540F4B0928304CF
:10B12000A09282049092810480928004255031097B
:10B130002230310540F430928304209282045092F0
:10B140008104409280049C012B5031092A30310542
:10B1500098F4EB81FC812281338130937704209332
:10B160007604789EB001799E700D1124675A7D4F48
:10B1700083E39FE00E945F46FFEFEF1AFF0A8B8197
:10B180009C8102969C838B830E5F1F4F0CCF0F9088
:10B190000F900F900F90DF91CF911F910F91FF9023
:10B1A000EF90DF90CF90BF90AF909F908F907F9067
:10B1B0005F904F903F902F900895FF920F931F93B1
:10B1C000CF93DF93F82E0AE010E0C0E0D0E08F2D9F
:10B1D0000E94D64CC80FD91F65E070E080E090E077
:10B1E0000E94204D0150110991F7CE016AE070E0F4
:10B1F0000E946B89CB01DF91CF911F910F91FF903E
:10B2000008952F923F924F925F926F927F928F920A
:10B210009F92AF92BF92CF92DF92EF92FF920F93E5
:10B220001F93CF93DF93CDB7DEB763970FB6F89434
:10B23000DEBF0FBECDBF8B8B60E00E94974C80912C
:10B24000770B882329F082E090E0A0E0B0E004C012
:10B250008FE090E0A0E0B0E08F87988BA98BBA8B4D
:10B260006AEC79E089ED9EE00E945F4669ED7EE040
:10B27000CE0101960E944B474AE050E06FEF7FEF0E
:10B28000CE0101960E94EC75CE0101960E9489467E
:10B29000C12CD12C7601312C1D861E86212C02E377
:10B2A00010E0412C512C32018B890E94D64C092E82
:10B2B000000CAA0BBB0B480E591E6A1E7B1E65E0D4
:10B2C00070E080E090E00E94204D0150110961F78C
:10B2D0008090230290902402A0902502B090260234
:10B2E000C301B2010E94B48420E030E040EA50E49F
:10B2F0000E94138520E030E040E85AE30E94138565
:10B3000020E030E048E452E40E940487A501940163
:10B310000E943D8620E030E040E751E40E94138522
:10B320002B013C01A50194016AE979E989E390E4E4
:10B330000E943D869B01AC01C301B2010E940487BB
:10B3400020E030E0A9010E943E8620E030E040E2AB
:10B3500051E40E9413855B018C01232D3D854E85B0
:10B36000522D0E94F387181624F43A2CBD860E87BE
:10B37000212E20E030E0A901B501C8010E94AE8471
:10B3800087FF04C0A12CB12C00E010E022E0A50151
:10B39000B801CE0101960E94BD46BE016F5F7F4F8E
:10B3A000CE0107960E944B4767ED79E0CE010796E4
:10B3B0000E94A545BC0183ED9EE00E947446CE012B
:10B3C00007960E948946CE0101960E94894663ED48
:10B3D0007EE0CE0101960E944B474AE050E060E0DB
:10B3E00070E0CE0101960E94BB74CE0101960E94CE
:10B3F00089460E94584D4090730B5090740B60909A
:10B40000750B7090760B930182010C591F4F2F4FD3
:10B410003F4F061717072807390708F4C6C00E94D0
:10B42000584D0E94B2844B015C01C301B2010E94DD
:10B43000B48420E030E048EC51E40E943E869B0159
:10B44000AC01C501B4010E94AE8487FDAEC06CE3BF
:10B4500070E080E090E00E94204D9FEFC91AD90A69
:10B46000E90AF90A8F859889A989BA898C159D05F9
:10B47000AE05BF050CF013CF64E670E080E090E00D
:10B480000E94204D0E94557464E670E080E090E0D8
:10B490000E94204D6CED79E083ED9EE00E945F46B6
:10B4A00063ED7EE0CE0101960E944B4744E150E0FF
:10B4B00060E070E0CE0101960E94EC75CE0101962D
:10B4C0000E94894622E0432D5D856E85722DCE0156
:10B4D00001960E94BD46BE016F5F7F4FCE01079669
:10B4E0000E944B4767ED79E0CE0107960E94A54583
:10B4F000BC0183ED9EE00E947446CE0107960E9437
:10B500008946CE0101960E94894663ED7EE0CE0118
:10B5100001960E944B4742E350E06FEF7FEFCE0170
:10B5200001960E94BB74CE0101960E9489460E943A
:10B53000AD7462E370E080E090E00E94204D64EE24
:10B5400079E0CE0101960E943A4A63ED7EE0CE0199
:10B5500001960E94BC4568EE79E00E94A54569ED20
:10B560007EE00E94BC45BC0189ED9EE00E947446CD
:10B57000CE0101960E94894663960FB6F894DEBF0D
:10B580000FBECDBFDF91CF911F910F91FF90EF9034
:10B59000DF90CF90BF90AF909F908F907F906F90F3
:10B5A0005F904F903F902F9008950E94AD744FCFC1
:10B5B0002F923F924F925F926F927F928F929F92C3
:10B5C000AF92BF92CF92DF92EF92FF920F931F93B1
:10B5D000CF93DF93CDB7DEB72B970FB6F894DEBFCE
:10B5E0000FBECDBF7C018BEB8F838AEA888781E019
:10B5F000898784E68E9D90018F9D300D11243B87B5
:10B600002A87C12CD12C212C312C812C912C540136
:10B610002E143F048CF1C501B4010E94B48420E0D3
:10B6200030E040E251E40E9404874B015C01B70125
:10B63000FF0C880B990B0E94B4849B01AC01C501DF
:10B64000B4010E9404872B960FB6F894DEBF0FBE9C
:10B65000CDBFDF91CF911F910F91FF90EF90DF90C1
:10B66000CF90BF90AF909F908F907F906F905F90A2
:10B670004F903F902F9008952A853B85C216D306A0
:10B6800054F6C6016AE070E00E947F89892B49F474
:10B6900043E050E0BE01695F7F4F85EB9CE00E9474
:10B6A000544765E070E080E090E00E94204D3FEF5D
:10B6B000C31AD30A00E010E0412C512C320185EB73
:10B6C0009CE00E94C947892B39F424E042165104BA
:10B6D000610471040CF09CCF063011050CF098CF7A
:10B6E00085EB9CE00E94C947892B69F085EB9CE0C3
:10B6F0000E94A747E1E0F0E0EC0FFD1FE00FF11F13
:10B7000080830F5F1F4F65E070E080E090E00E9453
:10B71000204D0630110501F599818F8198131CC0C9
:10B720009A818885981318C09B818985981314C0C5
:10B730002C818D8190E0A0E0B0E0BA2FA92F982F46
:10B740008827820F911DA11DB11D880E991EAA1E6A
:10B75000BB1E8FEF281A380A9FEF491A590A690A47
:10B76000790AADCFCF93DF93CDB7DEB728970FB669
:10B77000F894DEBF0FBECDBF1D8290E49E8324E10E
:10B780002F8324E5288719829A8390E19B8390E593
:10B790009C839091D20F691710F06FEF690F409161
:10B7A000D30F262F30E0FE01E20FF31F403121F4CA
:10B7B000943011F4918101C09581682F690F606800
:10B7C0008BEC9FE028960FB6F894DEBF0FBECDBF7E
:10B7D000DF91CF910C945141CF93DF93BC0182E56F
:10B7E0009DE00E94634AEC0182E59DE00E94314B9E
:10B7F0008C0F9D1FDF91CF910895CF93DF93BC01F4
:10B8000082E59DE00E94874AEC0182E59DE00E946E
:10B81000314B8C0F9D1FDF91CF910895CF93DF9314
:10B82000AB01BC012AE030E082E59DE00E94E44AE1
:10B83000EC0182E59DE00E94314B8C0F9D1FDF9152
:10B84000CF9108954F925F926F927F928F929F92C5
:10B85000AF92BF92CF92DF92EF92FF926B017C0189
:10B86000B42E9B01AC010E944389882319F06BEF31
:10B8700079E027C026013701E89477F82FEF3FEFF2
:10B880004FE75FE7C301B2010E94438981110DC0F8
:10B890002FEF3FEF4FE75FE7C301B2010E94AE8495
:10B8A00018161CF46FEF79E00CC02FEF3FEF4FE755
:10B8B0005FE4C701B6010E94F387181694F463E0B1
:10B8C0007AE082E59DE0FF90EF90DF90CF90BF900F
:10B8D000AF909F908F907F906F905F904F900C945F
:10B8E000874A2FEF3FEF4FE75FECC701B6010E9499
:10B8F000AE8487FDE4CF20E030E0A901C701B601A6
:10B900000E94AE8487FF0BC06DE282E59DE00E943D
:10B910004E4A4C01F7FAF094F7F8F09402C0812CEB
:10B92000912CA12C60E070E080E09FE3AB1441F02B
:10B9300020E030E040E251E40E940487A394F6CF77
:10B940009B01AC01C701B6010E943E862B013C0160
:10B950000E94A2876B017C010E94B2849B01AC0112
:10B96000C301B2010E943D862B013C012AE0B701D0
:10B97000A60182E59DE00E949C4A7C01E80CF91C2E
:10B98000BB2039F06EE282E59DE00E944E4AE80E4F
:10B99000F91EDB2CDD2031F120E030E040E251E403
:10B9A000C301B2010E9413852B013C010E94A287B2
:10B9B0004B01A12CB12C2AE0B501A40182E59DE048
:10B9C0000E949C4AE80EF91EC501B4010E94B2848F
:10B9D0009B01AC01C301B2010E943D862B013C01D9
:10B9E000DA94D8CFC701FF90EF90DF90CF90BF904F
:10B9F000AF909F908F907F906F905F904F90089541
:10BA000021CF2091170C9091E40F213208F04AC009
:10BA10008091F40B8111FCCF32E03093F40B31E0D4
:10BA20003093F30B3FEF3093F20B1092F10B209316
:10BA3000F00BA7EFBBE040ED5BE0FA013E2F341BBB
:10BA4000321718F43D913193F9CF1092CF0B20911A
:10BA5000CF0B990F922B9093CF0B9091CE0B9130EF
:10BA600061F41092CE0B9091CF0B9093BB0090910C
:10BA7000BC0093FDF8CF95EC01C095EE9093BC000F
:10BA80009091F40B9230E1F39091F20B9F3F79F09B
:10BA90008091F20B803241F08091F20B803331F0D3
:10BAA00084E005C081E003C082E001C083E0109221
:10BAB000F60B1092170C1092F50B089591E09093ED
:10BAC000F50B8093E40F1092F60B1092170C08956B
:10BAD0001092CD0B1092CC0B1092F60B1092170C0B
:10BAE0001092F40B81E08093F30B1092CE0B61E087
:10BAF00084E10E94654C61E085E10E94654CE9EBC0
:10BB0000F0E080818E7F808380818D7F808388E4D8
:10BB10008093B80085E48093BC0008952F923F92F3
:10BB20004F925F926F927F928F929F92AF92BF924D
:10BB3000CF92DF92EF92FF920F931F93CF93DF93F9
:10BB4000CDB7DEB728970FB6F894DEBF0FBECDBFD6
:10BB500040917C0B50917D0BC0907E0BD0907F0B61
:10BB60004C155D052CF03C2D2D2D6A01432F522FD5
:10BB7000E0E8FBE060E070E0CB0101911191041777
:10BB8000150754F44A01550FAA08BB08680D791D22
:10BB90008A1D9B1DA80115C0C016D10654F40D2C9A
:10BBA000000CEE08FF086C0D7D1D8E1D9F1D6801A9
:10BBB00008C0012E000C220B330B600F711F821F77
:10BBC000931F2BE0EC3CF207C1F60E94B48420E006
:10BBD00030E048E152E40E9404876B017C010CE7ED
:10BBE0001BE0812C912C5401D8016D917D918D0128
:10BBF000072E000C880B990B0E94B484A7019601B4
:10BC00000E943D869B01AC010E9413859B01AC0103
:10BC1000C501B4010E943E864B015C01BBE00C3CB7
:10BC20001B0711F720E030E04CE152E40E9404874A
:10BC30000E9402894B015C0120E030E040E85FE3B4
:10BC40000E94F38718160CF06EC00CE71BE0212C45
:10BC5000312C19821A821B821C82F80181919191E8
:10BC60008F019C01990F440B550B2D833E834F830D
:10BC70005887CA01B9010E94B484A70196010E94A5
:10BC80003D862B013C0120E030E0A9010E94F387B2
:10BC9000181624F077FA709477F87094A50194013F
:10BCA000C301B2010E94AE8487FF13C089819A81CB
:10BCB000AB81BC812D813E814F815885820F931FBE
:10BCC000A41FB51F89839A83AB83BC833FEF231ADC
:10BCD000330A4BE00C3C140709F0BFCF20E030E002
:10BCE00040EC5FE3C501B4010E9413854B015C0188
:10BCF00055E0251631040CF4A8CF69817A818B8137
:10BD00009C810E94B4846B017C01B101330C880BCF
:10BD1000990B0E94B4849B01AC01C701B6010E943B
:10BD200004876B017C01C701B60128960FB6F89411
:10BD3000DEBF0FBECDBFDF91CF911F910F91FF905E
:10BD4000EF90DF90CF90BF90AF909F908F907F90BB
:10BD50006F905F904F903F902F9008954F925F9219
:10BD60006F927F928F929F92AF92BF92CF92DF920B
:10BD7000EF92FF920F931F93CF93DF9300D01F9208
:10BD8000CDB7DEB76B017C0111E0A12EB12C4501CE
:10BD9000880C991C880C991CF401E456FB4F4080D8
:10BDA000518062807380A3019201C701B6010E9495
:10BDB000F387181614F41F5FE8CFA3019201C7019F
:10BDC000B6010E94AE8484010C571B4F811106C03E
:10BDD000D8016D917D918D919C9142C0C50181509A
:10BDE000904C880F991F880F991FFC01E456FB4F58
:10BDF000208131814281538129833A834B835C8343
:10BE0000FC01EC57FB4F80809180A280B380C7017A
:10BE1000B6010E943D866B017C01A5019401D80109
:10BE20006D917D918D919C910E943D869B01AC010D
:10BE3000C701B6010E9413856B017C0129813A81FB
:10BE40004B815C81C301B2010E943D869B01AC0124
:10BE5000C701B6010E940487A50194010E943E8695
:10BE60000F900F900F900F90DF91CF911F910F9136
:10BE7000FF90EF90DF90CF90BF90AF909F908F900A
:10BE80007F906F905F904F900895DF92EF92FF92B6
:10BE90000F931F93CF93DF937C018B01EA01461729
:10BEA000570720F4812F8A01C62FD82F69EC79E03B
:10BEB000C7010E943A4A8091EF0E9091F00E081748
:10BEC0001907E0F48C179D0708F4EC01E091EB0EE4
:10BED000F091EC0EEC0FFD1FD08010826091EB0E04
:10BEE0007091EC0E600F711FC7010E945F46E091D8
:10BEF000EB0EF091EC0EEC0FFD1FD082C701DF912D
:10BF0000CF911F910F91FF90EF90DF900895CF9305
:10BF1000DF93EC014091EF0E5091F00EB6DFCE01B1
:10BF2000DF91CF9108950F931F930E94584D609316
:10BF3000BD0C7093BE0C8093BF0C9093C00CE0912D
:10BF4000B50CF091B60C0284F385E02D85EB9CE0F6
:10BF5000199597FF1FC00E94584D0091BD0C10917C
:10BF6000BE0C2091BF0C3091C00CDC01CB01801BBA
:10BF7000910BA20BB30B0091B90C1091BA0C20914C
:10BF8000BB0C3091BC0C80179107A207B307B8F225
:10BF90008FEF9FEF1F910F910895682F8FEE9DE017
:10BFA0000C942455CF93DF931F92CDB7DEB76091E9
:10BFB0007F108EED93E069830E94CA8569816817BE
:10BFC00021F08EED93E00E94D285609180108FED7C
:10BFD00093E069830E94CA856981681721F08FED1B
:10BFE00093E00E94D2858FE790E10F90DF91CF918F
:10BFF0000895CF92DF92EF92FF920F931F93CF930A
:10C00000DF931F92CDB7DEB76C0109E010E17C0130
:10C0100086E7E80EF11CF80161918F01C601698382
:10C020000E94CA856981681719F0C6010E94D285ED
:10C03000FFEFCF1ADF0ACE14DF0469F789E090E141
:10C040000F90DF91CF911F910F91FF90EF90DF90B4
:10C05000CF9008959091F40B9111FCCF613208F0CC
:10C0600060E291E09093F40B9093F30B2FEF209309
:10C07000F20B1092F10B260F2093F00B9093CF0B45
:10C080009091CF0B880F892B8093CF0B8091CE0B93
:10C09000813061F41092CE0B8091CF0B8093BB0066
:10C0A0008091BC0083FDF8CF85EC01C085EE8093C4
:10C0B000BC008091F40B8130E1F38091F10B861785
:10C0C00010F46091F10BA0EDBBE029EE3FE0F90127
:10C0D0008E2F821B861718F48D918193F9CF1092C1
:10C0E000CD0B6093CC0B862F08951F93CF93DF93D6
:10C0F0001F92CDB7DEB7682F87E76983DFDC6981E0
:10C100008FEE9DE00E9424557CDC87E7D7DC61E060
:10C1100087E7A0DF8FEE9DE00E94D454182F71DCDA
:10C12000812F0F90DF91CF911F9108950F931F934F
:10C13000CF93DF931F92CDB7DEB7682F87E7698370
:10C14000BDDC69818FEE9DE00E9424555ADC87E7B3
:10C15000B5DC62E087E77EDF8FEE9DE00E94D4547D
:10C1600000E010E0182F8FEE9DE00E94D454082BC1
:10C17000192B47DCC8010F90DF91CF911F910F91D0
:10C18000089587E79BDC64EF8FEE9DE00E942455C5
:10C190006EE28FEE9DE00E94245533DC65E070E096
:10C1A00080E090E00E94204D86EFC0CF3F924F92FA
:10C1B0005F926F927F928F929F92AF92BF92CF9237
:10C1C000DF92EF92FF920F931F93CF93DF93CDB740
:10C1D000DEB728970FB6F894DEBF0FBECDBFD1DF14
:10C1E0006C01E12CF12C1091F10E1295110F110F31
:10C1F000107C1C5C87E762DC64EF8FEE9DE00E94A0
:10C200002455612F8FEE9DE00E942455FADB80912A
:10C21000F10E811105C065E070E080E090E012C091
:10C22000813029F468E070E080E090E00BC082305B
:10C2300029F46EE070E080E090E004C06AE170E014
:10C2400080E090E00E94204D86EF70DF4C01A12C31
:10C25000B12CBA2CA92C982C882488EF46DF882A88
:10C260003090F10E8091060F9091070FA701960173
:10C27000281B390B41095109A091040FB091050FFA
:10C280000E94FC856B017C01AFE0F594E794D794A4
:10C29000C794AA95D1F76091FE0E7091FF0ECB0165
:10C2A000770FAA0BBB0BBC01CD01BBE0660F771F5C
:10C2B000881F991FBA95D1F72091000F3091010F77
:10C2C0008901330F220B330BA90198012C0D3D1D61
:10C2D0004E1D5F1D0E94E085C20ED31EE41EF51E9A
:10C2E00020EAC21A2FE0D20AE108F108A70196015C
:10C2F000C701B6010E945C899B01AC011CE0559509
:10C300004795379527951A95D1F729833A834B831B
:10C310005C830091F20E1091F30EA091F60EB09195
:10C32000F70EA70196010E9406862B013C018DE0C5
:10C3300075946794579447948A95D1F7A091F80E15
:10C34000B091F90E29813A814B815C810E94068669
:10C35000BB2797FDB095AB2F840D951DA61DB71D6E
:10C360000296A11DB11D32E0B595A79597958795C9
:10C370003A95D1F79C01AD0130584F4F5F4FA091D6
:10C38000020FB091030F0E94FC852B013C014FE08E
:10C3900076946794579447944A95D1F788E090E053
:10C3A00083199109A501940104C0569547953795C5
:10C3B00027958A95D2F72D833E834F83588748016E
:10C3C000110FAA08BB0852E0880C991CAA1CBB1CC0
:10C3D0005A95D1F7A091FA0EB091FB0E29813A81BE
:10C3E0004B815C810E9406869B01AC016BE05595F8
:10C3F0004795379527956A95D1F729833A834B83DB
:10C400005C83A091F40EB091F50EA70196010E94F5
:10C410000686DC01CB017BE0B595A79597958795BE
:10C420007A95D1F729813A814B815C81820F931FE4
:10C43000A41FB51F880D991DAA1DBB1D032C04C088
:10C44000880F991FAA1FBB1F0A94D2F7BC01CD0108
:10C450006E5F7F4F8F4F9F4F24E030E040E050E011
:10C460000E94E0858D819E81AF81B885821B930BF0
:10C47000A40BB50B9C01AD0180E593ECA0E0B0E00E
:10C48000BC01CD0104C096958795779567953A9440
:10C49000D2F70E945C8997FD0BC0660F771F881F3B
:10C4A000991FA30192010E940C8669017A010AC0BA
:10C4B000A30192010E940C8669017A01CC0CDD1C5B
:10C4C000EE1CFF1C9927F7FC9A958F2D7E2D6D2D64
:10C4D0009B01AC010E945C899B01AC01AEEDBBE00D
:10C4E0000E94FC854C01BB2497FCB094AB2CA3E4C8
:10C4F000B3EEA70196010E940886BB2797FDB09571
:10C50000AB2F880D991DAA1DBB1D8153914FAF4FB5
:10C51000BF4F44E0B595A795979587954A95D1F774
:10C52000BC01CD016C0D7D1D8E1D9F1D28960FB683
:10C53000F894DEBF0FBECDBFDF91CF911F910F9159
:10C54000FF90EF90DF90CF90BF90AF909F908F9033
:10C550007F906F905F904F903F900895CF92DF92C1
:10C56000EF92FF920F931F930CDEAC0160E070E03E
:10C57000E1EFFEE0858996899A01AB01281B390B12
:10C5800041095109A389B4890E94FC856B017C0192
:10C590008FE0F594E794D794C7948A95D1F7658591
:10C5A0007685CB01770FAA0BBB0BBC01CD012BE02D
:10C5B000660F771F881F991F2A95D1F72785308925
:10C5C0008901330F220B330BA90198012C0D3D1D5E
:10C5D0004E1D5F1D0E94E085D701C601820F931F8B
:10C5E000A41FB51F0896A11DB11DBC01CD0134E0EB
:10C5F00095958795779567953A95D1F70E94B4847C
:10C6000020E030E040E251E40E9404871F910F9146
:10C61000FF90EF90DF90CF9008954F925F926F92CE
:10C620007F928F929F92AF92BF92DF92EF92FF9292
:10C630000F931F93CF93DF9300D01F921F92CDB71C
:10C64000DEB7182F19821A821B821C821D8261E0BC
:10C650000E94974C60E0812F0E94654C62E170E07F
:10C6600080E090E00E94204D61E0812F0E94654CA7
:10C670008BE990E00197F1F760E0812F0E94974CE1
:10C6800051E1E52E57E2F52E812F0E943B4C892B7C
:10C6900039F481E0E81AF108B9F78EEF9FEF75C021
:10C6A00041E1E42E47E2F42E812F0E943B4C01979A
:10C6B00029F481E0E81AF108B9F7EFCF28E2E22E79
:10C6C000F12C07E0D12CAA24A394B12C91E1892E5E
:10C6D00097E2992E812F0E943B4C892B29F481E00F
:10C6E000881A9108B9F7D9CF0E94FB4C2B013C0165
:10C6F00081E1882E87E2982E812F0E943B4C019782
:10C7000029F481E0881A9108B9F7C7CF0E94FB4C41
:10C71000DC01CB0184199509A609B7098997A10500
:10C72000B10578F0E1E0F0E0EC0FFD1FED0DF11D3B
:10C730002081C501002E01C0880F0A94EAF7822BE0
:10C740008083011103C0D39407E001C0015081E050
:10C75000E81AF10809F0BACF8981282F30E0309328
:10C76000E60F2093E50F2B81422F50E05093E80F06
:10C770004093E70F280F81E090E03D81321302C023
:10C7800080E090E09195819591090F900F900F9026
:10C790000F900F90DF91CF911F910F91FF90EF902D
:10C7A000DF90BF90AF909F908F907F906F905F9041
:10C7B0004F900895EF92FF920F931F93CF93DF93C3
:10C7C000C82F8B017A0183E579D96C2F8FEE9DE01C
:10C7D0000E94245516D983E571D9602F83E53ADC90
:10C7E000E701CE018E199F093091CC0B2091CD0B22
:10C7F000321731F08FEE9DE00E94D4548993F1CF2F
:10C800008017910729F01092390F81E080933A0F39
:10C81000DF91CF911F910F91FF90EF90F2C8CF93CE
:10C82000DF93AC01990F660B770B2AE030E082E5CD
:10C830009DE00E94E44AEC0182E59DE00E94314BBC
:10C840008C0F9D1FDF91CF9108951F93CF93DF939E
:10C850001F92CDB7DEB7162FAE014F5F5F4F61E07D
:10C8600070E0A8DF898190E002C0959587951A95C0
:10C87000E2F781700F90DF91CF911F910895CF93D0
:10C88000DF93D82FC62F83E519D96D2F8FEE9DE04A
:10C890000E9424556C2F8FEE9DE00E942455DF915D
:10C8A000CF91AFC8FF920F931F93CF93DF931F9247
:10C8B000CDB7DEB7182F062FF42EAE014F5F5F4FB6
:10C8C00061E070E077DF8981FF2049F041E050E0CE
:10C8D00001C0440F0A95EAF7482B498309C021E0BB
:10C8E00030E001C0220F0A95EAF72095282329831A
:10C8F0006981812FC4DF0F90DF91CF911F910F913C
:10C90000FF900895CF93DF9342E00E94225CEC01F8
:10C9100082E59DE00E94314B8C0F9D1FDF91CF91EE
:10C920000895AF92BF92CF92DF92EF92FF921F9342
:10C93000CF93DF93CDB7DEB72A970FB6F894DEBF5B
:10C940000FBECDBF182F47E45FE066E070E082E3E2
:10C950009F8330DF2091480F30E0322F22278091D3
:10C96000470F282B3A83298320914A0F30E0322F3A
:10C9700022278091490F282B3C832B8320914C0F39
:10C9800030E0322F222780914B0F282B3E832D83BE
:10C990009E012F5F3F4F59015BE3C52E5FE0D52E0F
:10C9A000E12E9F81F92EF501619171915F01F601F0
:10C9B00021913191419151916F01072E000C880B0B
:10C9C000990B2F83388749875A870E94B4842F8117
:10C9D000388549855A850E941385F70161937193C3
:10C9E000819391937F01F7E4CF16FFE0DF06D9F63C
:10C9F0002A960FB6F894DEBF0FBECDBFDF91CF9160
:10CA00001F91FF90EF90DF90CF90BF90AF9008956F
:10CA1000CF92DF92EF92FF92CF93DF93CDB7DEB745
:10CA20002C970FB6F894DEBF0FBECDBF6CE57DE04E
:10CA3000CE0101960E9443474CE251E06FEF7FEF39
:10CA4000CE0101960E94BB74CE0101960E948946D8
:10CA500080917A0490917B04E0DDE12CF12C64E676
:10CA600070E080E090E00E94204D80917A049091E7
:10CA70007B04D3DD2FEFE21AF20A23E0E216F10481
:10CA800074F32AE0E216F1041CF4892B41F703C089
:10CA9000892B09F04FC16091E70F7091E80F072EC5
:10CAA000000C880B990B0E94B4846B017C0160938D
:10CAB00085107093861080938710909388108091D2
:10CAC000E50F9091E60FBC01990F880B990B0E941E
:10CAD000B48460938110709382108093831090933C
:10CAE000841021E0B701A601CE0107960E94BD4641
:10CAF0006DE678E0CE0101960E943A4ABE01695F78
:10CB00007F4FCE0101960E94BC45BC0189ED9EE09D
:10CB10000E947446CE0101960E948946CE01079676
:10CB20000E9489464091811050918210609183103B
:10CB30007091841021E0CE0107960E94BD4663E00B
:10CB400079E0CE0101960E943A4ABE01695F7F4FAB
:10CB5000CE0101960E94BC45BC0189ED9EE00E9479
:10CB6000DB45CE0101960E948946CE0107960E94C0
:10CB7000894660E978E089ED9EE00E94CD4569EC48
:10CB800079E0CE0101960E943A4A44E150E060E02B
:10CB900070E0CE0101960E94EC75CE0101960E94D4
:10CBA00089466091851070918610809187109091D0
:10CBB00088100E949D874AE0CE0101960E94184786
:10CBC000BE016F5F7F4F83ED9EE00E940746CE015E
:10CBD00001960E94894660E086E00E94B25B63EDA8
:10CBE0007EE08BEC9FE00E94554A6FED8BEC9FE05E
:10CBF0000E944E4A69E079E08BEC9FE00E94444B32
:10CC000060918110709182108091831090918410B6
:10CC10000E949D874AE050E08BEC9FE00E942B4BE6
:10CC200060E978E08BEC9FE00E94444B64E670E0A2
:10CC300080E090E00E94204DC0908510D09086103A
:10CC4000E0908710F090881020E030E040EF51E451
:10CC5000C701B6010E94F38787FD03C06DE47DE044
:10CC600054C020E030E040ED51E4C701B6010E941D
:10CC7000F38787FD1FC06DE37DE0CE0101960E9422
:10CC800043474AE050E06FEF7FEFCE0101960E94EC
:10CC9000BB74CE0101960E94894680914702882389
:10CCA00031F06CED75E080E090E00E94204D6DE287
:10CCB0007DE02BC020E030E040EB51E4C701B6013D
:10CCC0000E94F38787FD03C06FE17DE01EC060E135
:10CCD0007DE0CE0101960E9443474AE050E06FEFAD
:10CCE0007FEFCE0101960E94BB74CE0101960E9497
:10CCF000894680914702882331F06CED75E080E031
:10CD000090E00E94204D62E07DE0CE0101960E94FD
:10CD100043474AE050E06FEF7FEFCE0101960E945B
:10CD2000BB74CE0101960E94894662E370E080E008
:10CD300090E0CAC00E9455746EE170E080E090E01F
:10CD40000E94204D0BDC6B017C0164E670E080E00A
:10CD500090E00E94204D6DE678E089ED9EE00E9413
:10CD60005F4621E0B701A601CE0101960E94BD46B3
:10CD7000BE016F5F7F4F89ED9EE00E94DB45CE01D3
:10CD800001960E94894669ED7EE0CE0101960E94DF
:10CD90004B474AE050E060E070E0CE0101960E940F
:10CDA000EC75CE0101960E9489460E94997468E54F
:10CDB00079E089ED9EE00E94CD45C0928510D09229
:10CDC0008610E0928710F092881020E030E040EF6B
:10CDD00051E4C701B6010E94F38787FD03C062EFEB
:10CDE0007CE054C020E030E040ED51E4C701B601E2
:10CDF0000E94F38787FD1FC062EE7CE0CE010196A2
:10CE00000E9443474AE050E06FEF7FEFCE0101966A
:10CE10000E94BB74CE0101960E9489468091470210
:10CE2000882331F06CED75E080E090E00E94204DA9
:10CE300062ED7CE02BC020E030E040EB51E4C70124
:10CE4000B6010E94F38787FD03C064EC7CE01EC03E
:10CE500065EB7CE0CE0101960E9443474AE050E03A
:10CE60006FEF7FEFCE0101960E94BB74CE01019659
:10CE70000E94894680914702882331F06CED75E06D
:10CE800080E090E00E94204D67EA7CE0CE010196B0
:10CE90000E9443474AE050E06FEF7FEFCE010196DA
:10CEA0000E94BB74CE0101960E9489466CE271E03B
:10CEB00080E090E00E94204D80914702882331F06D
:10CEC00068EE73E080E090E00E94204D2C960FB653
:10CED000F894DEBF0FBECDBFDF91CF91FF90EF90F2
:10CEE000DF90CF900895CF93DF93FC0124813581AB
:10CEF000232B69F0EC01BC0182E59DE00E94344BDC
:10CF0000BE0188E19CE0DF91CF910C94344BDF911E
:10CF1000CF9108950F931F93CF93DF93CDB7DEB7D3
:10CF20002C970FB6F894DEBF0FBECDBF0E94DD5820
:10CF30008C0190938A108093891062E370E080E006
:10CF400090E00E94204D4AE0B801CE0101960E9477
:10CF50001847BE016F5F7F4F89ED9EE00E94074634
:10CF6000CE0101960E9489468091370F9091380F2B
:10CF7000892B09F45BC063E37FE0CE0101960E9438
:10CF80004B47BE016F5F7F4FCE0107960E944B4714
:10CF900044E150E060E070E0CE0107960E94EC753D
:10CFA000CE0107960E94894667E07AE0CE01079697
:10CFB0000E943A4A69ED7EE0CE0107960E94BC4588
:10CFC000BC0183ED9EE00E947446CE0107960E944C
:10CFD000894663ED7EE0CE0107960E944B4744E10F
:10CFE00050E06FEF7FEFCE0107960E94BB74CE0139
:10CFF00007960E948946BE016F5F7F4FCE0107965C
:10D000000E944B476BE679E0CE0107960E94A5454A
:10D0100063ED7EE00E94BC45BC0189ED9EE00E946C
:10D020007446CE0107960E94894650C062E17AE0BC
:10D0300083ED9EE00E945F4663ED7EE0CE010196A7
:10D040000E944B4744E150E060E070E0CE01019661
:10D050000E94EC75CE0101960E94894662E179E05A
:10D06000CE0101960E943A4A69ED7EE0CE0101961A
:10D070000E94BC45BC0183ED9EE00E947446CE0137
:10D0800001960E94894663ED7EE0CE0101960E94E2
:10D090004B4744E150E06FEF7FEFCE0101960E94D5
:10D0A000BB74CE0101960E94894667E07AE0CE010A
:10D0B00001960E943A4A69ED7EE0CE0101960E94F7
:10D0C000BC45BC0189ED9EE00E947446CE010196EC
:10D0D0000E9489468091770B882331F060E273E0EB
:10D0E00080E090E00E94204D2C960FB6F894DEBFB1
:10D0F0000FBECDBFDF91CF911F910F910895CF92B9
:10D10000DF92EF92FF920F931F93CF93DF93CDB7F0
:10D11000DEB728970FB6F894DEBF0FBECDBF8234BE
:10D1200009F474C0D4F4803309F490C07CF48332E1
:10D1300009F483C08A3209F0A7C06DE775E08BEE71
:10D140009EE00E945F468FEF9FEF09C1813309F493
:10D150008CC0813409F44FC097C0813609F44BC0AC
:10D1600034F4833409F45DC0843449F08DC08336CF
:10D1700009F457C00CF44AC0843609F085C0809188
:10D18000E90E9091EA0E892B09F4ECC085EE9EE041
:10D190000E940E4597FDE6C061EA7CE082E59DE0D5
:10D1A0000E94634A65EE7EE082E59DE00E94344B7A
:10D1B00085EE9EE00E940E450AEF1FEF2FEF3FEF36
:10D1C00068017901C61AD70AE80AF90AB701A60167
:10D1D0002AE0CE0101960E94EC46BE016F5F7F4FB0
:10D1E00085EE9EE00E940746CE0101960E94894688
:10D1F00085EE9EE0B1C064E775E08BEE9EE00E9494
:10D200005F4680913C0B90913D0BA9C061E775E0B2
:10D210008BEE9EE00E945F461092770B8CEF9FEFA3
:10D220009EC067E775E08BEE9EE00E945F4681E05E
:10D230008093770B8DEF9FEF92C06AE775E08BEEDE
:10D240009EE00E945F468EEF9FEF89C06BE675E01F
:10D2500085EE9EE00E945F466BE675E08BEE9EE0F9
:10D260000E945F4680E090E07AC06EE775E085EE50
:10D270009EE00E945F466EE775E08BEE9EE00E94A6
:10D280005F4681E090E06BC01A8219821C821B828B
:10D290001E821D828F831886BE01695F7F4FCE017B
:10D2A00001960E945F46BE016F5F7F4F85EE9EE054
:10D2B0000E940746CE0101960E94894685EE9EE0B7
:10D2C0000E940E45CB010E94591D64E670E080E08B
:10D2D00090E00E94204D4CC08FEFE81AF80A89EECA
:10D2E000E81683E0F80659F06EE170E080E090E027
:10D2F0000E94204D0E941053182F112369F36AE2F7
:10D3000070E0611B710917FD73954AE0CE0101962B
:10D310000E941847BE016F5F7F4F8BEE9EE00E9418
:10D320000746CE0101960E9489466BEE7EE085EEAF
:10D330009EE00E9474466BE97CE082E59DE00E94DD
:10D34000634A612F82E59DE00E944E4A82E59DE09E
:10D350000E94314B8BEE9EE00E940E45CB010E9455
:10D36000591D06C00E941053182FE12CF12CC5CF77
:10D3700028960FB6F894DEBF0FBECDBFDF91CF91D8
:10D380001F910F91FF90EF90DF90CF9008951F9322
:10D39000CF93DF93182FCCE7DBE0812F0E94D64C90
:10D3A000899399936CE370E080E090E00E94204DB7
:10D3B0008BE0CC3CD80789F70E948E5D20E030E0FE
:10D3C00040EA50E40E94138520E030E040E85AE350
:10D3D0000E941385DF91CF911F9108954F925F9224
:10D3E0006F927F928F929F92AF92BF92CF92DF9275
:10D3F000EF92FF92CF93DF93CDB7DEB760970FB672
:10D40000F894DEBF0FBECDBF8091770B882331F03B
:10D4100032E0432E512C612C712C05C02EE1422E9E
:10D42000512C612C712C62E77DE089ED9EE00E9419
:10D43000E14569ED7EE0CE0101960E944B474AE04E
:10D4400050E06FEF7FEFCE0101960E94BB74CE01DA
:10D4500001960E948946812C912C5401C12CD12C1B
:10D46000760183E20E945E5D87E090E00E94CD5FDE
:10D470000E94015D66E970E080E090E00E94204D2E
:10D4800083E20E945E5D80E290E00E94CD5F0E9498
:10D49000015D66E970E080E090E00E94204D62E06E
:10D4A00083E20E942A6040E050E0BA018091CC0BF8
:10D4B00090E02091CD0B821B910918161906ACF44F
:10D4C0008FEE9DE04D875E876F87788B0E94D454E6
:10D4D0004D855E856F857889762F652F542F44277B
:10D4E000480F511D611D711DE1CFCB01BA010E9492
:10D4F000B4842AE939E949E95FE30E9404870E947C
:10D500009D87AB01BC01C416D506E606F70614F4E8
:10D510006A017B012AE0CE0101960E94EC46BE0121
:10D520006F5F7F4FCE0107960E944B4766E17AE01E
:10D53000CE0107960E94A545BC0183ED9EE00E94A6
:10D540007446CE0107960E948946CE0101960E943C
:10D55000894663ED7EE0CE0101960E944B474EE185
:10D5600050E060E070E0CE0101960E943A75CE0175
:10D5700001960E9489468FEF881A980AA80AB80A6D
:10D58000481459046A047B040CF06BCF2AE0B701FD
:10D59000A601CE0101960E94EC46BE016F5F7F4F4F
:10D5A000CE0107960E944B4766E17AE0CE010796CE
:10D5B0000E94A545BC0183ED9EE00E947446CE0109
:10D5C00007960E948946CE0101960E94894663ED26
:10D5D0007EE0CE0101960E944B474AE050E060E0B9
:10D5E00070E0CE0101960E94EC75CE0101960E947A
:10D5F00089462AE0B701A601CE0107960E94EC46B3
:10D600006AE17AE0CE0101960E943A4ABE01695F62
:10D610007F4FCE0101960E94BC456DE17AE00E94E9
:10D62000A54569ED7EE00E94BC45BC0189ED9EE008
:10D630000E947446CE0101960E948946CE0107964B
:10D640000E94894662E370E080E090E00E94204DF5
:10D6500060960FB6F894DEBF0FBECDBFDF91CF91BD
:10D66000FF90EF90DF90CF90BF90AF909F908F9002
:10D670007F906F905F904F9008952F923F924F92BE
:10D680005F926F927F928F929F92AF92BF92CF9252
:10D69000DF92EF92FF920F931F93CF93DF93CDB75B
:10D6A000DEB7C954D1090FB6F894DEBF0FBECDBFA7
:10D6B0002B013C0127962FAF279728963FAF28973D
:10D6C00029964FAF29972A965FAF2A970E94584D07
:10D6D00022966CAF7DAF8EAF9FAF229727962FAD6E
:10D6E000279728963FAD289729964FAD29972A96D8
:10D6F0005FAD2A9780E9481681E0580661047104FD
:10D7000034F060E9462E55245394612C712C20315D
:10D7100097E23907410551052CF42DA73EA74FA7E5
:10D7200058AB0AC090E1C92E97E2D92EE12CF12C1A
:10D73000CDA6DEA6EFA6F8AA8091770B882321F06C
:10D740002DA73EA74FA758AB22966CAD7DAD8EADF1
:10D750009FAD229728EE33E040E050E00E94E08544
:10D7600026962CAF3DAF4EAF5FAF269721E02DAB95
:10D7700019A61AA61BA61CA68E01035F1F4FCC2458
:10D78000DD247601C418D508E608F708C9AADAAA84
:10D79000EBAAFCAAC9A4DAA4EBA4FCA42DA53EA57F
:10D7A0004FA558A9C216D306E406F5060CF029C306
:10D7B00069A57AA58BA59CA50E94B48420E030E0E1
:10D7C0004AE754E40E940487AB01BC0123E0C8018E
:10D7D0000E94BD46B80183ED9EE00E940746C80145
:10D7E0000E9489462DA53EA54FA558A92A3031058E
:10D7F0004105510594F42AE026964CAD5DAD6EAD21
:10D800007FAD2697C8010E94EC46B80183ED9EE0EB
:10D810000E940746C8010E948946CE01019681D820
:10D8200062E27AE089ED9EE00E945F46AE014F5FC2
:10D830005F4F1A01C12CD12C7601D1018D909D90A2
:10D84000AD90BD901D01A5019401C501B4010E94D8
:10D8500013859B01AC01C701B6010E943E866B0196
:10D860007C0123E0B501A401C8010E948E46B801E5
:10D87000CE0143960E944B476BE679E0CE0143967A
:10D880000E94A545BC0189ED9EE00E94DB45CE01CA
:10D8900043960E948946C8010E9489462016310697
:10D8A00061F6C701B6010E9402896B017C01BDE2ED
:10D8B0004B16B1E05B06610471042CF0F6D760E012
:10D8C00080E00E94B25B23E0B701A601CE0143963F
:10D8D0000E94BD466FE27AE0C8010E943A4A63EDB9
:10D8E0007EE0C8010E94BC4562E37AE00E94A54543
:10D8F000BE016D5E7F4F0E94BC4567E37AE00E94E7
:10D90000A545BC0189ED9EE00E94DB45C8010E944F
:10D910008946CE0143960E9489462DEC3CEC4CE4AE
:10D920005FE3C701B6010E94F38729813A814B81E9
:10D930005C812DA33EA34FA358A718160CF0A7C1D6
:10D940002AE939E949E95FE3C701B6010E94AE84DB
:10D9500087FF9DC1CDA8CC2009F499C189849A8400
:10D96000AB84BC8420E030E0A901C501B4010E9471
:10D97000AE84CD80DE80EF80F884882309F12DA16C
:10D980003EA14FA158A5CA01B9010E9413856EABF3
:10D990007FAB88AF99AFA7019601C701B6010E947E
:10D9A00013859B01AC016EA97FA988AD99AD0E943A
:10D9B0003E860E940289A50194010E94B18604C09E
:10D9C0006BED7FE089EC9FE320EE3EE245E652E41A
:10D9D0000E9413856EAB7FAB88AF99AF20E030E03B
:10D9E000A901C701B6010E94AE84882309F12DA1C7
:10D9F0003EA14FA158A5CA01B9010E9413856AAF83
:10DA00007BAF8CAF9DAFA5019401C501B4010E940D
:10DA100013859B01AC016AAD7BAD8CAD9DAD0E94C1
:10DA20003E860E940289A70196010E94B18604C029
:10DA30006BED7FE089EC9FE320EE3EE245E652E4A9
:10DA40000E9413856AAF7BAF8CAF9DAF20E030E0C2
:10DA5000A9016DA17EA18FA198A50E94AE84882303
:10DA6000F9F0A5019401C501B4010E9413854B0191
:10DA70005C01A7019601C701B6010E9413859B01B5
:10DA8000AC01C501B4010E943E860E9402892DA10D
:10DA90003EA14FA158A50E94B1866B017C0108C030
:10DAA0008BEDC82E8FE0D82E89ECE82E8FE3F82E70
:10DAB00060E37AE0C8010E943A4A63ED7EE0C80163
:10DAC0000E94BC456AE37AE00E94A545BC0189ED4D
:10DAD0009EE00E947446C8010E94894660E37AE095
:10DAE000C8010E943A4A63ED7EE0C8010E94BC452D
:10DAF00064E57AE00E94A545BC0183ED9EE00E94AA
:10DB00007446C8010E94894621E04EA95FA968AD0C
:10DB100079ADCE014F960E94BD4621E04AAD5BAD86
:10DB20006CAD7DADCE0149960E94BD4620EE3EE231
:10DB300045E652E4C701B6010E941385AB01BC0162
:10DB400021E0C8010E94BD46B801CE0143960E9463
:10DB50004B476BE679E0CE0143960E94A545BE0196
:10DB6000675E7F4F0E94BC456BE679E00E94A54549
:10DB7000BE01615E7F4F0E94BC45BC018DEC9EE002
:10DB80000E947446CE0143960E948946C8010E94B5
:10DB90008946CE0149960E948946CE014F960E9441
:10DBA00089462DE2421621E052066104710474F4A4
:10DBB00069A57AA58BA59CA525E030E040E050E062
:10DBC0000E94E085672B682B692BA1F563ED7EE051
:10DBD000C8010E944B4745E050E06FEF7FEFC8015E
:10DBE00049D7C8010E9489466DE57AE0C8010E94C4
:10DBF0003A4A45E050E061EF7FEFC801EDD7C80138
:10DC00000E94894669EC79E0C8010E943A4AC8013D
:10DC100072D6C8010E9489466DEC7EE0C8010E9460
:10DC20004B4745E050E060E070E0C801A4D6C80171
:10DC30000E9489466DEC7EE089ED9EE00E94DB4506
:10DC40003FE1431651046104710434F4C9A4DAA419
:10DC5000EBA4FCA4F7FC10C069ED7EE0C8010E94B3
:10DC60004B47C80140D9C8010E94894669EC79E058
:10DC700089ED9EE00E945F46B201C30177FE04C0B9
:10DC800069A97AA98BA99CA90E94204DA7C023E06D
:10DC90004DA15EA16FA178A5CE0143960E94BD461D
:10DCA00060E37AE0C8010E943A4A63ED7EE0C80171
:10DCB0000E94BC456FE57AE00E94A545BE016D5EFD
:10DCC0007F4F0E94BC4568E37AE00E94A545BC01F5
:10DCD00083ED9EE00E947446C8010E948946CE01F1
:10DCE00043960E94894649855A856B857C8523E049
:10DCF000CE0149960E948E464D815E816F81788566
:10DD000023E0C8010E948E46B801CE0143960E94CE
:10DD10004B4764E67AE0CE0143960E94A545BE01DA
:10DD2000675E7F4F0E94BC4568E37AE00E94A5458C
:10DD3000BC018DEC9EE00E947446CE0143960E9489
:10DD40008946C8010E948946CE0149960E948946AB
:10DD50002DE2421621E052066104710474F469A5B3
:10DD60007AA58BA59CA525E030E040E050E00E941C
:10DD7000E085672B682B692BE1F463ED7EE0C80139
:10DD80000E944B474AE050E06FEF7FEFC80172D628
:10DD9000C8010E9489466DEC7EE0C8010E944B4795
:10DDA0004AE050E060E070E0C801E5D5C8010E949B
:10DDB000894669ED7EE0C8010E944B47C80193D8AF
:10DDC000C8010E94894669EC79E089ED9EE00E94D5
:10DDD0005F46C301B2010E94204D1DAA0E94584D0A
:10DDE0006B017C0122962CAD3DAD4EAD5FAD22970F
:10DDF000C21AD30AE40AF50AC9A6DAA6EBA6FCA65B
:10DE0000C9CC63ED7EE0CE010D960E944B474AE0FF
:10DE100050E06FEF7FEFCE010D96DED6CE010D966E
:10DE20000E948946CDA8CC2099F16DE57AE0CE011B
:10DE30000D960E943A4A45E050E061EF7FEFCE0137
:10DE40000D96CAD6CE010D960E9489468091770B19
:10DE5000882389F06AE67DE0CE010D960E94434753
:10DE600045E050E060E070E0CE010D96B5D6CE0101
:10DE70000D960E94894669EC79E0CE010D960E94CC
:10DE80003A4ACE010D9637D5CE010D960E948946AD
:10DE90006DEC7EE0CE010D960E944B474AE050E0CB
:10DEA0006FEF7FEFCE010D9666D5CE010D960E94E5
:10DEB0008946C75BDF4F0FB6F894DEBF0FBECDBFFC
:10DEC000DF91CF911F910F91FF90EF90DF90CF9056
:10DED000BF90AF909F908F907F906F905F904F908A
:10DEE0003F902F9008954F925F926F927F928F9202
:10DEF0009F92AF92BF92CF92DF92EF92FF920F93D9
:10DF00001F93CF93DF93CDB7DEB7C654D1090FB6B9
:10DF1000F894DEBF0FBECDBF8C0169EC79E0CE0175
:10DF20008B960E943A4A69EC79E0CE0185960E9470
:10DF30003A4ABE016F5F7F4F88E09FE00E944949E7
:10DF40008D889E88AF88B88C498C5A8C6B8C7C8C61
:10DF50008D8D9E8DAF8DB8A127968CAF9DAFAEAF46
:10DF6000BFAF2797C8010197039708F0C0C1A3016D
:10DF70009201C501B40190580E94B1862BED3FE09B
:10DF800049EC5FE30E943E8620913F0230914002BF
:10DF900040914102509142020E943E866B017C01F9
:10DFA00020E030E0A9010E94AE8487FD09C0C09244
:10DFB0009310D0929410E0929510F092961010C0A9
:10DFC0002BED3FE049EC50E4C701B6010E943E86CC
:10DFD0006093931070939410809395109093961083
:10DFE000C0909310D0909410E0909510F0909610FF
:10DFF0002BED3FE049EC50E4C701B6010E94F387E6
:10E00000181684F42BED3FE049EC50E4C701B6014B
:10E010000E943D86609393107093941080939510A6
:10E020009093961020E030E044E353E46091931025
:10E030007091941080919510909196100E94138584
:10E040002BED3FE049E450E40E94048760938F1079
:10E050007093901080939110909392100E949D87DE
:10E060004AE0CE01C7960E94184767E67AE0CE01E3
:10E07000C1960E943A4ABE01695C7F4FCE01C196AB
:10E080000E94BC4561E77AE00E94A545BC018FED86
:10E090009EE00E947446CE01C1960E948946CE0140
:10E0A000C7960E948946C0908F10D0909010E09043
:10E0B0009110F090921020E030E044EB52E4C70160
:10E0C000B6010E94AE84181694F020E030E040E0E3
:10E0D0005FE3C701B6010E943E860E949D874AE029
:10E0E000CE01C7960E94184768E77AE023C020E077
:10E0F00030E044E353E4C701B6010E94AE84181631
:10E10000A4F1A701960160E070E884E393E40E9423
:10E110003D8660938F107093901080939110909330
:10E1200092100E949D874AE0CE01C7960E94184730
:10E130006BE77AE0CE01C1960E943A4ABE01695C63
:10E140007F4FCE01C1960E94BC45BC01CE018B968B
:10E150000E947446CE01C1960E948946CE01C796A0
:10E160000E9489466EE077E063C020E030E047E837
:10E1700053E4C701B6010E94AE84181604F120E0F2
:10E1800030E044E353E4C701B6010E943D8620E03D
:10E1900030E040E05FE30E943E8660938F10709312
:10E1A000901080939110909392100E949D874AE066
:10E1B000CE01C7960E9418476BE77AE01FC0A701FF
:10E1C000960160E070E084EB93E40E943D8620E0DD
:10E1D00030E040E05FE30E943E8660938F107093D2
:10E1E000901080939110909392100E949D874AE026
:10E1F000CE01C7960E94184768E77AE0CE01C19623
:10E200000E943A4ABE01695C7F4FCE01C1960E94CE
:10E21000BC45BC01CE018B960E947446CE01C196CE
:10E220000E948946CE01C7960E9489466EE77AE031
:10E23000CE0185960E945F46BE01655D7F4FCE018F
:10E24000C1960E944B474AE050E060E070E0CE018A
:10E25000C196C2D4CE01C1960E9489460E94584DF3
:10E26000C0909710D0909810E0909910F0909A106C
:10E27000A4E6CA0ED11CE11CF11CC616D706E8069E
:10E28000F90608F423C20E94584D0E94B2846B0123
:10E290007C016091971070919810809199109091E5
:10E2A0009A100E94B48420E030E048EC51E40E94CF
:10E2B0003E869B01AC01C701B6010E94AE8487FD7A
:10E2C00005C26BE679E0CE01C1960E943A4ABE01D2
:10E2D0006B5D7F4FCE01C1960E94BC45BC01CE0153
:10E2E0008B960E94DB45CE01C1960E948946C801EB
:10E2F0000297029708F0C4C120E030E040E251E408
:10E30000C501B4010E9413856B017C0120E030E05F
:10E3100040E251E4C301B2010E9413854B015C014C
:10E3200020E030E040E251E427966CAD7DAD8EAD4B
:10E330009FAD27970E9413852B013C010E94584DE9
:10E340002091CA0A3091CB0A4091CC0A5091CD0A53
:10E35000621B730B840B950B0E94B28420E030E0AB
:10E360004AE754E40E940487AB01BC0123E0CE01DC
:10E37000C7960E94BD4660E37AE0CE01C1960E9436
:10E380003A4ABE01695C7F4FCE01C1960E94BC45EE
:10E390006CE676E00E94A545BC018DEC9EE00E94F3
:10E3A0007446CE01C1960E948946CE01C7960E944E
:10E3B00089466DEC7EE0CE01C1960E944B476FED21
:10E3C0007EE0CE01C1960E94BC45BE01655D7F4FD7
:10E3D0000E94BC45BC01CE018B960E947446CE01C2
:10E3E000C1960E94894660E87AE089ED9EE00E942D
:10E3F0005F4621E0B701A601CE01C1960E94BD464D
:10E40000BE016F5C7F4F89ED9EE00E94DB45CE012F
:10E41000C1960E94894621E0B301A201CE01CD96AA
:10E420000E94BD4621E0B501A401CE01C7960E941D
:10E43000BD466BE679E0CE01C1960E943A4ABE0124
:10E44000695C7F4FCE01C1960E94BC456BE679E0C6
:10E450000E94A545BE01635C7F4F0E94BC456BE8EE
:10E460007AE00E94A545BC0189ED9EE00E94DB4553
:10E47000CE01C1960E948946CE01C7960E94894668
:10E48000CE01CD960E948946A7019601C701B6012B
:10E490000E9413856B017C01A5019401C501B401A3
:10E4A0000E9413859B01AC01C701B6010E943E8604
:10E4B0006B017C01A3019201C301B2010E9413858B
:10E4C0009B01AC01C701B6010E943E860E940289F1
:10E4D0006B017C0160938B1070938C1080938D1076
:10E4E00090938E106FE87AE089ED9EE00E94CD4512
:10E4F00021E0B701A601CE01C1960E94BD46BE0132
:10E500006F5C7F4FCE01C7960E944B476DE97AE062
:10E51000CE01C7960E94A545BC018FED9EE00E94EA
:10E520007446CE01C7960E948946CE01C1960E94CC
:10E5300089466FED7EE089ED9EE00E94DB45C0904C
:10E540008B10D0908C10E0908D10F0908E1020E009
:10E5500030E04AE754E4C701B6010E94F38787FD23
:10E5600029C020E030E04AE754E4C701B6010E9428
:10E570000487AB01BC0123E0CE01C1960E948E4608
:10E58000BE016F5C7F4FCE01C7960E944B476EE97C
:10E590007AE0CE01C7960E94A545BC018FED9EE0B2
:10E5A0000E947446CE01C7960E948946CE01C1964C
:10E5B0000E94894620E030E64AE656E460918B10DE
:10E5C00070918C1080918D1090918E100E94AE846D
:10E5D000BE01655D7F4F87FF4FC0CE01C1960E948F
:10E5E0004B476FE27AE0CE01C1960E94A54569EDE6
:10E5F0007EE00E94BC45BC0189ED9EE00E9474460D
:10E60000CE01C1960E94894603301105A1F469ED3F
:10E610007EE0CE01C1960E944B47CE01C1960E947A
:10E620007367CE01C1960E94894669EC79E089ED55
:10E630009EE00E945F4663E97AE0CE01C1960E94A7
:10E640003A4A6FED7EE0CE01C1960E94BC45BC0106
:10E65000CE01C7960E944B474AE050E06FEF7FEF34
:10E66000CE01C79688D1CE01C7960E948946CE01B9
:10E67000C1960E94894604C089ED9EE00E947446BE
:10E680006AE070E080E090E00E94204DCE01859627
:10E690000E948946CE018B960E948946CA5BDF4F55
:10E6A0000FB6F894DEBF0FBECDBFDF91CF911F91A3
:10E6B0000F91FF90EF90DF90CF90BF90AF909F9021
:10E6C0008F907F906F905F904F90089569EC79E004
:10E6D000CE01C1960E943A4ACE01C1960CD1CE011C
:10E6E000C1960E948946BE016B5D7F4F8BEC9FE017
:10E6F0000E94554AE6CD1F93CF93DF93CDB7DEB787
:10E70000A8970FB6F894DEBF0FBECDBF182F0E949A
:10E71000685D8EE10E945E5D62E08FEE9DE00E948A
:10E72000245560E08FEE9DE00E9424550E94015D1B
:10E730008EE10E945E5D61E08FEE9DE00E942455B7
:10E7400060E28FEE9DE00E9424550E94015D80E210
:10E7500090E090930C0F80930B0F80E090E8A9E875
:10E76000B4E480934C0290934D02A0934E02B09378
:10E770004F0280E090E0A5E7B4E4809348029093D4
:10E780004902A0934A02B0934B02BE016F5F7F4FD4
:10E7900088E09FE00E94FC48112309F476C08BE2D8
:10E7A0009EE00E94EC5B6CE17EE082E59DE00E94D1
:10E7B000634ACE0101960E94FD5B6DE07EE082E53A
:10E7C0009DE00E94634A6D857E858F8598890E94B1
:10E7D0000E5C6EEF7DE082E59DE00E94634A6989F0
:10E7E0007A898B899C890E940E5C6FEE7DE082E5C0
:10E7F0009DE00E94634A20E030E040E251E4698DF0
:10E800007A8D8B8D9C8D0E94138542E050E00E9492
:10E81000005D8CE99AE00E94FD5B60EE7DE082E5A0
:10E820009DE00E94634A20E030E040E251E46D8DBB
:10E830007E8D8F8D98A10E94138542E050E00E944A
:10E84000005D8CE99AE00E94FD5B61ED7DE082E570
:10E850009DE00E94634A20E030E040E251E469A17B
:10E860007AA18BA19CA10E94138542E050E00E94F6
:10E87000005D8CE99AE00E94FD5B8CEA9DE00E94BD
:10E88000EC5B89EC99E00E94FD5B64EF71E080E055
:10E8900090E00E94204DA8960FB6F894DEBF0FBE00
:10E8A000CDBFDF91CF911F91089580917F04882380
:10E8B00009F180917E048823E9F061E08BEC9FE010
:10E8C0000E9451418BE39FE10197F1F760E080E006
:10E8D0000E94B25B69EA7EE08BEC9FE00E94634A93
:10E8E00061E080E00E94B25B69E97EE08BEC9FE032
:10E8F0000C94634A0895CF93DF9320917F042223E1
:10E90000A9F020917E04222389F0EC016FED8BECBD
:10E910009FE00E944E4A8C819D81892B39F0BE0177
:10E920008BEC9FE0DF91CF910C94554ADF91CF9112
:10E93000089580917F04882379F080917E04882354
:10E9400059F06FED8BEC9FE00E944E4A69E579E04B
:10E950008BEC9FE00C94444B089580917F048823B6
:10E9600049F080917E04882329F060E08BEC9FE0E1
:10E970000C94CE3E08958F929F92AF92BF92EF92E9
:10E98000FF920F931F93CF93DF937C01EB018A01DA
:10E9900080917F04882309F462C080917E048823DB
:10E9A00009F45DC077FF18C0C095D09561E08C2F49
:10E9B0000E94B25BB7018BEC9FE00E94554A68E869
:10E9C0007EE08BEC9FE00E94634AF701848161E066
:10E9D0008C0F0E94B25B33C00E94584D8090730B25
:10E9E0009090740BA090750BB090760B24E6820E7D
:10E9F000911CA11CB11C86169706A806B90678F5CD
:10EA000061E08C2F0E94B25BB7018BEC9FE00E940B
:10EA1000554A67E77EE08BEC9FE00E94634AF7016E
:10EA2000848161E08C0F0E94B25B0E94584D60931C
:10EA3000730B7093740B8093750B9093760BB801E6
:10EA4000110F880B990BDF91CF911F910F91FF90C0
:10EA5000EF90BF90AF909F908F900C94204DDF91DE
:10EA6000CF911F910F91FF90EF90BF90AF909F902B
:10EA70008F900895AF92BF92CF92DF92EF92FF9264
:10EA80000F931F93CF93DF93CDB7DEB762970FB687
:10EA9000F894DEBF0FBECDBF20917F04222309F47E
:10EAA0008AC020917E04222309F485C06A017B017B
:10EAB0005C010E94584D0091971010919810209180
:10EAC000991030919A100C591F4F2F4F3F4F061736
:10EAD00017072807390708F06EC0F7FE08C087013E
:10EAE0000095109560E0802F0E94B25B43C060E00B
:10EAF00080E00E94B25B0E94584D28EE33E040E077
:10EB000050E00E94E085BA01A9012AE0CE010196F9
:10EB10000E94EC46BE016F5F7F4FCE0107960E94B8
:10EB20004B476CE676E0CE0107960E94A545BC01F6
:10EB3000CE010D960E944B47CE0107960E94894652
:10EB4000CE0101960E948946BE01635F7F4F8BEC28
:10EB50009FE00E94554A09891A89E114F10431F0B5
:10EB60000E0D1F1D60E0802F0E94B25BCE010D963E
:10EB70000E948946B5018BEC9FE00E94554A66E6EB
:10EB80007EE08BEC9FE00E94634AF501848160E0A7
:10EB9000800F0E94B25B0E94584D60939710709353
:10EBA00098108093991090939A10B601DD0C880B01
:10EBB000990B0E94204D62960FB6F894DEBF0FBEEF
:10EBC000CDBFDF91CF911F910F91FF90EF90DF901C
:10EBD000CF90BF90AF900895BF92CF92DF92EF9207
:10EBE000FF920F931F93CF93DF93CDB7DEB762975A
:10EBF0000FB6F894DEBF0FBECDBF6C018B017A015A
:10EC000080917F04882309F475C080917E04882355
:10EC100009F470C077FF07C00095109560E0802F61
:10EC20000E94B25B46C060E080E00E94B25B0E943E
:10EC3000584D28EE33E040E050E00E94E085BA01F4
:10EC4000A9012AE0CE0101960E94EC46BE016F5F49
:10EC50007F4FCE0107960E944B476CE676E0CE01CF
:10EC600007960E94A545BC01CE010D960E944B4718
:10EC7000CE0107960E948946CE0101960E948946E0
:10EC8000BE01635F7F4F8BEC9FE00E94554AB988BD
:10EC900060E08B2D0E94B25B0115110511F40B2D64
:10ECA00004C060E0802F0E94B25BCE010D960E94EE
:10ECB0008946B6018BEC9FE00E94554A65E57EE0EF
:10ECC0008BEC9FE00E94634AF601848160E0800F34
:10ECD0000E94B25B0E94584D6093971070939810F9
:10ECE0008093991090939A10B701FF0C880B990BA1
:10ECF0000E94204D62960FB6F894DEBF0FBECDBFC6
:10ED0000DF91CF911F910F91FF90EF90DF90CF9007
:10ED1000BF9008950895CF92DF92EF92FF920F93E4
:10ED20001F93CF93DF93EC016A017B01E889F98996
:10ED300082E080834115514E61057105B1F060E0BC
:10ED400079E08DE390E0A70196010E940C8689018D
:10ED50009A01015011092109310936952795179516
:10ED60000795980101151041A8F0E889F9891082EA
:10ED700060E874E88EE190E0A70196010E940C869D
:10ED8000DA01C9010197A109B109B695A79597952F
:10ED900087959C01EC85FD853083EE85FF8520837A
:10EDA000188EEC89FD8986E08083EA89FB89808161
:10EDB00080618083EA89FB89808188608083EA8919
:10EDC000FB89808180688083EA89FB8980818F7DCF
:10EDD0008083DF91CF911F910F91FF90EF90DF9093
:10EDE000CF900895CF92DF92EF92FF920F931F93EF
:10EDF000E82FF92F05C0015011092109310961F1EE
:10EE0000908196239417B9F305C001501109210987
:10EE1000310911F1908196239413F7CFC12CD12C95
:10EE2000E12CF12C0AC08FEFC81AD80AE80AF80AB8
:10EE30000C151D052E053F0579F08081862384176A
:10EE400091F36C2D7D2D8E2D9F2D1F910F91FF9095
:10EE5000EF90DF90CF90089560E070E080E090E068
:10EE60001F910F91FF90EF90DF90CF900895CF9377
:10EE7000DF93CDB7DEB72C970FB6F894DEBF0FBE89
:10EE8000CDBF789484B5826084BD84B5816084BD33
:10EE900085B5826085BD85B5816085BD80916E0038
:10EEA000816080936E001092810080918100826069
:10EEB00080938100809181008160809381008091A6
:10EEC00080008160809380008091B1008460809395
:10EED000B1008091B00081608093B000809191007A
:10EEE0008260809391008091910081608093910075
:10EEF000809190008160809390008091A100826059
:10EF00008093A1008091A10081608093A1008091F5
:10EF1000A00081608093A000809121018260809395
:10EF20002101809121018160809321018091200144
:10EF300081608093200180917A00846080937A00C0
:10EF400080917A00826080937A0080917A0081605B
:10EF500080937A0080917A00806880937A00109282
:10EF6000C10061E089E10E94974C61E089E10E9463
:10EF7000654C20E042E060E18BEC9FE00E94DA41CA
:10EF80000E9419520E9428568EED93E09093690BCF
:10EF90008093680B0E94CA8580937F108FED93E069
:10EFA0000E94CA858093801080917F10909180107C
:10EFB0001816190654F410924702019731F4109272
:10EFC000801010927F100E94D25F67E779E08BEC8F
:10EFD0009FE00E94444B40E855E260E070E082E52B
:10EFE0009DE099DE40E855E260E070E088E19CE059
:10EFF00092DE64E670E080E090E00E94204D809117
:10F000004702882331F068EE73E080E090E00E94D0
:10F01000204D82E59DE00E94A747F82E82E7F81672
:10F0200009F425C11092690B1092680B59E0C52EA6
:10F0300050E1D52E00E010E0C8010E94CA85F6011B
:10F0400081936F010F5F1F4F06371105A9F780915C
:10F05000091090910A10A0910B10B0910C108536F8
:10F060009105A105B1050CF402C180934302909370
:10F070004402A0934502B093460280910D109091F6
:10F080000E10A0910F10B091101080933F0290933A
:10F090004002A0934102B0934202809111109091DE
:10F0A0001210A0911310B091141080933B02909312
:10F0B0003C02A0933D02B0933E0265E270E1CE01B6
:10F0C00001960E943A4ABE016F5F7F4F85EC9FE038
:10F0D0000E940746CE0101960E9489468091151034
:10F0E00090911610A0911710B091181080933702CC
:10F0F00090933802A0933902B0933A02809119108C
:10F1000090911A10A0911B10B0911C1080933302A3
:10F1100090933402A0933502B093360280911D1073
:10F1200090911E10A0911F10B091201080932F027B
:10F1300090933002A0933102B0933202809121105B
:10F1400090912210A0912310B091241080932B0253
:10F1500090932C02A0932D02B0932E0280912D103B
:10F1600090912E10A0912F10B09130108093C00478
:10F170009093C104A093C204B093C3048091311052
:10F1800090913210A0913310B09134108093BC0450
:10F190009093BD04A093BE04B093BF04809135103A
:10F1A00090913610A0913710B09138108093B80428
:10F1B0009093B904A093BA04B093BB048091391022
:10F1C00090913A10A0913B10B0913C108093B40400
:10F1D0009093B504A093B604B093B70480913D100A
:10F1E00090913E10A0913F10B09140108093270263
:10F1F00090932802A0932902B0932A028090531082
:10F2000090905410A0905510B0905610A501940104
:10F21000C501B4010E944389811108C08092230274
:10F2200090922402A0922502B092260200E010E003
:10F23000F801E95AFF4E80809180A280B380A50139
:10F240009401C501B4010E944389811107C0F801EE
:10F25000E05CF44F80829182A282B3820C5F1F4FE8
:10F260000832110529F781E090E00E94A2574EE88C
:10F27000E42EEF0CF1E0FE1570F4809109109091EE
:10F280000A10A0910B10B0910C1085369105A105C4
:10F29000B1050CF041C18091430290914402A091CC
:10F2A0004502B09146028093091090930A10A093F2
:10F2B0000B10B0930C1080913F0290914002A091EE
:10F2C0004102B091420280930D1090930E10A093D2
:10F2D0000F10B093101080913B0290913C02A091CE
:10F2E0003D02B0913E028093111090931210A093B2
:10F2F0001310B093141082E7F81220C085E290E159
:10F30000892BE1F00091C90F1091CA0F0115110569
:10F3100019F41092251012C00730110510F007E003
:10F3200010E06091C50F7091C60FA80185E290E1D1
:10F330000E94048CF801EB5DFF4E10828091370231
:10F3400090913802A0913902B0913A028093151041
:10F3500090931610A0931710B09318108091330259
:10F3600090913402A0913502B09136028093191029
:10F3700090931A10A0931B10B0931C1080912F0231
:10F3800090913002A0913102B091320280931D1011
:10F3900090931E10A0931F10B093201080912B0209
:10F3A00090912C02A0912D02B0912E0280932110F9
:10F3B00090932210A0932310B09324108091C00446
:10F3C0009091C104A091C204B091C30480932D1008
:10F3D00090932E10A0932F10B09330108091BC0406
:10F3E0009091BD04A091BE04B091BF0480933110F0
:10F3F00090933210A0933310B09334108091B804DE
:10F400009091B904A091BA04B091BB0480933510D7
:10F4100090933610A0933710B09338108091B404B5
:10F420009091B504A091B604B091B70480933910BF
:10F4300090933A10A0933B10B0933C108091270218
:10F4400090912802A0912902B0912A0280933D1048
:10F4500090933E10A0933F10B093401080912302F0
:10F4600090912402A0912502B0912602809353101E
:10F4700090935410A0935510B0935610E0E4FBE025
:10F48000A7E5B0E141915191619171914D935D93E7
:10F490006D937D938BE0E836F807A1F782E59BE05A
:10F4A0000E94EC5B21E4A22E20E1B22E31E1C32EBA
:10F4B00032E0D32E00E010E0809111029091120210
:10F4C00080179107F4F04601F601819191916F0147
:10F4D000F501819391935F014AE050E0B80182E524
:10F4E0009DE00E942B4B68E879E082E59DE00E9458
:10F4F000444BF401808191810E940F640F5F1F4F84
:10F50000DBCFF1E0FE1540F01092690B1092680B12
:10F5100080E090E00E94F95F64E670E080E090E0B7
:10F520000E94204DF89482E08093B0008093B10057
:10F5300094E69093B3001092B20080937000789498
:10F540008093FB0D1092FE0D8091FC0D60E00E94F7
:10F55000974C6DE879E0CE0101960E943A4A4AE064
:10F5600050E06FEF7FEFCE01019636DBCE010196C2
:10F570000E94894660ED78E0CE0107960E943A4AE3
:10F5800065EC7FE0CE0107960E94BC45BC01CE0130
:10F5900001960E944B474AE050E06FEF7FEFCE01AB
:10F5A0000196E9D9CE0101960E948946CE010796BF
:10F5B0000E9489466BE879E0CE0107960E943A4A9C
:10F5C00065EC7FE0CE0107960E94BC456DE979E0CD
:10F5D0000E94A545BC01CE0101960E944B47CE0179
:10F5E00001960E947367CE0101960E948946CE0162
:10F5F00007960E94894664E670E080E090E00E94F1
:10F60000204D0E94685D64E670E080E090E00E941A
:10F61000204D83E20E945E5D81E090E00E94CD5F1C
:10F620000E94015D83E090E090933F0B80933E0B3E
:10F630008CE40E94DF4F4B015C0162E370E080E0EC
:10F6400090E00E94204DA5019401C501B4010E94E3
:10F650004389882309F46CC086E60E94DF4F4B0182
:10F660005C0162E370E080E090E00E94204DA50123
:10F670009401C501B4010E944389882309F458C04C
:10F6800081E090E090933F0B80933E0B40E052EC82
:10F6900061E070E085EB9CE03EDB64E670E080E0DA
:10F6A00090E00E94204D0E94955040E052EC61E0B5
:10F6B00070E085EB9CE02FDB8CED95E0A0E0B0E006
:10F6C0008093B90C9093BA0CA093BB0CB093BC0C74
:10F6D00064E670E080E090E00E94204D92E0C92E48
:10F6E000D12CE12C65E070E080E090E00E94204D9C
:10F6F00000E010E0812C912C5401E11032C185EB27
:10F700009CE00E94C947892B39F4E5E18E169104EB
:10F71000A104B1040CF025C1033011050CF45AC149
:10F7200020C1EE2009F42BC189E39BE00E94EC5B31
:10F7300080913E0B90913F0B039721F48AE09BE070
:10F740000E94EC5B83E08093F10E0E94685D80ED87
:10F750000E947560853509F068C18AEA0E9496604A
:10F760009093F30E8093F20E8CEA0E949660909331
:10F77000F50E8093F40E8EEA0E9496609093F70E39
:10F780008093F60E80EB0E9496609093030F809317
:10F79000020F82EB0E9496609093050F8093040FF6
:10F7A00084EB0E9496609093070F8093060F86EB80
:10F7B0000E9496609093F90E8093F80E88EB0E9459
:10F7C00096609093FB0E8093FA0E8AEB0E949660EF
:10F7D0009093FD0E8093FC0E8CEB0E9496609093AC
:10F7E000FF0E8093FE0E8EEB0E9496609093010FA9
:10F7F0008093000F60ED7AE089ED9EE00E94E14584
:10F800000E94D6600E94B4840E949D870E94B484A6
:10F8100020E030E048EC52E40E940487AB01BC01D8
:10F8200022E0CE0107960E94BD46BE01695F7F4F70
:10F83000CE0101960E944B4760EC76E0CE01019626
:10F840000E94A545BC0189ED9EE00E94DB45CE01EA
:10F8500001960E948946CE0107960E94894669ED6D
:10F860007EE082E59DE00E94344B69EB7AE089ED11
:10F870009EE00E94E14560914302709144028091B4
:10F880004502909146020E94B48420E030E048ECAA
:10F8900052E40E940487AB01BC0122E0CE0107962E
:10F8A0000E94BD46BE01695F7F4FCE0101960E9456
:10F8B0004B4760EC76E0CE0101960E94A545BC0165
:10F8C00089ED9EE00E94DB45CE0101960E948946AB
:10F8D000CE0107960E94894669ED7EE082E59DE0B3
:10F8E0000E94344BF1E6FF1205C081E00E948B3983
:10F8F00081E011C082E59DE00E94A747182F64E6D1
:10F9000070E080E090E00E94204D113671F380E0BD
:10F910000E948B3980E00E947B7364E670E080E097
:10F9200090E00E94204D10914702112331F068EEC3
:10F9300073E080E090E00E94204D6BE775E085EE7B
:10F940009EE00E945F4682E090E090933D0B8093A2
:10F950003C0B11110E9408650E9491070E94784893
:10F96000FBCF64E670E080E090E00E94204DCA94F6
:10F97000CD2809F4D6CECC24C394D12CB3CE10928A
:10F980003F0B10923E0B0E94955064E670E080E0C1
:10F9900090E00E94204D40E855E260E070E085EB89
:10F9A0009CE0B9D985EB9CE00E94C947892B09F4FA
:10F9B000BFCE8FE19BE00E94EC5B82E090E09093F1
:10F9C0003F0B80933E0B64E670E080E090E00E9485
:10F9D000204DAECE85EB9CE00E94C947892B69F093
:10F9E00085EB9CE00E94A747E1E0F0E0EC0FFD1FF3
:10F9F000E00FF11F80830F5F1F4F65E070E080E034
:10FA000090E00E94204D023011054CF089818B3B23
:10FA100031F4EE24E3948A818A3A09F0E12C8FEFE5
:10FA2000881A980AA80AB80A68CE64EE7AE0CE016D
:10FA300001960E944347CE0101960E947367CE0152
:10FA400001960E9489461092100267CF8DEC9EE0CD
:10FA50000E94894683ED9EE00E94894689ED9EE0E2
:10FA60000E9489468FED9EE00E94894685EE9EE0C9
:10FA70000E9489468BEE9EE00E94894683E39FE0C8
:10FA80000E9489468FEB9FE00E94894685EC9FE0AB
:10FA90000C948946CF92DF92EF92FF921F93CF93FF
:10FAA000DF93182FCAE0D0E0C12CD12C7601812F32
:10FAB0000E94D64CBC01990F880B990B55D79B011E
:10FAC000AC01C701B6010E943E866B017C0162E376
:10FAD00070E080E090E00E94204D219741F720E007
:10FAE00030E040E251E4C701B6010E94048720E003
:10FAF00030E040EA50E497D720E030E040E85AE3B5
:10FB000092D7DF91CF911F91FF90EF90DF90CF9030
:10FB100008958F929F92AF92BF92CF92DF92EF9211
:10FB2000FF92CF9310921B0C10921A0C88EE93E068
:10FB3000A0E0B0E080931C0C90931D0CA0931E0CD1
:10FB4000B0931F0C24E035E03093190C2093180C6F
:10FB500045E351E05093250C4093240C44E351E0DD
:10FB60005093270C4093260C40E351E05093290C0E
:10FB70004093280C41E351E050932B0C40932A0C06
:10FB800042E351E050932D0C40932C0C46E351E09E
:10FB900050932F0C40932E0C1092310C1092320C7B
:10FBA0001092330C1092340C1092B80C1092B70CC7
:10FBB0008093B90C9093BA0CA093BB0CB093BC0C7F
:10FBC0003093B60C2093B50C45ED50E05093C20C29
:10FBD0004093C10C44ED50E05093C40C4093C30CCF
:10FBE00040ED50E05093C60C4093C50C41ED50E001
:10FBF0005093C80C4093C70C42ED50E05093CA0C90
:10FC00004093C90C46ED50E05093CC0C4093CB0C84
:10FC10001092CE0C1092CF0C1092D00C1092D10CEE
:10FC20001092550D1092540D8093560D9093570DD0
:10FC3000A093580DB093590D3093530D2093520D4E
:10FC400025EC30E030935F0D20935E0D24EC30E026
:10FC50003093610D2093600D20EC30E03093630D04
:10FC60002093620D21EC30E03093650D2093640DFC
:10FC700022EC30E03093670D2093660D26EC30E0E7
:10FC80003093690D2093680D10926B0D10926C0DDE
:10FC900010926D0D10926E0D1092F20D1092F10DEA
:10FCA0008093F30D9093F40DA093F50DB093F60DA2
:10FCB00086E195E09093F00D8093EF0D1092CE0FBA
:10FCC0001092CD0F82E395E09093CC0F8093CB0FF1
:10FCD0001092DB0F8FEF8093DA0F1092D90F1092F2
:10FCE000DC0F8FE38093D60F1092D70F1092D80FAE
:10FCF0001092D50F1092D40F84E08093DD0F82E034
:10FD00008093DE0F81E08093DF0FC0E1C093E00FAE
:10FD100080E28093E10F80E48093E20F80E880939B
:10FD2000E30F40E050E063E08BEC9FE00E94BA3EBE
:10FD30006CEE79E085EC9FE00E943A4A63EF79E04F
:10FD40008FEB9FE00E943A4A88E18093BC0F81E1EB
:10FD50008093BD0FC093BE0F61E088E10E94974C75
:10FD600061E08091BC0F0E94654C60E08091BD0F06
:10FD70000E94974C60E08091BE0F0E94974C61E01A
:10FD80008091BD0F0E94654C61E08091BE0F0E9482
:10FD9000654C61E08091BC0F0E94654C10924F0F42
:10FDA0001092530F1092520F1092540F88E295E068
:10FDB00090934E0F80934D0F80E090E0FC01E35B49
:10FDC000F04F148E10A2178E11A206968C33910557
:10FDD000A9F78AEC94E09093B00F8093AF0F86EC74
:10FDE00094E09093B20F8093B10F84E08093B30FAF
:10FDF0008093B40F8EEC94E09093AE0F8093AD0F90
:10FE00008AE090E09093B60F8093B50F84EF91E075
:10FE10009093B80F8093B70F1092BB0F1092BA0F48
:10FE20001092A90F1092AA0F1092AB0F1092AC0F64
:10FE30001092B90F81E08093390F10923A0F83EC42
:10FE40009BEAA6E7BBE380933B0F90933C0FA09304
:10FE50003D0FB0933E0F88ED9BE6A6E7BBE3809392
:10FE60003F0F9093400FA093410FB093420F82EF4A
:10FE700094EEA4E6BBE38093430F9093440FA093CA
:10FE8000450FB093460F69EC79E083E39FE00E9451
:10FE90003A4A8091C4049091C5049093320F8093A4
:10FEA000310F8090C0049090C104A090C204B09023
:10FEB000C3042091BC043091BD044091BE04509114
:10FEC000BF04C501B401D9D66B017C0160932D0F2D
:10FED00070932E0F80932F0F9093300F6091B80482
:10FEE0007091B9048091BA049091BB046093210F82
:10FEF0007093220F8093230F9093240F8092250FED
:10FF00009092260FA092270FB092280F2091B40450
:10FF10003091B5044091B6045091B704AED69B0120
:10FF2000AC01C701B60170D76093290F70932A0FF7
:10FF300080932B0F90932C0F84E595E09093090FFD
:10FF40008093080F8FEF9FEFDC0180931D0F90933C
:10FF50001E0FA0931F0FB093200F69EC79E08BEE7A
:10FF60009EE00E943A4A69EC79E085EE9EE00E94AC
:10FF70003A4A69EC79E08FED9EE00E943A4A69ECDA
:10FF800079E089ED9EE00E943A4A69EC79E083EDE0
:10FF90009EE00E943A4A69EC79E08DEC9EE00E9476
:10FFA0003A4A87E08093FC0D1092FD0DCF91FF90AF
:10FFB000EF90DF90CF90BF90AF909F908F9008957B
:10FFC000EF920F931F93CF93DF93E80147FD02C099
:10FFD00034E001C034E1E42F440FFF0BF7FF03C00E
:10FFE000F195E195F109E32E022F2E2FAE01BBD042
:10FFF000CE01DF91CF911F910F91EF900895662769
:020000021000EC
:1000000077273EC21F93FC0199278827BC01E894FB
:1000100011911032E9F3193010F01E30C8F31B3281
:1000200049F01D3241F4689405C04ED0610F711D36
:10003000811D911D119110531A30B8F33EF4909523
:100040008095709561957F4F8F4F9F4F1F910895B9
:10005000FB01DC0105900D920020E1F70895FC0101
:1000600005900020E9F7809590958E0F9F1F0895C9
:100070004532510518F4423008F004C0FB011082EB
:10008000CB010895BB274A3031F4992322F4BDE215
:10009000909581959F4F4FC02532310518F422303D
:1000A00008F004C0FA011082CA010895BB272A3063
:1000B00051F4992342F4BDE2909580957095619535
:1000C0007F4F8F4F9F4F16C0592F482F372F262F06
:1000D000660F771F881F991F660F771F881F991F4C
:1000E000620F731F841F951F660F771F881F991F4C
:1000F0000895BB27FA01A62F6217710581059105A6
:10010000330B30FB66F0AA27660F771F881F991FF5
:10011000AA1FA21710F0A21B63953850A9F7A05D83
:10012000AA3308F0A95DA19336F7B111B1931082FB
:10013000CA0104C4BB27FB015527AA27880F991FB2
:10014000AA1FA41710F0A41B83955051B9F7A05D06
:10015000AA3308F0A95DA193009779F7B111B19383
:100160001192CB01EBC34F925F926F927F929F925D
:10017000AF92BF92CF92DF92EF92FF920F931F93B5
:10018000CF93DF93CDB7DEB729970FB6F894DEBFD4
:100190000FBECDBF6A01122FB02E2BE3201720F027
:1001A000FF24F394F00E02C0BCE3FB2E0F2D27E0DA
:1001B000AE014F5F5F4FCAD2AC018981982F997011
:1001C000913031F0E1FC06C0E0FE06C090E205C0CF
:1001D0009DE203C09BE201C090E0EE2DE07183FF41
:1001E0003CC0911102C083E001C084E0811718F483
:1001F000212F281B01C020E0E1110BC0F601822F46
:1002000030E2882319F031938150FBCFC20ED11C0C
:1002100020E0992329F0D6019C93F60131966F01D5
:10022000C6010396E2FE0AC03EE4D6013C9341E4D7
:1002300011964C93119712963C9306C03EE6F60138
:10024000308341E641833283FC01322F40E2332385
:1002500009F442C041933150FACF82FF44C091115A
:1002600002C083E001C084E0811718F4212F281B0D
:1002700001C020E0E1110BC0F601822F30E288239B
:1002800019F031938150FBCFC20ED11C20E099238D
:1002900029F0D6019C93F60131966F01C6010396B1
:1002A000E2FE0BC039E4D6013C933EE411963C9348
:1002B000119736E412963C9307C039E6F601308375
:1002C0003EE6318336E63283FC01322F40E23323AF
:1002D00019F041933150FBCFFC01E20FF11D108268
:1002E0008EEF9FEFB7C0F1E0911101C0F0E06F2FEA
:1002F00070E01416150624F49A012F5F3F4F02C0D8
:1003000021E030E0260F371FBB2029F06B2D70E075
:100310006F5F7F4F02C060E070E0260F371F612FD4
:1003200070E0261737071CF4121B212F01C020E0B4
:100330003E2D387159F4D601322F60E2332319F083
:100340006D933150FBCFC20ED11C20E0FF2331F062
:10035000D6019C93B6016F5F7F4F6B01E1110BC01B
:10036000F601922F30E3992319F031939150FBCF8E
:10037000C20ED11C20E09F2D940F3A81782F70710E
:10038000A72E84FF03C0313309F49150191624F4C9
:10039000993018F098E001C091E0E42F852F57FFC5
:1003A00002C0E0E080E06E2F782FE0E0F0E0AEE207
:1003B0009A2E3A01691A71082A01461A570A0B2D1A
:1003C00010E01195019511096F3F8FEF780729F41F
:1003D000D6019C92C60101966C014617570784F01E
:1003E000661677066CF47F01E40CF51CA1E0B0E022
:1003F000AC0FBD1FEA0EFB1ED7011196BC9002C0C8
:1004000090E3B92E615071093196C60101967C01C5
:100410006017710724F0D601BC926C01D5CF641728
:10042000750741F4363320F4353321F4A11002C0AE
:1004300081E3B82EF601B082F701822F90E2882383
:1004400019F091938150FBCFF701E20FF11D10825B
:1004500080E090E029960FB6F894DEBF0FBECDBFC6
:10046000DF91CF911F910F91FF90EF90DF90CF9090
:10047000BF90AF909F907F906F905F904F90089546
:100480006F927F928F929F92AF92BF92CF92DF92A4
:10049000EF92FF920F931F93CF93DF93EC017B01B9
:1004A0006115710519F0DB018D939C938E010F5F2F
:1004B0001F4F7880872D90E021D2892B11F0E80121
:1004C000F5CFBDE27B1205C00F5F1F4F7980C1E001
:1004D00008C0EBE27E1204C08E010E5F1F4F7980D0
:1004E000C0E06801F1E0CF1AD10843E050E066E0D7
:1004F00072E0C6010BD2892BE9F4680122E0C20E3A
:10050000D11C45E050E061E072E0C601FFD1892BCB
:1005100021F4680187E0C80ED11CE114F10419F040
:10052000D701CD92DC92C111F9C060E070E080E8A3
:100530009FE7FDC043E050E06EEF71E0C601E6D1F9
:10054000892B51F4E114F10409F4EDC00E5F1F4F43
:10055000F70111830083E7C0680160E070E0CB0120
:1005600000E010E0F601D0EDD70DDA3050F52C2F79
:100570002260622E2C2F2870C2FF05C0211127C0D7
:100580000F5F1F4F24C0222311F001501109A5E075
:10059000B0E09B01AC0130D34B015C01880C991C8D
:1005A000AA1CBB1CC501B4016D0F711D811D911DDD
:1005B0006839A9E97A078A07A9E19A0740F0C66075
:1005C00005C0DE3F51F4C3FD44C0C8606C2EBFEFD0
:1005D000CB1ADB0A7080C62DC5CF2D2F2F7D25317C
:1005E000C1F540814D3211F4C06106C04B3221F09B
:1005F000319621E030E006C03296D60111964C913A
:1006000022E030E0A0EDA40FAA3018F0E21BF30BBB
:1006100020C040E050E04038BCE05B075CF49A0149
:10062000220F331F220F331F420F531F440F551F3A
:100630004A0F511D3196DF0111972C91A0EDA20FA9
:10064000AA3048F3C4FF03C0519541955109040FE6
:10065000151FC1FF07C0E114F10421F03197D70144
:10066000ED93FC937FD1C370C33019F06B017C0113
:1006700006C06B017C01F7FAF094F7F8F09420E0E3
:1006800030E0A901C701B60169D1882309F443C04C
:1006900017FF06C0119501951109CDE1D2E002C006
:1006A000C5E3D2E05E01B8E1AB1AB1084601BE2D48
:1006B000AF2D90E2E92EF12C0E151F057CF0FE0106
:1006C0002591359145915491B4018B2F9A2FABD13F
:1006D0004B01B82FA92F0E191F09EECF2497F594BF
:1006E000E794CA15DB0541F76401EB2EFA2E8E2D37
:1006F000880F8F2D881F8F3F41F020E030E0A90147
:10070000C701B6012BD1811106C082E290E090931F
:100710009C1080939B10C701B60109C060E070E097
:1007200080E89FEF04C060E070E080EC9FE7DF911D
:10073000CF911F910F91FF90EF90DF90CF90BF90DE
:10074000AF909F908F907F906F900895283008F021
:1007500027E03327DA01990F311D87FD916000965C
:100760006105710539F432602E5F3D9330E32A95BF
:10077000E1F708959F3F30F080387105610509F079
:100780003C5F3C5F3D93913008F08068911DDF93A2
:10079000CF931F930F93FF92EF92192F987F969507
:1007A000E92F96959695E90FFF27ED56FD4F99276E
:1007B0003327EE24FF24A701E7010590089407944E
:1007C00028F4360FE71EF81E491F511D660F771FCC
:1007D000881F991F0694A1F70590079428F4E70E47
:1007E000F81E491F561FC11D770F881F991F661FCE
:1007F0000694A1F70590079428F4F80E491F561F98
:10080000C71FD11D880F991F661F771F0694A1F778
:100810000590079420F4490F561FC71FD81F990F42
:10082000661F771F881F0694A9F78491109517708B
:1008300041F0D695C79557954795F794E7941A9543
:10084000C1F7E9E3F2E0689415901591359165914F
:10085000959105907FE27395E118F10A430B560BD1
:10086000C90BD009C0F7E10CF11E431F561FC91F69
:10087000D01D7EF4703311F48A95E6CFE8940150D0
:1008800030F0080F0AF40027021708F4202F2395F0
:10089000022F7A3328F079E37D932A95E9F710C087
:1008A0007D932A9589F606949795679537951795C0
:1008B0001794E118F10A430B560BC90BD00998F0B5
:1008C00023957E9173957A3308F070E37C9320131F
:1008D000B8F77E9170617D9330F0839571E37D93DD
:1008E00070E32A95E1F71124EF90FF900F911F918B
:1008F000CF91DF91992787FD909508959111F6C0CA
:10090000803219F089508550D0F70895FB01DC0141
:100910004150504088F08D9181341CF08B350CF49F
:10092000805E659161341CF06B350CF4605E861B53
:10093000611171F3990B0895881BFCCFDC01FC0158
:10094000672F71917723E1F7329704C07C916D9303
:1009500070836291AE17BF07C8F3089540D008F4C2
:1009600081E00895E89409C097FB3EF49095809546
:10097000709561957F4F8F4F9F4F9923A9F0F92F65
:1009800096E9BB279395F695879577956795B795E3
:10099000F111F8CFFAF4BB0F11F460FF1BC06F5FC9
:1009A0007F4F8F4F9F4F16C0882311F096E911C0DB
:1009B000772321F09EE8872F762F05C0662371F0FC
:1009C00096E8862F70E060E02AF09A95660F771F10
:1009D000881FDAF7880F9695879597F90895990FEC
:1009E0000008550FAA0BE0E8FEEF16161706E807F9
:1009F000F907C0F012161306E407F50798F0621B1A
:100A0000730B840B950B39F40A2661F0232B242BEE
:100A1000252B21F408950A2609F4A140A6958FEF0D
:100A2000811D811D08950BD07BC06CD028F071D042
:100A300018F0952309F05DC062C01124A5C081D0D3
:100A4000A0F3959FD1F3950F50E0551F629FF001E1
:100A5000729FBB27F00DB11D639FAA27F00DB11D3A
:100A6000AA1F649F6627B00DA11D661F829F2227C3
:100A7000B00DA11D621F739FB00DA11D621F839F4A
:100A8000A00D611D221F749F3327A00D611D231F20
:100A9000849F600D211D822F762F6A2F11249F576E
:100AA00050408AF0E1F088234AF0EE0FFF1FBB1F91
:100AB000661F771F881F91505040A9F79E3F510530
:100AC00070F017C061C05F3FECF3983EDCF3869591
:100AD00077956795B795F795E7959F5FC1F7FE2BDB
:100AE000880F911D9695879597F9089599278827DE
:100AF000089597F99F6780E870E060E008959FEFA0
:100B000080EC089500240A941616170618060906A4
:100B1000089500240A941216130614060506089573
:100B2000092E0394000C11F4882352F0BB0F40F4FB
:100B3000BF2B11F460FF04C06F5F7F4F8F4F9F4F3B
:100B4000089557FD9058440F551F59F05F3F71F0BD
:100B50004795880F97FB991F61F09F3F79F0879524
:100B60000895121613061406551FF2CF4695F1DFAD
:100B700008C0161617061806991FF1CF869571053D
:100B8000610508940895E894BB2766277727CB0171
:100B900097F90895F999FECF92BD81BDF89A9927EA
:100BA00080B50895262FF999FECF1FBA92BD81BD59
:100BB00020BD0FB6F894FA9AF99A0FBE01960895DF
:100BC000052E97FB16F400940FD057FD05D024D0C6
:100BD00007FC02D046F408C0509540953095219509
:100BE0003F4F4F4F5F4F0895909580957095619559
:100BF0007F4F8F4F9F4F089531D0A59F900DB49F89
:100C0000900DA49F800D911D11240895B7FFF4CF7E
:100C1000F3DF821B930B0895A1E21A2EAA1BBB1BC4
:100C2000FD010DC0AA1FBB1FEE1FFF1FA217B307B8
:100C3000E407F50720F0A21BB30BE40BF50B661FCE
:100C4000771F881F991F1A9469F760957095809592
:100C500090959B01AC01BD01CF010895A29FB00109
:100C6000B39FC001A39F700D811D1124911DB29FE0
:100C7000700D811D1124911D08955058BB27AA277E
:100C80000ED04ECF3FDF30F044DF20F031F49F3FF5
:100C900011F41EF434CF0EF4E095E7FB2ACFE92FD0
:100CA00050DF80F3BA17620773078407950718F0BF
:100CB00071F49EF568CF0EF4E0950B2EBA2FA02D9F
:100CC0000B01B90190010C01CA01A0011124FF27F9
:100CD000591B99F0593F50F4503E68F11A16F040F4
:100CE000A22F232F342F4427585FF3CF46953795F3
:100CF0002795A795F0405395C9F77EF41F16BA0BB8
:100D0000620B730B840BBAF09150A1F0FF0FBB1F65
:100D1000661F771F881FC2F70EC0BA0F621F731FAE
:100D2000841F48F4879577956795B795F7959E3F0B
:100D300008F0B3CF9395880F08F09927EE0F979599
:100D400087950895DFDE58F080E891E009F49EEF82
:100D5000E0DE28F040E851E059F45EEF09C0CFCE64
:100D600012CFE92FE078EDDE68F3092E052AC1F3F2
:100D7000261737074807590738F00E2E07F8E025E1
:100D800069F0E025E0640AC0EF6307F8009407FA11
:100D9000DB01B9019D01DC01CA01AD01EF9343D034
:100DA000BFDE0AD05F91552331F02BED3FE049E4DF
:100DB00050FD49EC63CF0895DF93DD27B92FBF774E
:100DC00040E85FE31616170648075B0710F4D92FB3
:100DD0000ED19F938F937F936F9352D2EEE4F1E005
:100DE000DDD09EDE2F913F914F915F9128DEDD2374
:100DF00049F09058A2EA2AED3FE049EC5FE3D07851
:100E00005D274DDFDF918CCE0CD08ACE82DE40F0A4
:100E100079DE30F021F45F3F19F06BCE5111B4CE82
:100E20006ECE8FDE98F39923C9F35523B1F3951B4A
:100E3000550BBB27AA2762177307840738F09F5FFB
:100E40005F4F220F331F441FAA1FA9F333D00E2E6A
:100E50003AF0E0E830D091505040E695001CCAF7D7
:100E600029D0FE2F27D0660F771F881FBB1F26179C
:100E700037074807AB07B0E809F0BB0B802DBF016F
:100E8000FF2793585F4F2AF09E3F510568F031CEFF
:100E90007BCE5F3FECF3983EDCF3869577956795C4
:100EA000B795F7959F5FC9F7880F911D9695879520
:100EB00097F90895E1E0660F771F881FBB1F62173F
:100EC00073078407BA0720F0621B730B840BBA0BFD
:100ED000EE1F88F7E095089519F40EF00ACE53CE70
:100EE0000ECE37DEC8F39638C0F707F80F92E894B5
:100EF0002BE33AEA48EB5FE7A4DD0F920F920F92E3
:100F00004DB75EB70F92FBD0EBE7F1E047D04F91C2
:100F10005F91EF91FF91E595EE1FFF1F49F0FE579E
:100F2000E0684427EE0F441FFA95E1F74195550B11
:100F300067D00F9007FE5BC0089504D06894B1118C
:100F400023CE089506DE88F09F5790F0B92F992799
:100F5000B751A0F0D1F0660F771F881F991F1AF0C4
:100F6000BA95C9F712C0B13081F00DDEB1E0089535
:100F70000ACE672F782F8827B85F39F0B93FCCF3B6
:100F8000869577956795B395D9F73EF490958095BA
:100F9000709561957F4F8F4F9F4F0895DF93CF934B
:100FA0001F930F93FF92EF92DF927B018C01689465
:100FB00005C0DA2EEF0143DDFE01E894A5912591ED
:100FC000359145915591AEF3EF0169DEFE01970130
:100FD000A801DA9479F7DF90EF90FF900F911F91BD
:100FE000CF91DF910895FBDC08F48FEF08959B010A
:100FF000AC0160E070E080E89FE306CF7ACD47C1A6
:10100000A8DDE8F39923D9F3940F511DBBF3915058
:10101000504094F059F0882332F0660F771F881FF4
:1010200091505040C1F79E3F510544F7880F911DE4
:101030009695879597F908955F3FACF0983E9CF0A0
:10104000BB27869577956795B79508F4B16093951A
:10105000C1F7BB0F58F711F460FFE8CF6F5F7F4F08
:101060008F4F9F4FE3CF90CD0AD029ED3BE54EED5A
:101070005EE3D9CC0EF00BC142CD68943ACD69DD68
:10108000C8F39923D1F3C6F3DF93CF931F930F9344
:10109000FF92C92FDD2788232AF02197660F771F3B
:1010A000881FDAF720E030E040E85FEB9FE3883903
:1010B00020F0803E30F021968F77E0DDE3EAF1E02A
:1010C00003C0DCDDE0EDF1E069DF8B01BE01EC0186
:1010D000FB2E6F5771097595771F880B990B44DCB0
:1010E00028E132E741E35FE3AADCAF2D9801AE01CE
:1010F000FF900F911F91CF91DF91D1DD11CDFA01BA
:10110000DC01AA0FBB1F9B01AC01BF5728F42227AB
:101110003327442750781FC0B75188F4AB2F0024E1
:10112000469537952795011CA395D2F3002069F0C9
:10113000220F331F441FB395DAF30DD09ECD6130DB
:101140007105A0E88A07B94630F49B01AC01662717
:10115000772788279078309621F020833183428347
:1011600053830895FA01EE0FFF1F309621053105D4
:1011700099F16115710561F48038BFE39B0749F16E
:1011800068949038810561F08038BFEF9B0741F08B
:10119000992342F5FF3FE1053105210511F1E8945E
:1011A0000894E795D901AA2329F4AB2FBE2FF85F45
:1011B000D0F310C0FF5F70F4A695E0F7F73950F058
:1011C00019F0FF3A38F49F779F930CD00F9007FCEB
:1011D000905808953EF093CC60E070E080E89FE383
:1011E00008954FE79F775F934F933F932F9347DF88
:1011F0002F913F914F915F9116DC73CE11F40EF455
:101200007ECC45C0A6DCD0F39923D9F3CEF39F570B
:10121000550B87FF4AD00024A0E640EA9001805891
:101220005695979528F4805C660F771F881F20F0ED
:1012300026173707480730F4621B730B840B2029ED
:1012400031294A2BA69517940794202531254A2742
:1012500058F7660F771F881F20F0261737074807B3
:1012600030F4620B730B840B200D311D411DA095D2
:1012700081F7B901842F9158880F96958795089525
:101280009B01AC01D0CBABDB880B990B08959F3F42
:1012900031F0915020F4879577956795B795880F31
:1012A000911D9695879597F9089591505040660F36
:1012B000771F881FD2F70895DB018F939F939CDCE3
:1012C000BF91AF91A29F800D911DA39F900DB29FE2
:1012D000900D11240895AA1BBB1B51E107C0AA1F42
:1012E000BB1FA617B70710F0A61BB70B881F991FC7
:1012F0005A95A9F780959095BC01CD01089597FB6B
:10130000072E16F4009406D077FD08D0E4DF07FC22
:1013100005D03EF4909581959F4F08957095619505
:101320007F4F0895EE0FFF1F881F8BBF0790F69128
:10133000E02D19940F93083090F0982F872F762F77
:10134000652F542F432F322F22270850F4CF220F1E
:10135000331F441F551F661F771F881F991F0A954B
:10136000B2F70F91089597FB10F8169400080F93A9
:10137000083098F00850232F342F452F562F672F11
:10138000782F892F902DF4CF059497958795779591
:10139000679557954795379527950A95AAF70F9121
:1013A0000895CF93DF938230910510F482E090E0AE
:1013B000E0919F10F091A01020E030E0C0E0D0E07C
:1013C000309711F14081518148175907C0F04817F3
:1013D000590761F482819381209719F09B838A8356
:1013E0002BC09093A01080939F1026C0211531052B
:1013F00019F04217530718F49A01BE01DF01EF01FB
:101400000280F381E02DDCCF2115310509F1281B85
:10141000390B2430310590F412968D919C911397DD
:101420006115710521F0FB019383828304C09093C1
:10143000A01080939F10FD01329644C0FD01E20F81
:10144000F31F81939193225031092D933C933AC01D
:1014500020919D1030919E10232B41F42091E004A7
:101460003091E10430939E1020939D102091DE0472
:101470003091DF042115310541F42DB73EB740917D
:10148000E2045091E304241B350BE0919D10F09190
:101490009E10E217F307A0F42E1B3F0B2817390705
:1014A00078F0AC014E5F5F4F2417350748F04E0FC0
:1014B0005F1F50939E1040939D108193919302C0A3
:1014C000E0E0F0E0CF01DF91CF9108950F931F93FB
:1014D000CF93DF93009709F48CC0FC0132971382FD
:1014E000128200919F101091A0100115110581F436
:1014F00020813181820F931F20919D1030919E1089
:101500002817390779F5F0939E10E0939D1071C06C
:10151000D80140E050E0AE17BF0750F412962D916D
:101520003C911397AD012115310509F1D901F3CF94
:101530009D01DA013383228360817181860F971FB9
:101540008217930769F4EC0128813981260F371F30
:101550002E5F3F4F318320838A819B8193838283D7
:10156000452B29F4F093A010E0939F1042C01396EE
:10157000FC93EE931297ED01499159919E01240F2E
:10158000351FE217F30771F480819181840F951F55
:10159000029611969C938E938281938113969C93CD
:1015A0008E931297E0E0F0E0D80112968D919C9115
:1015B0001397009719F0F8018C01F6CF8D919C914B
:1015C00098012E5F3F4F820F931F20919D10309105
:1015D0009E102817390769F4309729F41092A0104B
:1015E00010929F1002C01382128210939E100093DB
:1015F0009D10DF91CF911F910F9108956F927F926F
:101600008F929F92AF92BF92CF92DF92EF92FF9212
:101610000F931F93CF93DF93EC01009781F4CB01DD
:10162000DF91CF911F910F91FF90EF90DF90CF90BE
:10163000BF90AF909F908F907F906F90B2CEFC0143
:10164000E60FF71F9C0122503109E217F30708F457
:10165000A8C0D9010D911C91119706171707A8F082
:101660000530110508F49BC0C80104978617970739
:1016700008F495C002501109061B170B0193119332
:101680006D937C93CF0122DF8AC05B01A01AB10A5F
:101690004C01800E911EA0919F10B091A01040E0CF
:1016A00050E0E12CF12C109709F44AC0A815B905B7
:1016B000D1F56D907C901197630182E0C80ED11C2A
:1016C000CA14DB0480F1A3014A195B096A0182E0B4
:1016D000C80ED11C1296BC9012971396AC91B5E02F
:1016E000CB16D10440F0B282A38351834083D90149
:1016F0006D937C930AC00E5F1F4FC301800F911F33
:10170000F90191838083EB2DFA2FE114F10431F07C
:10171000D7011396FC93EE93129741C0F093A0105B
:10172000E0939F103CC08D919C91119748175907E9
:1017300008F4AC017D0112960D90BC91A02DB3CFA1
:1017400080919D1090919E1088159905E1F446179F
:101750005707C8F48091DE049091DF04009741F4AC
:101760008DB79EB74091E2045091E304841B950B22
:10177000E817F907B0F4F0939E10E0939D10F9017B
:10178000718360830CC0CB010CDE7C01009749F0B3
:10179000A801BE011BD0CE0199DEC70104C0CE0155
:1017A00002C080E090E0DF91CF911F910F91FF90F8
:1017B000EF90DF90CF90BF90AF909F908F907F90F1
:1017C0006F90089581E090E0F89447C0FB01DC0140
:1017D00002C001900D9241505040D8F70895FB018E
:1017E000DC0101900D920020E1F70895FB01DC017E
:1017F0004150504030F08D910190801919F4002033
:10180000B9F7881B990B0895FB01DC01415050404A
:1018100048F001900D920020C9F701C01D9241507F
:101820005040E0F70895FB0151915523A9F0BF0105
:10183000DC014D9145174111E1F759F4CD010190BB
:10184000002049F04D9140154111C9F3FB014111B0
:10185000EFCF81E090E00197089517E0CEE5D7E063
:1018600000E005C0802FFE015DDD2196011DCF3512
:0C187000D10780E00807B1F7F894FFCF23
:10187C000000F0410AD7C3BF9A99F93F0000A0407D
:10188C000108000100020003000400050006000826
:10189C00000800A4707D3F0000A841CDCC2C400A6C
:1018AC00D78B4000803B450000803F6666A63FA179
:1018BC006733BD7C8C0100010000754400808944B5
:1018CC0001180408101C000000566F6C74616765E9
:1018DC0000000000000000000000000000000000FC
:1018EC0054656D702B48756D000000000000000001
:1018FC0000000000000000495220466C616D65003C
:10190C000000000000000000000000000000476123
:10191C007300000000000000000000000000000048
:10192C0000000000007048000000000000000000F3
:10193C0000000000000000000000000054757262FE
:10194C006964697479000000000000000000000068
:10195C00000000434F3200000000000000000000B7
:10196C00000000000000000000004F3200000000EA
:10197C00000000000000000000000000000000005B
:10198C000049522054656D700000000000000000FA
:10199C000000000000000000536F756E6400000032
:1019AC0000000000000000000000000000000050DB
:1019BC004D000000000000000000000000000000CE
:1019CC00000000000000434834000000000000004C
:1019DC0000000000000000000000000000416C63EB
:1019EC006F686F6C00000000000000000000000039
:1019FC0000000000434F0000000000000000000049
:101A0C000000000000000000000000483200000050
:101A1C0000000000000000000000000000000000BA
:101A2C0000004F7A6F6E650000000000000000009F
:101A3C0000000000000000000048325300000000CD
:101A4C00000000000000000000000000000000008A
:101A5C004E483300000000000000000000000000B1
:101A6C00000000000000002000000000000000004A
:101A7C00000000000000000000000000000020003A
:101A8C00000000000000000000000000000000004A
:101A9C00000000000055560000000000000000008F
:101AAC000000000000000000000000005468657297
:101ABC006D6F6D65746572730000000000000000AE
:101ACC000000004D6F74696F6E0000000000000094
:101ADC000000000000000000000037003900080082
:101AEC003D003E003F00390038003700380001014E
:101AFC003E003D0062BE3C3993522A409352AA40AC
:101B0C0017D900418C968141B73AC9418B899D3ECA
:101B1C000000A0410000204200007042133BF14243
:101B2C00ECC43A430000804027882640643B5F3E6B
:101B3C0021B0B23E3D002E3032342F3133353132AC
:101B4C00334134353642373839432A302344000088
:101B5C00A11080005E00BC0077016400000008004A
:101B6C003700380039003F003E003D0011001000E6
:101B7C00000000001148544798475748C947A747E9
:101B8C00BB47000000002455F454F154E53EE854E2
:101B9C00D454C55400000000D34C944C634C00004A
:101BAC000000CE3E5447F154F054DA41BA3E573F50
:101BBC00383F00000000000000008A767544754430
:101BCC0000000000BC5553558A764949FC48070073
:101BDC002D37002D38002D39002D3130002D3131AD
:101BEC00002D34002D35002D33002D32002D310009
:101BFC0073657269616C3A200042543A20005300BC
